:1000000000400020A1710000E1710000E3710000D8
:1000100000000000000000000000000000000000E0
:10002000000000000000000000000000E57100007A
:100030000000000000000000E7710000E97100000E
:10004000EB710000DD5200001D760000EB71000036
:10005000EB71000000000000EB710000EB7100008C
:10006000EB710000F5790000D5310000EB71000064
:10007000EB710000EB710000EB710000EB71000010
:10008000EB710000A1760000EB710000EB71000045
:10009000EB710000EB710000EB710000EB710000F0
:1000A000EB710000EB710000000000000000000098
:1000B0000000000000000000000000000000000040
:1000C00010B5064C2378002B07D1054B002B02D02E
:1000D000044800E000BF0123237010BD640200202B
:1000E0000000000090E50000044B10B5002B03D089
:1000F0000349044800E000BF10BDC04600000000F6
:100100006802002090E50000164B002B00D1144B34
:100110009D46402292029A1A924600218B460F4633
:100120001348144A121A0BF0B1FA0F4B002B00D0EF
:1001300098470E4B002B00D0984700200021040068
:100140000D000D48002802D00C4800E000BF0BF065
:100150005DFA2000290007F0B3FA0BF031FAC0462F
:100160000000080000400020000000000000000027
:1001700064020020C42F00200000000000000000E6
:1001800002000120104011D1042A0ED91368180969
:1001900080B2002809D001388000031D11180979A8
:1001A000002902D001309842F8D170470020FCE7C6
:1001B0000378002B03D05AB2002A01DB01307047CC
:1001C0003F229343C03B59424B41C01803789343AD
:1001D000802BF4D10130F9E710B500240378002B0F
:1001E00001D1200010BDFFF7E3FF0134F6E770B541
:1001F000002204000D00411C092003F015FB00281B
:1002000006D001236200134343600023A34200DBB6
:1002100070BD9A00A958821891600133F6E770B555
:10022000012803DC1C2001F045F870BD01230D6896
:1002300011201D42F7D04868184206D1042804D97D
:100240000F2302681340042B01D00E20EBE703F0CC
:1002500049F96D100400002D03DDFFF7BDFFA84232
:1002600006DA1220DFE72000FFF7A2FF0400013DBD
:10027000012DF8D120787F2809DDDF280BDCF82359
:100280003F22DB00800118406378134018430123AC
:1002900040001843C9E7EF280BDCFC226378120109
:1002A0009B0113403F220007000C0343A07810403D
:1002B000ECE7F72812DCFC22637892021B03134060
:1002C000E0228004520310403F221843E378134099
:1002D000FC220343A07812018001E8E7012040429C
:1002E000D5E7F8B54D680F00EB0706D4042D04D907
:1002F0000F232E683340092B03D00B2000F0DAFFC8
:10030000F8BD6B683609B6B25C10731EA3420FD8F5
:100310000321200009F076F86421642803DC010041
:10032000032800DA03212800891903F0AFFA050039
:100330002B6800201B099BB2013B9C42E0D23A682B
:10034000A31C9B005A510123013464001C436C60C0
:10035000D6E7F0B585B0012803DC1C2000F0AAFF29
:1003600012E001274B683A000093022806D08B6800
:100370003B4203D05F10002F00DC17000124009BDC
:10038000234203D00120404205B0F0BD009B042B66
:10039000F8D91B680D680F2619003140042921D1B6
:1003A000254205D1042D03D92B681E40042E01D00F
:1003B0000E20D3E70098FFF7E3FEB842E2DB009897
:1003C00003F090F80600280003F08CF80100781E76
:1003D00030180BF011FD0028D4D0801B01304000F4
:1003E0002043D1E709293DD1009B5B685B10019355
:1003F0009F42C7DC25422CD1042D2AD92B683340DB
:10040000042B26D1280003F06DF8039602907E1C81
:10041000009AB300D058854201D17800E0E720422D
:100420000ED104280CD90368039A1340042B07D17A
:1004300003F058F8010002980BF0A8FC0028ECD05B
:10044000019B37009E42E2DD9CE71F00019B9F421B
:1004500098DC7B1C00999A008A58AA42F5D1780052
:100460000124BDE7032900D08CE71A0992B25B0F83
:1004700092000B40D31A01939F4200DD82E7254290
:1004800029D1042D27D92A681640032E19D1100925
:1004900080B2520F800032402C1D801A019B26181A
:1004A0001B1A0193009B781E0433019A904200DDD1
:1004B00068E722001918B2420FD316D1013040006C
:1004C000CEE7042E07D1280003F00CF80400280022
:1004D000FFF756FEE2E70F2040E70D78AC461578AF
:1004E000AC4502D101310132E5E70130DDE710B55D
:1004F00002F0DCFF43000120184310BDC30711D4F4
:1005000004280FD90F2302681340032B0AD1194086
:100510000133591AC0234907DB051940024B1A4021
:10052000114301607047C046FFFFFF9FF7B507000A
:100530000E001C20012F06DD4C68012322001A400A
:10054000009203D10D2000F0B5FE53E0022F02D03F
:100550008A681A42F6D0012335681D4200D0A9E00E
:10056000042D00D8A6E01C41002C00DC1C000F204C
:1005700029680840092828D16B685B100093022F76
:1005800005D0B368009A5B109A4200DD0093009B8F
:1005900001221D1B0135EB43DB171D40691C09209F
:1005A00003F042F9071E09D001236D001D4303002B
:1005B0003268083345600099A14201DA3800FEBD77
:1005C0000134A100515802C3F5E7042845D12800A1
:1005D00002F088FFFFF700FE0190022F04D0B368FD
:1005E0005B10984200DD0193019BA34204DA0020D6
:1005F00003F08CF90700E1E7280002F073FF070021
:10060000009BA34221DB2800009702F06BFF05004E
:100610003800FFF7CDFD019B01340700A342F7DA54
:10062000009BC41A200003F071F9071EC6D002F027
:1006300059FF0190306802F055FF2200009B591BC2
:10064000411801980BF006F8B8E73800FFF7B0FD45
:10065000009B070001330093D2E703282AD10B093E
:100660009BB2490F9B000140591A022F04D0B26877
:100670005210914200DD1100A14205DA0022032050
:10068000110003F0D1F8B5E703200E1B331DD91775
:100690000140C9188910002203F0C6F8071E00D1D6
:1006A0008CE7013631000334FFF728FF381D291984
:1006B0003200C7E7212046E7F8B5002805DC1C20FA
:1006C00000F0F8FD05002800F8BD01260C68264062
:1006D0000FD06410E343DB171C40E11C891000229B
:1006E000032003F0A1F8051EEDD02100FFF706FF5F
:1006F000E9E7042C01D80025E5E70F232268134021
:10070000042B1BD12000FFF73BFDC31C0700032077
:10071000D9170140C9188910320003F085F8051E69
:10072000D1D03900FFF7EAFE200002F0DBFE2B1DDE
:1007300001003A0018000AF08DFFC4E7092BDAD156
:100740000320636832005F10FB1CD9170140C918F1
:10075000891003F069F8051ECDD03900FFF7CEFEF1
:10076000FF20BE42AFDA0122B300E3189B681342B8
:1007700008D01341FF2B00DD0300D943C917AA1984
:100780000B4013710136ECE710B57F2902DC0170D4
:10079000013010BD1A4B99420CDC40238A115B4298
:1007A000134303703F230B4080214942194341709A
:1007B0000230EEE7134B994210DC20230A135B4210
:1007C00013433F24802203708B1152422340214067
:1007D00013430A43437082700330DAE70A4B9942AD
:1007E000D7DCF0230370603B4370113B8A11FF3B61
:1007F0001A4382703F2211401943C1700430C8E788
:10080000FF070000FFFF0000FF0F0100F0B50D0023
:1008100085B0002803DC1C2000F04CFD0DE00968C9
:100820000122080010400AD002AC11412000FFF75D
:10083000ABFF011B200003F075F804001AE0042947
:100840003FD90F230C682340092B3AD14B685B102A
:10085000019303239C46019B9A420EDD03F056F858
:10086000041E07D02E68012502F03CFE2F00019BDC
:100870009D421DDD200005B0F0BD01329300CC5833
:100880000123234001D10D20C6E764107F2C0DDD2C
:100890000D4E0223B44209DD0C4E6346B44205DD21
:1008A00000270B4EE30FA6427B419B00C018D2E706
:1008B0000135AB00F1583942E5D04910FFF764FF2C
:1008C000D5E72120A8E7C046FF070000FFFF000092
:1008D000FF0F010010B504000120084010D10429C9
:1008E0000DD90F230A681340042B08D1080002F029
:1008F000F9FD010020000BF049FA4342584110BDB8
:100900000020FCE7F7B50F00012803DC1C2000F0F5
:10091000D1FCFEBD01264D682E4006D1042D04D920
:100920000F222B681A40092A01D00B20EFE76A68D2
:100930001B099BB25410A34200D85C1E39681E48A4
:10094000FFF7C8FF01230190002813D139681B4825
:10095000FFF7C0FF002811D0002C0DD00123621C2E
:10096000013C9C409200535123436B6004E00136EC
:10097000B200AB50B442FADA0020CAE73B680D205F
:10098000DA07C4D55B10002B11DD9C420FDB9B0006
:10099000A200291DEB1889180433994209D10123BB
:1009A000013C9C40AA181C4353606C60E4E7122091
:1009B000ADE758681860EFE71FCD000023CD0000B9
:1009C000002310B50C000B70C30705D50D4942106C
:1009D00020000BF09FF908E00B49002802D0042802
:1009E00004D10A4920000BF0B5F910BD0428FCD948
:1009F0000F2302681340042BF7D102F073FD044962
:100A00000200E5E724D7000028CD00002ECD00002D
:100A100033CD0000F0B593B0060002911C20012EEA
:100A20001DDD029B01251B681C002C4000D0ADE0A1
:100A3000042B00D8E6E01A680F231A40092A4AD18D
:100A40000394039A029992008A5817002F4005D107
:100A5000042A03D910681840092806D0222000F083
:100A600029FC0190019813B0F0BD52685210A418EF
:100A7000039A013203929642E3D1611C012202F0F3
:100A8000D3FE0190002802D100230193EAE7019BE5
:100A90006400190025435D600831029ABB00D058FC
:100AA00002684368120992B25B109A4200D8531E42
:100AB0000022934209DCDA43D21713409B00C91885
:100AC000039B01379F42E8DBCCE794000519AD6832
:100AD00001320D51EDE72700032A59D10193029A03
:100AE000BB00D3582B42B9D1042BB7D91868019950
:100AF0000140032939D1020992B2430F92000B4001
:100B0000D31A1C190137BE42E9D10320E31CD917BF
:100B10000140C9188910002202F086FE01900028C9
:100B2000B2D000252100FFF7E9FC019B1E1D029AAF
:100B3000AB00D45801231C421FD1042C1DD90F2116
:100B400023681940032918D1180980B25B0F80006F
:100B50000B40C01A0023834213DBC343DB1718404A
:100B600001353618BD42E2DB7CE7042900D075E789
:100B70001800FFF705FB2418C4E72000FFF700FB6F
:100B8000E8E7E2181279F2540133E4E700273C0069
:100B90000F25029ABB00D3580122134234D1042BF3
:100BA00032D9186801002940042935D11800FFF70F
:100BB000E7FA24180137BE42EBD1200002F0A6FE6E
:100BC0000190002800D15FE7029FB600BB19041D09
:100BD000029301233D681D4229D1042D27D90F26F8
:100BE0002B681E40042E37D12800FFF7C9FA0600F3
:100BF000280002F077FC0100200032000AF02AFDF4
:100C0000A41922E02700C3E7180005A9FFF7D8FEC2
:100C100005A80BF0C5F8CCE7032900D01EE70209B0
:100C200092B2430F92000B40D31A1C19C2E705A9D8
:100C30002800FFF7C5FE05A80BF0B2F805A90500CE
:100C4000020020000AF006FD6419029B0437BB4233
:100C5000BFD10023237005E7032EF6D11A0992B203
:100C60005B0F92001E40961B291DC5E7F0B50D00D5
:100C700095B0002806DC1C2000F01CFB04002000BE
:100C800015B0F0BD0C68012123000B40009306D184
:100C9000042C04D922680F331A40092A01D00B20F2
:100CA000EAE7626852100392002A03DC009802F01F
:100CB0002DFEE3E73F4A019201280BD06868084205
:100CC00008D1042806D902681340042B02D102F08F
:100CD00009FC019001980BF063F806000F27039BB5
:100CE0000834013B04935E43039B02909B001B1955
:100CF000059301232068184251D104284FD9036875
:100D00003B40042B52D1FFF73BFA059B04343618C5
:100D1000A342EED1300002F0F9FD041EAFD02B68E3
:100D20000593029B002B03D0686802F0DBFB019067
:100D3000200002F0D7FB0500009B059A9B00D3180A
:100D40009F68380002F0CEFB012306001F4201D14C
:100D5000042F04D807A93800FFF732FE07AE300091
:100D60000BF01EF807000200310028000AF072FCA8
:100D7000029BED19002B0AD0049B009A934206DDDA
:100D80002800029A01990AF065FC029BED18009B6D
:100D900001330093009A039B9342CDD16FE707A9DB
:100DA000FFF70EFE07A80AF0FBFFAEE702F09AFB82
:100DB000F9E7C046C7D1000010B50024A04207DD06
:100DC0000B6801341C4003D05C10E343DB171C406C
:100DD000611C0122092002F027FD002803D0012315
:100DE00064001C43446010BD0A6870B51000012502
:100DF000284034D1042A32D90F24136849681C4092
:100E0000092C17D154681B099BB22C41A34200D86E
:100E10005C1E844205DC02200133984206DB002080
:100E20000FE085005519A9600130F2E784001151E7
:100E30000130F2E7032C12D1294203D1132000F034
:100E400039FA70BD4910FF29F8D81B099BB204324A
:100E50009B00D3189342E2D911700132FAE70B20BC
:100E600000F028FADBE700000123F7B500254E6803
:100E70000F0033400093AB420ED11D00042E0BD95E
:100E80000F2233681A40092A10D172681B099BB2DD
:100E90005510AB4200D85D1E3968CB0717D54C10F2
:100EA000002C01DDA5421DDA122032E0042A04D113
:100EB0003000FFF765F90500EEE7009D032AEBD14E
:100EC0001D09ADB25B0FAD001340ED1AE4E72E48EB
:100ED000FFF700FD002814D00AF0B8FE290008F042
:100EE00077FB4C1C009B002B4CD1042E4AD9326856
:100EF0000F331340092B10D10134A400A459200052
:100F0000FEBD39682148FFF7E5FC2C000028E9D137
:100F1000113000F0CFF90400F1E7042B2AD13000A2
:100F200002F0E0FA0500FFF757F9A042BCDB012C04
:100F30001ADC300002F0D6FA00902800FFF738F9EA
:100F4000461B300002F0E2FC041ED8D002F0CAFAC0
:100F50000190786802F0C6FA009B3200E91A411845
:100F600001980AF077FBCAE72800FFF721F9013C56
:100F70000500DCE7032B05D13419E478023B64005B
:100F80001C43BCE70B20C4E718CD000023CD0000B4
:100F9000F7B54D680F002A0001210A402FD1042D1A
:100FA0002DD90F242B68BE681C40092C14D1696808
:100FB0001B099BB24C100192A34200D85C1E3968F9
:100FC0002A48FFF787FC00282DD00F232A681340FA
:100FD000092B1DD1012317E0032C10D10E4203D1A0
:100FE000132000F067F9FEBD72100192FF2AF7D8B6
:100FF0001A0992B25B0F92001C40141BDFE70B2012
:10100000EFE701339A00AE509C42FADA0020EAE79B
:10101000032BFBD12B0001335A1BA242F6DC6A469C
:101020001279DA70F7E73968CB0706D5491000293D
:1010300001DD8C4209DA1220D3E70D48FFF74AFCA4
:101040002100002801D11130CBE70F232A6813407B
:10105000092B03D1013189004E51D7E7032BD5D19C
:101060006B461B796D18EB70D0E7C0461FCD0000B2
:1010700023CD000010B50124086820421AD10428AD
:1010800018D90F2102681140092901D1406810BD0B
:10109000032908D113099BB2500F9B000840181A6E
:1010A00040002043F3E7042904D102F01BFAFFF7C4
:1010B00093F8F5E70B2000F0FDF8E8E710B5034AD8
:1010C0000B21034804F0CCF910BDC046C0CC000091
:1010D000B8CC000000207047042070470120704702
:1010E00010B5002002F012FC10BD00207047002057
:1010F0007047002070470020704700207047002094
:1011000070470020704700207047000010B5034A68
:101110000C21034804F0A4F910BDC046A8CD00007E
:1011200008CE000010B50124044002D04410200075
:1011300010BD042810D90F2302681340042B07D1D7
:1011400002F0D0F921000A220AF0F2FE0400EEE7D4
:10115000032B01D10430F5E70D22014B1A70E6E7AD
:10116000A4020020012210B5024018D1042802D99F
:1011700003681A0992B201230B4012D1042902D943
:101180000B681B099BB20024934206D104309B00DC
:101190000431C318984206D30124200010BD002258
:1011A000E9E70023EFE704780A78002C01D1002A50
:1011B000F2D0013001319442ECD00024EDE7000080
:1011C000F7B50700009101933049314B002A02D056
:1011D00002220A70013A00261A601B68CE54BE42F1
:1011E00000DBF7BD009AB300D058294B274D1C688F
:1011F000C8239B0065191C1B0123184206D0254AF1
:101200004310210028000AF053FD09E0224A00287B
:1012100002D004281BD1214A210028000AF048FDF1
:101220001A4C20000AF0BCFD194A019B1060002BEB
:101230000BD07B1EB34208DD194B984205D8431CE6
:101240001360202222540022E2540136C7E704280A
:1012500019D90F2301680B40042B04D102F042F985
:10126000104A0300CDE7092B03D143680E4A5B10F7
:10127000C7E7032B08D10A0992B2490F92000B402D
:10128000D31A0A4ABDE70123094ABAE7A50200209A
:10129000C805002024D7000028CD00002ECD000076
:1012A0001F0300004FDD000078D0000087D0000051
:1012B00092D00000014B187000207047A40200205B
:1012C00070B501F06BFE094C0100251D1F2228009E
:1012D0000AF07EFD28000AF063FD04230430800834
:1012E000000118432060200070BDC046800200202D
:1012F000C368F0B59D00836889B05D190300183399
:1013000006930369069A9F00069B0290DF194369C2
:1013100001939B00D3180393CD4B1B78002B26D150
:101320007F222B68CB491C1213409B005B5804356D
:1013300001929F46029B587804F0C0FC0023029A59
:10134000137027E0C24B1B78002B10D12B68019A39
:101350001C121340BF4A9B009B580435E9E7069BCB
:101360003A1DD11ABA4BD82928DD1A221A70029BCD
:10137000B74C9B6821780193EA1A029B92109B78E4
:1013800012021A43029B587804F0A0FC0023029A30
:1013900023701370029B069A9B680193ED1A029BBF
:1013A000AD10DD60069BFE1A029BB6101E61039B0A
:1013B0009B1A029A9B10536109B0F0BD1B783C60E8
:1013C000002B01D01700D2E72B6801991C120B40AB
:1013D000A0499B005B5817000435AAE7069B3A1DFD
:1013E000D11A9B4BD82902DD1A221A70BFE7286850
:1013F0001B78291D3860002B02D017000D00B6E7BE
:101400006B6801991C120B4092499B005B581700B6
:1014100008358EE7069B3A1DD11A8D4BD82902DD7F
:101420001A221A70A3E7A4001B782C193C60002B29
:1014300001D017009BE72B6801991C120B408549CE
:101440009B005B581700043573E7069B3A1DD11AC1
:101450007F4BD82902DD1A221A7088E77E49A40042
:1014600061581B783960002B01D017007FE72B688B
:1014700001991C120B4077499B005B5817000435FB
:1014800057E7043F744B3A68A400E250704B1B7856
:10149000002B00D06BE72B68019A1C1213406D4A99
:1014A0009B009B58043544E76B4BA400E058FFF7C2
:1014B00039FE043F06003868FFF734FE3618012075
:1014C000654B76000643E650614B1B78002B00D03D
:1014D0004DE72B68019A1C1213405E4A9B009B58F3
:1014E000043526E7069B3A1DD11A594BD82902DD4F
:1014F0001A221A703BE70698039C0121A04202D2EF
:1015000021000C3909681B783960002B01D01700C5
:101510002DE72B6801991C120B404E499B005B582C
:101520001700043505E7069B3A1DD11A484BD82908
:1015300002DD1A221A701AE70699039881420FD227
:1015400003000C3B1B6845495B106418E41AA400B7
:1015500023583B603E4B1B78002B05D0170006E755
:10156000182119700023F4E72B6801991C120B4015
:1015700038499B005B5817000435DAE6069B039A4E
:10158000934219D213000C3B1B68344A043FA41841
:101590005B10E31A039A39689B0099502C4B1B7817
:1015A000002B00D0E3E62B68019A1C121340294A55
:1015B0009B009B580435BCE61822254B1A70EDE7BA
:1015C000069B039A93422DD2244B3E1FE31814002E
:1015D0000C3C04932368049A5B10D31A039A9B0073
:1015E0009858FFF79FFD07903068FFF79BFD246830
:1015F000049B64101C1B079BA4001F1801207F0084
:10160000039B0743E7503700114B1B78002B00D09A
:10161000ADE62B68019A1C1213400E4A9B009B58A2
:10162000043586E618220A4B1A70EDE7069B3A1D30
:10163000D11A074BD82902DD1A221A7097E60399AE
:10164000A40061581B783960002B09D017008EE682
:10165000A402002078CE0000902D0020FDFFFF3F67
:101660002B6801991C120B40D8499B005B5817004E
:1016700004355EE6043F039B3A68A400E250D44B75
:101680001B78002B00D072E62B68019A1C121340C5
:10169000CE4A9B009B5804354BE6039BA4001C19C3
:1016A0002368043F38685E10FFF73CFD36180120C0
:1016B000C74B76001B7806432660002B00D056E609
:1016C0002B68019A1C121340C04A9B009B5804359A
:1016D0002FE6069BA4003F1BBD4CBB420CD82378D1
:1016E000002B00D043E62B68019A1C121340B74A26
:1016F0009B009B5804351CE6B64801F0E3FE2378B6
:10170000002B00D033E62B68019A1C121340AF4A1D
:101710009B009B5804350CE6A300ED18002C00DA62
:1017200038E6AB4B1B78002B00D020E62B68019AE3
:101730001C121340A54A9B009B580435F9E5043F51
:101740003B68042B04D1A300ED18002C00DA21E63D
:101750009F4B1B78002B00D009E62B68019A1C12C6
:1017600013409A4A9B009B580435E2E5043F3B68CE
:10177000042B04D0A300ED18002C00DA0AE6944BE9
:101780001B78002B00D0F2E52B68019A1C12134045
:101790008E4A9B009B580435CBE53E1F3068C3073B
:1017A0000AD540100138002809DB01234000A400BD
:1017B00018432D193060EDE5FFF7B4FCF2E7844BD8
:1017C00037001B78002B00D0D1E52B68019A1C1242
:1017D00013407E4A9B009B580435AAE53A00069BBD
:1017E0000C32D31AD82B03DD1A22794B1A70BEE5BE
:1017F000FF2361005B001940FE3BFF3B194339604A
:10180000029906988968241204916D1A0299AD1004
:1018100089782D020D4303999D40091A891099403A
:101820001D430B43BB60029B7D609C70E4B26A4B1E
:10183000E4000392E358029A9360654A1278002A02
:1018400003D008331D00039F91E51D00019A9B689A
:101850000C351C1213405D4A9B009B58039F68E5A2
:101860003B1F1C68039A069B93422DD10A20E30775
:101870000CD4042C13D90F2322681340042B11D14C
:10188000200001F02FFE0AF08BFA0630643003F0DE
:1018900021FE00280FD1043D069B03937AE5072023
:1018A000042CF3D02000431E9841FA234042FF331A
:1018B00018400730EAE7029B2100587804F018FA34
:1018C0000023029A1370E7E7039B039A0C3B1B6803
:1018D00002995B109B00D31A0C3B1C601F1D130068
:1018E000083B1B685A108A70D2B23B49D2005B0099
:1018F00055589B0A029A9B009560ED18039B069A27
:10190000043B1B685B109B00D3180393304B1B7880
:10191000002B00D02BE52B68019A1C1213402B4A98
:101920009B009B58043504E53B1F1868FFF7FAFB42
:10193000A40006003F1B1E2827DC00280DDC244BDA
:101940001B78002B00D012E52B68019A1C12134063
:101950001E4A9B009B580435EBE401F00DFB033E4F
:10196000361801F009FB1D4B801B9842F9D8184B23
:101970001B78002B00D0FAE42B68019A1C1213404C
:10198000124A9B009B580435D3E40123029A13703A
:1019900001F0F2FA029B0A3886195E60FAE43B1FF6
:1019A0001868FFF7BFFBA40006003F1B002817DCE8
:1019B000074B1B78002B00D0D9E42B68019A1C122E
:1019C0001340024A9B009B580435B2E478CE0000D5
:1019D000A4020020A4D00000982500203F420F0060
:1019E000D64B984203DD1D22D54B1A70BFE401236C
:1019F000029A137001F0C0FAFA239B005E43029B27
:101A00000A3E30185860C5E4A300FF1A00232000E6
:101A10001A003900FFF7D4FBCA4ECB4C31682000C6
:101A200001F080FFC94B31681860200004F002F813
:101A30003168200004F063F9C14B1B78002B00D003
:101A400095E42B68019A1C121340C14A9B009B58D5
:101A500004356EE4BA4BA4001B783F1B002B00D06A
:101A600085E42B68019A1C121340B94A9B009B58CD
:101A700004355EE4029803F091FDB14B1B78002B16
:101A800000D074E42B68019A1C121340B04A9B00EA
:101A90009B5804354DE43B1F1B68002B3ED13B0097
:101AA0000C3B1B68DA072CD5390001225B1058006B
:101AB000083902430A60002B44DD0122590011431A
:101AC000381F01603900083909681141CB1A390003
:101AD0000C390968114224D09B189340A400134389
:101AE000039AA350964B1B78002B00D03FE42B6841
:101AF000019A1C121340964A9B009B580435FFF72D
:101B000018FC042B06D90F211A680A40092A01D1B2
:101B10005B68C9E719228A4B1A7028E45B10013B05
:101B2000C9E7042909D90F200A680240092A04D10B
:101B300002339B005B58A400D2E71922804B1A7035
:101B4000FFF715FC0435CDE7A300069AFB189B1A96
:101B5000D82B13DC0122631E002C14DC784B1B787D
:101B6000002B01D0FFF703FC2B68019A1C121340D5
:101B7000774A9B009B580435FFF7DBFB1A22704B1A
:101B80001A70FFF7F4FB3A601C000437E3E7069A8B
:101B90003B1D9B1A6A4ED82B03DD1A233370FFF7C7
:101BA000E6FB069B039AA40093422AD23B1F1868C7
:101BB000FFF7B8FA011E21DD039B0C3B1A68521097
:101BC00082421BDB9007801A624B4018C018039BAF
:101BD0008000C2583B1B1A60594B3F1B1B780437CF
:101BE000002B01D0FFF7C3FB2B68019A1C12134096
:101BF000574A9B009B580435FFF79BFB202333700B
:101C0000EAE71823FBE7514BA4001A683B1B1F00AF
:101C10001A604B4B04371B78002B01D0FFF7A7FB52
:101C20002B68019A1C121340494A9B009B580435AB
:101C3000FFF77FFB3B1F1A68042A11D1A4002D195E
:101C40003F4B1B78002B01D0FFF791FB2B68019ACB
:101C50001C1213403E4A9B009B580435FFF769FB5A
:101C60001F00EDE73A1F1368042B04D00023136014
:101C70003A00A4002D19324B1B78002B02D017001C
:101C8000FFF775FB2B6801991C120B4030499B0034
:101C90005B5817000435FFF74CFBA3009C46FE1A67
:101CA000002C17DC1C22264B1A700023336063467D
:101CB000FF1A234B04371B78002B01D0FFF757FB8B
:101CC0002B68019A1C121340214A9B009B58043533
:101CD000FFF72FFB002033685A108300F1580123CF
:101CE0000B4003D10D21164A1170DFE749108A42DB
:101CF00000DD0A0001308442EFDC0123520013436F
:101D0000D4E7A3009C46FE1A002C25DC1C220C4BB9
:101D10001A70002333606346FF1A094B04371B789F
:101D2000002B01D0FFF723FB2B68019A1C121340F4
:101D3000074A9B009B580435FFF7FBFA80EE3600FC
:101D4000A4020020C8050020A502002008000020F1
:101D500078CE0000FCFFFF3F002033685A1083005C
:101D6000F15801230B4003D10D21E04A1170D1E756
:101D700049108A4200DA0A0001308442EFDC012374
:101D800052001343C6E73B00083B1868FFF7CAF947
:101D90003B1F06001868FFF7C5F90023864200DAEA
:101DA0000433A4003A1B17001360D04B04371B7890
:101DB000002B01D0FFF7DBFA2B68019A1C121340AD
:101DC000CB4A9B009B580435FFF7B3FA3B00083B16
:101DD0001868FFF7A7F93B1F06001868FFF7A2F97C
:101DE000F30FC217B0425341A4003A1B17009B00E7
:101DF0001360BE4B04371B78002B01D0FFF7B7FAF6
:101E00002B68019A1C121340B94A9B009B58043559
:101E1000FFF78FFA3B00083B18683B1F1968A600C4
:101E2000BE1B0423814202D0042802D80023336061
:101E300018E001239C461842F8D10F2302681A408B
:101E4000042AF3D163461942F0D10429EED90B6874
:101E50000B321340042BE9D1FFF784F9431E98415C
:101E600080003060A14BA4001B783F1B0437002B7F
:101E700001D0FFF77CFA2B68019A1C1213409C4A90
:101E80009B009B580435FFF754FA3B00083B186849
:101E90003B1F1968A600BE1B0023814202D0042804
:101EA00002D80423336018E001239C461842F8D17D
:101EB0000F2302681A40042AF3D163461942F0D175
:101EC0000429EED90B680B321340042BE9D1FFF73C
:101ED00049F94342584180003060844BA4001B788C
:101EE0003F1B0437002B01D0FFF741FA2B68019A02
:101EF0001C1213407E4A9B009B580435FFF719FAC9
:101F00003B00083B1868FFF70DF93B1F06001868F7
:101F1000FFF708F9F317C20F86425341A4003A1B9A
:101F200017009B001360714B04371B78002B01D006
:101F3000FFF71DFA2B68019A1C1213406C4A9B0094
:101F40009B580435FFF7F5F93B00083B1868FFF78D
:101F5000E9F83B1F06001868FFF7E4F80023864203
:101F600000DD0433A4003A1B170013605F4B0437F5
:101F70001B78002B01D0FFF7FAF92B68019A1C128D
:101F800013405B4A9B009B580435FFF7D2F93B1F77
:101F90001B68A400043B5A1E93413A1B17009B0088
:101FA0001360524B04371B78002B01D0FFF7DFF989
:101FB0002B68019A1C1213404D4A9B009B58043514
:101FC000FFF7B7F93B00083B1868FFF7ABF83B1F7A
:101FD00006001868FFF7A6F832180120A4003B1B82
:101FE0001F00520002431A60404B04371B78002B3D
:101FF00001D0FFF7BCF92B68019A1C1213403C4A30
:102000009B009B580435FFF794F93B00083B186888
:10201000FFF788F83B1F06001868FFF783F8321AAD
:102020000120A4003B1B1F00520002431A602F4BEB
:1020300004371B78002B01D0FFF799F92B68019A20
:102040001C1213402A4A9B009B580435FFF771F974
:102050003B00083B1868FFF765F83B1F060018684F
:10206000FFF760F802000120A4003B1B1F00724331
:10207000520002431A601D4B04371B78002B01D01D
:10208000FFF775F92B68019A1C121340184A9B0040
:102090009B580435FFF74DF93B1F1868FFF742F8CE
:1020A000061E17D11F23114A1370A4003B1B1F00EB
:1020B0001E600E4B04371B78002B01D0FFF757F939
:1020C0002B68019A1C121340094A9B009B58043547
:1020D000FFF72FF93B00083B1868FFF723F83100A2
:1020E00007F090F9012640000643DEE7A402002035
:1020F00078CE00003B1F1868FFF714F8061E17D1B2
:102100001F23F14A1370A4003B1B1F001E60EE4BFF
:1021100004371B78002B01D0FFF729F92B68019AAF
:102120001C121340E94A9B009B580435FFF701F944
:102130003B00083B1868FEF7F5FF310007F048FA4E
:10214000012649000E43DEE73B1F1868FEF7EAFF51
:10215000C217801850400122A4003B1B1F00400002
:1021600010431860D84B04371B78002B01D0FFF7C1
:10217000FEF82B68019A1C121340D44A9B009B580E
:102180000435FFF7D6F8A300FE1A3068012C24D1DD
:10219000FEF7C8FF0494079009F058FD079900293D
:1021A00000DC012107F014FA049BA400C9180123E4
:1021B00049001943C44B3F1B1B7831600437002B87
:1021C00001D0FFF7D4F82B68019A1C121340BF4AC4
:1021D0009B009B580435FFF7ACF8FEF7A3FF049073
:1021E0007068FEF79FFF049B0130C31A0793D3E783
:1021F000A300FE1A31002000049301F019FD049B96
:102200003060FF1AB04B04371B78002B01D0FFF76A
:10221000AEF82B68019A1C121340AC4A9B009B58E5
:102220000435FFF786F83B00083B1868FEF77AFF95
:102230003B1F06001868FEF775FF02000120A4008E
:102240003B1B1F003240520002431A609E4B043772
:102250001B78002B01D0FFF78AF82B68019A1C121B
:1022600013409A4A9B009B580435FFF762F83B00E5
:10227000083B1868FEF756FF06003B1F1868FEF77C
:1022800051FF320002430120A4003B1B1F005200FB
:1022900002431A608C4B04371B78002B01D0FFF7E8
:1022A00066F82B68019A1C121340884A9B009B58C1
:1022B0000435FFF73EF83B00083B1868FEF732FF95
:1022C00006003B1F1868FEF72DFF32004240012038
:1022D000A4003B1B1F00520002431A607A4B0437D4
:1022E0001B78002B01D0FFF742F82B68019A1C12D3
:1022F0001340764A9B009B580435FFF71AF83B1FA2
:102300001868FEF70FFFC0430122A4003B1B1F000B
:102310004000104318606C4B04371B78002B01D031
:10232000FFF725F82B68019A1C121340674A9B009F
:102330009B580435FEF7FDFF3B00083B1868FEF78D
:10234000F1FE06003B1F1868FEF7ECFE32008240EB
:1023500051000122A4003B1B1F000A431A605A4B84
:1023600004371B78002B01D0FFF701F82B68019A86
:102370001C121340554A9B009B580435FEF7D9FFA9
:102380003B00083B1868FEF7CDFE06003B1F1868AF
:10239000FEF7C8FE3200024151000122A4003B1B9F
:1023A0001F000A431A60484B04371B78002B01D0EA
:1023B000FEF7DDFF2B68019A1C121340434A9B0075
:1023C0009B580435FEF7B5FF3B000C3B1868FEF741
:1023D000A9FE3B00083B06001868FEF7A3FEF117B4
:1023E0000200C317300007F045F93B1F0490059128
:1023F0001868FEF797FE02000498059907F0EEF8BA
:1024000043000120A4003E1B370018432E4B3060D0
:102410001B780437002B01D0FEF7A9FF2B68019A27
:102420001C121340294A9B009B580435FEF781FF7C
:10243000A300FE1A310020000493FEF7BDFC049BAC
:102440003060FF1A204B04371B78002B01D0FEF7B9
:102450008EFF2B68019A1C1213401C4A9B009B584C
:102460000435FEF766FFA300FF1A39002000FEF7CF
:10247000BBFC154B1B78002B01D0FEF778FF2B68B7
:10248000019A1C121340114A9B009B580435FEF719
:1024900050FFA300FE1A310020000493FEF7E4FC75
:1024A000049B3060FF1A084B04371B78002B01D0C7
:1024B000FEF75DFF2B68019A1C121340034A9B0034
:1024C0009B580435FEF735FFA402002078CE0000AB
:1024D000A300FF1A39002000FEF75AFDE44B1B78D9
:1024E000002B01D0FEF743FF2B68019A1C1213400A
:1024F000E04A9B009B580435FEF71BFFA300FE1A21
:10250000310020000493FEF7B5FD049B3060FF1AF4
:10251000D74B04371B78002B01D0FEF728FF2B6820
:10252000019A1C121340D34A9B009B580435FEF7B6
:1025300000FF3B1F186800F0D5FF3A00083A126808
:102540000300A400D10729D4042A0CD910680F2253
:102550001040013808280FD806F0C0FE05202622BA
:102560000E0E0E0E2400C449180009F00FFC434261
:1025700058413B1B80001860BD4B3F1B1B78043744
:10258000002B01D0FEF7F3FE2B68019A1C121340BA
:10259000B84A9B009B580435FEF7CBFEB749E3E7EA
:1025A000B749E1E7B749DFE7B749DDE7069B3E1DDD
:1025B000F31AAF4CD82B03DD1A232370FEF7D7FE96
:1025C00000F0E4FC43000120184323783860002B1E
:1025D00002D03700FEF7CBFE2B68019A1C12134085
:1025E000A44A9B009B5837000435FEF7A2FE069BC9
:1025F0003E1DF31A9E4CD82B03DD1A232370FEF7E1
:10260000B6FE00F0B9FCA14B40001840012318436E
:1026100023783860002B02D03700FEF7A8FE2B6825
:10262000019A1C121340934A9B009B5837000435B3
:10263000FEF77FFE069B3E1DF31A8D4CD82B03DD63
:102640001A232370FEF793FE00F0A0FC904B1A684B
:10265000831A904201D28F4A9B1801205B000343EA
:102660003B602378002B02D03700FEF780FE2B68FA
:10267000019A1C1213407F4A9B009B583700043577
:10268000FEF757FE00F082FC814BA4001860784BE7
:102690003F1B1B78002B01D0FEF769FE2B68019AC7
:1026A0001C121340734A9B009B580435FEF741FEF1
:1026B0000123A600BE1B20001A003100FEF780FD9A
:1026C000754C2068643002F005FF002802D1043DFB
:1026D000FEF760FE029B21685A78704803F01DFBEC
:1026E0000123029A3700137000F046FC6C4B2268FD
:1026F0001B68063253431818029B5860FEF74AFEC7
:10270000A600BE1B2000012300223100FEF758FD69
:10271000614C2068643002F0DDFE0028D7D05F48AD
:1027200003F078F8DCE7A4003E1BFEF7C9FD370094
:102730004F4B30601B780437002B01D0FEF717FE9B
:102740002B68019A1C1213404A4A9B009B5804357F
:10275000FEF7EFFD464BA4001B783F1B002B01D07A
:10276000FEF705FE2B68019A1C121340414A9B009C
:102770009B580435FEF7DDFDA4003E1B300000F041
:1027800038FC37003A4B30601B780437002B01D0FF
:10279000FEF7EDFD2B68019A1C121340354A9B0091
:1027A0009B580435FEF7C5FDA4003E1B300000F029
:1027B00022FC37002E4B30601B780437002B01D0F1
:1027C000FEF7D5FD2B68019A1C121340294A9B0085
:1027D0009B580435FEF7ADFDA300FE1A3100200022
:1027E000049300F00BFC049B3060FF1A204B04376D
:1027F0001B78002B01D0FEF7BAFD2B68019A1C1242
:1028000013401C4A9B009B580435FEF792FDA40020
:102810003F1B380000F028FC154B1B78002B01D023
:10282000FEF7A5FD2B68019A1C121340114A9B006C
:102830009B580435FEF77DFDA300FE1A31002000F1
:10284000049300F039FC049B3060FF1A084B0437F6
:102850001B78002B01D0FEF78AFD2B68019A1C1211
:102860001340044A9B009B580435FEF762FDC046A6
:10287000A402002078CE0000B4D00000BCD000003C
:10288000C3D00000CAD00000CFD00000FEFFFF7F01
:10289000D005002037894100C8050020A50200208E
:1028A00004000020A4003F1B380000F047FCFC4B54
:1028B0001B78002B01D0FEF75AFD2B68019A1C12E1
:1028C0001340F84A9B009B580435FEF732FD012166
:1028D000200000F01BFCF24B1B78002B01D0FEF710
:1028E00046FD2B68019A1C121340EE4A9B009B5830
:1028F0000435FEF71EFD0021200000F007FCE84B28
:102900001B78002B01D0FEF732FD2B68019A1C12B8
:102910001340E44A9B009B580435FEF70AFDA400CF
:102920003E1B300000F02CFC3700DD4B30601B7884
:102930000437002B01D0FEF71AFD2B68019A1C12F8
:102940001340D84A9B009B580435FEF7F2FCA400C4
:102950003E1B300000F028FC3700D14B30601B7864
:102960000437002B01D0FEF702FD2B68019A1C12E0
:102970001340CC4A9B009B580435FEF7DAFCA400B8
:102980003F1B380000F0EAFBC54B1B78002B01D041
:10299000FEF7EDFC2B68019A1C121340C14A9B0004
:1029A0009B580435FEF7C5FCA4003F1B380003F01C
:1029B000EBFCBB4B1B78002B01D0FEF7D8FC2B683F
:1029C000019A1C121340B74A9B009B580435FEF72E
:1029D000B0FCA4003E1B300003F086FD3700B04B76
:1029E00030601B780437002B01D0FEF7C0FC2B6849
:1029F000019A1C121340AB4A9B009B580435FEF70A
:102A000098FCA4003F1B380003F062FCA44B1B7829
:102A1000002B01D0FEF7ABFC2B68019A1C1213406F
:102A2000A04A9B009B580435FEF783FCA4003E1B84
:102A3000300003F063FC3700994B30601B7804379B
:102A4000002B01D0FEF793FC2B68019A1C12134057
:102A5000944A9B009B580435FEF76BFCA300FF1AB9
:102A60003900200001F028FC8D4B1B78002B01D091
:102A7000FEF77DFC2B68019A1C121340894A9B00CB
:102A80009B580435FEF755FCA300FF1A39002000BF
:102A900001F026FA824B1B78002B01D0FEF767FC71
:102AA0002B68019A1C1213407E4A9B009B580435E8
:102AB000FEF73FFCA300FF1A3900200001F034FBB1
:102AC000774B1B78002B01D0FEF751FC2B68019A45
:102AD0001C121340734A9B009B580435FEF729FCD7
:102AE000A300FF1A3900200001F046FB6C4B1B7855
:102AF000002B01D0FEF73BFC2B68019A1C121340FF
:102B0000684A9B009B580435FEF713FCA300FE1A8D
:102B100031002000049303F047FD049B3060FF1A4E
:102B20005F4B04371B78002B01D0FEF720FC2B688D
:102B3000019A1C1213405B4A9B009B580435FEF718
:102B4000F8FBA300FE1A31002000049303F034FDCB
:102B5000049B3060FF1A524B04371B78002B01D0C6
:102B6000FEF705FC2B68019A1C1213404D4A9B008E
:102B70009B580435FEF7DDFBA300FE1A3100200050
:102B8000049303F021FD049B3060FF1A444B04378B
:102B90001B78002B01D0FEF7EAFB2B68019A1C1270
:102BA0001340404A9B009B580435FEF7C2FBA3002C
:102BB000FE1A31002000049303F00EFD049B3060E8
:102BC000FF1A374B04371B78002B01D0FEF7CFFBE1
:102BD0002B68019A1C121340324A9B009B58043503
:102BE000FEF7A7FBA300FF1A3900200001F0B0F99F
:102BF0002B4B1B78002B01D0FEF7B9FB2B68019AF9
:102C00001C121340274A9B009B580435FEF791FB8A
:102C1000A300FF1A3900200001F0D6FA204B1B78E0
:102C2000002B01D0FEF7A3FB2B68019A1C12134066
:102C30001C4A9B009B580435FEF77BFBA300FE1A41
:102C400031002000049301F03BFA049B3060FF1A2E
:102C5000134B04371B78002B01D0FEF788FB2B6841
:102C6000019A1C1213400F4A9B009B580435FEF733
:102C700060FBA300FF1A3900200001F0E9F9084BBE
:102C80001B78002B01D0FEF772FB2B68019A1C12F7
:102C90001340044A9B009B580435FEF74AFBC0468C
:102CA000A402002078CE0000069B029AFB1A9B101B
:102CB0001361A300FF1A3900200002F0E9FD184B50
:102CC0001B78002B01D0FEF752FB2B68019A1C12D7
:102CD0001340144A9B009B580435FEF72AFB069BC1
:102CE000029AFB1A9B101361A300FE1A3100200008
:102CF000049302F0CDFD049B3060FF1A084B0437AB
:102D00001B78002B01D0FEF732FB2B68019A1C12B6
:102D10001340044A9B009B580435FEF70AFBC0464B
:102D2000A402002078CE00000023F7B55A1E0192BD
:102D3000002B07DA01F0D6FA02F0DAFE03F04CF8C5
:102D40001923019300263000194B1968B14212DD96
:102D5000184B1A6801328A420FDAF0241A601D6893
:102D6000154F6C43E35D002B1FD0E419022B06D1F5
:102D70002000FEF7BDFA019BD8E70022EDE7012B0A
:102D80000DD1002801D100F0F7F8F0226A43BB18FA
:102D90005B680A49C31A8B4201D80223BB54F02353
:102DA0005D43054BEB5C022BE2D00136CCE7C0461D
:102DB000CC05002000000020381C00203F420F00FE
:102DC000012200210A4B0B481A6119500430195096
:102DD000A2210420C9005850C121C02089008002CE
:102DE00058501A60044BFC311960044B1A7070473C
:102DF00000A000400405000000E100E0F50500200F
:102E000004207047F8B550C9012322001A40101E53
:102E10002DD03340181E2AD0641000201A2C26D83A
:102E20001D4B761035009E4200DD1D001B4F3B5DA3
:102E3000012B05D00121200004F028FE01233B5581
:102E4000174B1B78002B01D1FFF7BAFF0023154A5F
:102E50009E420DDCFF2514491448D65CB44202D1D1
:102E60005E007052D5540133042BF6D10420F8BD16
:102E7000D15C8C4203D10C4A5B009D52F6E70133D2
:102E8000042BF5D10023D15CFF2901D1D454F2E702
:102E90000133042BF7D1E9E788130000D80500209F
:102EA000F50500201C0000200E000020DC050000BD
:102EB00070B530C9012322001A40101E1BD02B40D0
:102EC000181E18D064101A2C00D91924174E335D1F
:102ED000012B05D00121200004F0D8FD012333553A
:102EE00069100800124A1038124B904204D901228E
:102EF00052421A60042070BD1C600F4806F082FA2E
:102F00000E4B18800E4B1B78002B02D1FFF758FF99
:102F1000F0E701220B4B9A64A922D2009A5880183C
:102F2000A82280B2D2009850E4E7C046D80500201D
:102F3000908601001800002020A107000C0000204E
:102F4000F505002000A00040030010B50120002B73
:102F500002DC1B30FEF7AEF910BD0420704710B53F
:102F6000002803DC1C20FEF7A5F910BD0B6800202B
:102F7000DB07FAD40D30F6E70122034B1A64A822CE
:102F8000D20098587047C0460080004010B5FFF747
:102F9000F3FFFA21890006F0ABF910BD0048704735
:102FA00034D100001B20704770B5054E0400335C1F
:102FB0000D008B4202D004F069FD355570BDC0464E
:102FC000D805002070B50024084D635D012B09D1A0
:102FD0000021200004F080FD0021200004F056FDB7
:102FE0000023635501341B2CEED170BDD8050020A1
:102FF000704711207047372070470000F8B5012452
:103000000B6806000D00234204D10D20FEF752F993
:103010002000F8BD5B1004D103F07EF9400020438E
:10302000F7E72000072BF4D80D4A9B009C580D4F62
:103030003B5D002B05D00021200004F027FD00237C
:103040003B55012E06DD6B68042B03D102212000C5
:1030500004F01CFD200004F0C7FB01244000DEE763
:1030600014D10000D8050020F8B5012605683542C6
:1030700002D04468344203D10D20FEF71BF9F8BD9D
:103080006D101A2DFBD80A4F7B5D012B04D0310047
:10309000280004F0FBFC7E55064964108C4202DCDB
:1030A000E143C9172140280004F024FCE7E7C046AB
:1030B000D8050020FF03000070B501240D682542EB
:1030C00004D10D20FEF7F6F8200070BD6D101A2D0A
:1030D00017D80024012804DD4C68043C63425C419D
:1030E0006400094E735DA34204D02100280004F05F
:1030F000CDFC7455280004F00DFD03000420012BC5
:10310000E3D00020E1E7C046D805002070B50400F8
:103110000D001A280ED8084E335C012B04D0012173
:1031200004F0B4FC01233355290020004D1EA941B1
:1031300004F0D2FC70BDC046D8050020036810B56D
:10314000DA0703D40D20FEF7B5F810BD416858101A
:1031500004394A425141FFF7D9FFF6E737B56946CE
:103160000A00064B30CB30C203680220042B02D188
:1031700000F0DAFF37BD00F0FFFFFBE7DCD0000016
:1031800010B5084C237D002B05D00021142004F03D
:103190007DFC00232375142004F0BCFC43425841FD
:1031A000800010BDD805002010B5084CA37D002B71
:1031B00005D00021162004F069FC0023A375162019
:1031C00004F0A8FC43425841800010BDD8050020FF
:1031D00070470000F7B5304D304E6B6C002B15D0AA
:1031E000A8240023E40037596B642D4B186800288D
:1031F0000CDB2C4B19784A425141C9B2197004F0CA
:103200006BFC294B1B88DF19BFB23751AB6C002B0D
:1032100039D00021254B264FF458A9643A780C3454
:103220000193244D8A4206D02B68032B03D8224AEF
:10323000D05C04F051FC2B68204A0133134004D5C4
:103240000422013B5242134301331B4900228C46A6
:103250002B60042B18D06046C05C591CFF2802D19B
:103260000B000122F5E7002A00D02B60012104F0B9
:1032700033FC01233B702B68114A5B009B5AE41816
:10328000019BA4B2F450F7BD01235B422B600023E5
:103290003B700C4BF3E7C046FCA0004000A0004090
:1032A00018000020F40500200C0000204405000058
:1032B000F3050020D40500201C000020030000803E
:1032C0000E00002050460000084B094AFF201A80DB
:1032D0005A809A80DA800023064A07491370074A09
:1032E000087048708870C870136070470E00002026
:1032F000DC050000F30500201C000020D4050020A0
:103300000122024B52421A607047C046180000204A
:1033100010B5034A0621034802F0A2F810BDC046CA
:10332000E4D0000056D80000E12170B549021948E8
:1033300003F0CEFF002401220320174B17491A6126
:103340005C50043158508018083158501A600630CB
:1033500004F044FAFF21124AA15401341B2CFBD182
:10336000012200200F4B01001A6004230E4A0F4D6A
:103370001468002CFCD02C680002013B2043116033
:10338000002BF5D101220A4B1A6004F05DF901F01F
:10339000F5F870BDC01B002000800040040500004F
:1033A000D805002000D0004000D1004008D50040E2
:1033B00004D00040F8B50B4E070030000D0003F0BC
:1033C000CFFF0400A84200DD2C003D00EB1B9C4217
:1033D00005DD300003F0CEFF28700135F6E7200050
:1033E000F8BDC046C01B002010B50100014803F025
:1033F00077FF10BDC01B002010B5054C200003F066
:103400007DFFE1212000490203F062FF10BDC046AC
:10341000C01B0020C3070CD4064B1B68834208D88E
:10342000054B1B68984204D8031F1B68002B00D073
:103430001800704700060020FC0500200023012230
:1034400010B50A48990001334250642BFAD1084C58
:10345000084B00211A602000074A08F017F9074BB3
:10346000074A6360074B1A6010BDC046902D0020CC
:103470000406002008000020D409000030270000C6
:1034800008060020F805002010B5044B044A1A6015
:10349000044B054A1A60FFF7D1FF10BD000600205B
:1034A00004060020FC050020D80F0020044B1B68F8
:1034B0001868000980B20238C343DB171840704710
:1034C000F805002000B59BB00200054901A808F0EE
:1034D00021FC01A802F0BAF902F07EFCFCE7C0462C
:1034E000B7D100000B4BC20704D4042804D80A4B00
:1034F00000D00A4B180070470F2203681A40031DC2
:10350000042AF7D0064B092AF4D0064B032AF1D03F
:10351000054BEFE791D100002ECD000028CD000033
:103520009BD10000ABD10000A2D100000020064AD0
:103530000649131F186013681B099BB202339B00D6
:10354000D2188A42F5D3704708060020D80F002011
:10355000F7B50F240126314B314A1968314B324DF2
:10356000186813681F002740072F26D813681B0907
:103570009BB202339B00D218AA42F2D300242B4EF6
:10358000A500AD192868FFF745FF01342860642CB9
:10359000F6D1274C2068FFF73DFF2060254C2068BE
:1035A000002802D0FFF736FF20600025224B1B6861
:1035B0000093009B9D4214DBF7BD1B099BB29B004F
:1035C000D3189A42D2D01F68374208D1B94206D2E6
:1035D000B84204D3043F3F68002F00D01F60043B73
:1035E000EFE7F0236B43154A9B181A78002A01D1A4
:1035F0000135DEE71F693C2300266B43DB199B0086
:1036000001930136BB1BF3D4019BB4001C1B0B4B75
:103610001C19A069FFF7FEFEA061F2E7000600207A
:1036200008060020FC050020D80F0020902D002067
:1036300008000020D80F0020CC050020381C0020F6
:10364000F7B50124204246D1234B1B689C46984283
:1036500041D3224B1B68019398423CD8031F1B683F
:10366000002B38D10200036800941B099BB2002B89
:103670000FD10099131F196090422CD015682B1F91
:103680001B68990069180C68013B14600A602A00E5
:10369000EDE79D0055192968009C214219D18C4500
:1036A00017D8019C8C4214D30E1F3468002C10D103
:1036B0000F680F343C40072C08D92F60151F2B6072
:1036C0000B680A601B099BB20A00D0E700993160C1
:1036D000CDE7013BCBE7F7BD00060020FC0500204D
:1036E0000D4970B50A000D4D1368141F1B0926689B
:1036F0009BB2981C002E0BD000238A4200D00B00F6
:1037000023608300C91880001218AA42ECD370BD50
:103710001B011360F7E7C04608060020D80F002001
:10372000F8B5124C27000F223B681D09ADB21342B9
:103730000DD06E1CB600A74204D032003900200024
:1037400007F091FF0022A3190436A4191A6002356C
:10375000AD00074B7F199F42E5D31B1B9B10013B1C
:103760001B012360034B1C60F8BDC0460806002007
:10377000D80F0020F8050020F0B59BB0FFF7FCFB48
:1037800000240700214AA300D0580134FFF758FF56
:10379000642CF7D11E4B1868FFF752FF1D4B1868B9
:1037A000002801D0FFF74CFF00261B4B1B689E42F0
:1037B00017DBFFF795FFFFF7CBFEFFF7B1FFFFF732
:1037C000DBFB164BC21B1B6815491B6801A81B09B4
:1037D0009BB2023B08F09EFA01A802F037F81BB03A
:1037E000F0BDF02575430F4BED182B78002B01D160
:1037F0000136DAE72B695C1E002CF9DBA300EB181D
:103800009869FFF71DFF013CF6E7C046902D0020A8
:1038100008000020D80F0020CC050020F80500206B
:1038200071D10000381C0020F7B5174D4F1C2B68D4
:1038300006001B680C001B099BB201929F420BDB28
:10384000FFF79AFF2B681B681B099BB29F4203DBA3
:103850000A20FDF72FFDFEBD2868A71CBA00DB1B60
:1038600081181B010B6029600021031F19600F23C1
:103870001E4003002401264340C3083A9A189A4286
:10388000E9D9019902C3FAE7F8050020F7B503006A
:103890000122134004000D000193002B2BD1174B84
:1038A0001B68834227D8164B1B68834223D90F23FA
:1038B000144F386000681840FFF7B6FF019B3C6862
:1038C000061E3B6017D0236804301B099BB29D4243
:1038D00000DD1D00AA00211D251F07F0BBFEFFF71C
:1038E00025FE2E60FFF734FE00232B602268064B76
:1038F0001340236034002000FEBDC04600060020B7
:10390000FC050020D80F0020F0FF0F000323043037
:1039100010B5C11719400918891000220420FFF7BB
:1039200083FF10BD70B5050008000C00FFF7EEFF27
:103930000023002804D170BDE95CC2181171013365
:10394000A342F9DBE343DB171C4000230419237176
:10395000F1E7F0B50C009BB0022804DC1C20FDF759
:10396000A9FC1BB0F0BD01230868184206D1042849
:1039700004D90F2601683140042901D00E20EEE75A
:1039800061680D001D40F9D10429F7D90A68324059
:10399000042AF3D1A2681A4201D10D20DFE7FFF714
:1039A000A1FD06006068FFF79DFDA768010001AC5E
:1039B0007F103000257003F022F8390064232200C4
:1039C00003F082F8200008F0EBF901002000FFF777
:1039D000A9FFC6E710B51C4CA544041E02D1FFF791
:1039E00095FF0BE002F024FF0138062828D805F0E7
:1039F00075FC090911182904240000208023DB002C
:103A00009D4410BD200002F08FFF011B2000FFF736
:103A100089FFF3E7200002F035FF4300012018433F
:103A2000ECE780226946D200200002F042FF68469F
:103A300008F0B6F901006846E9E704210348E6E723
:103A40000020CCE70420D9E700FCFFFF00D20000F3
:103A500070B50C00022803DC1C20FDF72BFC70BDA8
:103A600001230868184206D1042804D90F250168EB
:103A70002940042901D00E20EFE761681942FAD1EC
:103A80000429F8D90A682A40042AF4D1A2681A4203
:103A900001D10D20E1E7FFF725FD05006068FFF784
:103AA00021FDA46801006410280002F0A8FF210095
:103AB00002F0E5FFFFF78EFFD1E770B50D0001289A
:103AC00003DC1C20FDF7F6FB70BD012408682042D2
:103AD00006D1042804D90F2102680A40042A01D023
:103AE0000E20EFE76A682242FAD1042AF8D9136857
:103AF0000B40042BF4D1FFF7F5FC06006868FFF7D4
:103B0000F1FC0100300002F07AFF02F0FCFF4000FF
:103B10002043D9E7F8B507000C001C20012F0BDD6E
:103B200001250868284206D1042804D90F2102681B
:103B30000A40042A03D00E20FDF7BCFBF8BD6268E2
:103B40002A42F8D1042AF6D913680B40042BF2D18B
:103B5000FFF7C8FC06006068FFF7C4FC0100022FF5
:103B600014D0A4682C4211D06410300002F047FF3A
:103B7000050002F05DFE012811D1002C02DD0135A7
:103B8000012C06D12800FFF725FFD7E70124644266
:103B9000EBE7280002F0D4FE013C0500F0E7022824
:103BA000F0D1002CEEDD0135012CEBD000222800F5
:103BB000110002F0F7FE02F0C3FE013C0500F3E73E
:103BC00010B501240868044016D04410200005F008
:103BD000ADFE154905F078FD07F05EFC04F0B0F885
:103BE0000022124B06F012FE04F052F807F0E4FB3C
:103BF00043000120184310BD042810D90F23026888
:103C00001340042B07D1FFF76DFC21000A2208F0B6
:103C10008FF90400DAE7032B01D10430F5E70D201A
:103C2000FDF748FBD2E7C046D30237390000D04049
:103C3000086870B501240500254006D1042804D980
:103C40000F2302681340042B03D00E20FDF732FB34
:103C500070BDFFF747FC03782900233B5A425341CC
:103C60001022C01808F064F980239B05C218044B89
:103C70009A4201D91420E9E740002043E8E7C04612
:103C8000FFFFFF3F10B5034A0621034801F0E8FBA0
:103C900010BDC046D0D10000C8D100000020704740
:103CA00010B51E20FDF706FB10BD10B51E20FDF758
:103CB00001FB10BD10B51E20FDF7FCFA10BD10B5BC
:103CC0001E20FDF7F7FA10BD10B51E20FDF7F2FA21
:103CD00010BD10B51E20FDF7EDFA10BD10B51E2069
:103CE000FDF7E8FA10BD10B51E20FDF7E3FA10BD90
:103CF00010B51E20FDF7DEFA10BD10B51E20FDF731
:103D0000D9FA10BD10B5034A0B21034801F0A8FBF6
:103D100010BDC0463CD2000094D200000120034BED
:103D20001860034B1B68834018437047FC0F00204A
:103D3000DC0F0020F0B5EFF310810123194083F36D
:103D40001088134C134AA4461268134E013A93404C
:103D5000124F134A002B17D0146803420FD03D684E
:103D60002C60C046C046C046C046C046C046C0469D
:103D7000C0460C4C1568246825605B08EAE7654678
:103D80002C6014683460F8E781F31088F0BDC046F9
:103D900008050050200000200C050050E80F00200E
:103DA000F00F0020E40F002030B585B001AD0C22EB
:103DB0000649280007F04EFC0024285D012101344B
:103DC000FFF7F2F80C2CF8D105B030BD29D3000074
:103DD000F7B56A463B4B01AE1380062393703A4B0E
:103DE00033800F23B370FFF7C7F8384B384DC01836
:103DF0002B68984201D200232B602C68002C41D103
:103E0000375D01213800FFF7CFF801340021380079
:103E100003F062FE032CF3D1002401276B461E5DE4
:103E200039003000FFF7C0F801343900300003F0EA
:103E300053FE032CF2D1C8200138C046C046C0460C
:103E4000C046C046C046C046C046C046C046C04642
:103E5000C046F1D16B4600211878FFF7A5F86B46F4
:103E600000215878FFF7A0F86B4600219878FFF7FB
:103E70009BF8FFF781F8FA2300241B01C018286083
:103E80002000FEBDFFF778F82B6800249842F7D396
:103E9000042003F0A9FC0600052003F0A5FC361859
:103EA000062003F0A1FC0B4B9B1B181A0A4BA042E7
:103EB00006DB18600023094A2B6013600124DFE74A
:103EC0001C60F7E7040500000D0E0000102700003D
:103ED000F40F002043030000DC0F0020FC0F002043
:103EE0000022054B10B51A60044B1B68934201D0A9
:103EF00002F03EFC002010BDF80F0020E41A002064
:103F000010B5041E10DA1A240A4BA400E25801234B
:103F10009340094A09491360094A1160094A0A494C
:103F200011600A4A136010BDFFF73CF8A042EADDB9
:103F3000EAE7C04650E00000F00F002008050050FE
:103F4000E80F0020E40F00200C0500501805005079
:103F5000F0B53B4B85B01B680C00002B03D1012052
:103F60004042FFF7CDFF246801222700174028D0E8
:103F7000FF236012184033496714661040431F4006
:103F80001E4005F03FFA050438002E49784305F03D
:103F900039FA0002054330002A49704305F032FA2D
:103FA000294B28431B68202B06D16400A40E274B05
:103FB000A400E35800021843FFF7BCFE002005B040
:103FC000F0BD042CFAD90F2321680B40092BF5D141
:103FD000636803925B100193019B9F42EEDABB0082
:103FE000E3189E68039B1E4228D0FF2370121840DE
:103FF00072101A401349751440431D40009205F099
:1040000001FA030428000F496843029305F0FAF906
:10401000029D0002054300980A49404305F0F2F969
:10402000094B28431B68202B06D17600B60E074BA0
:10403000B600F55800022843FFF77CFE0137CBE7B6
:10404000F00F0020590600002000002010D50000CD
:104050000200086810B5C3070FD540101823012AC5
:1040600003DD4A68042A00D10833054A1360FEF7CD
:10407000BFFFFFF745FF002010BD01204042EDE7E4
:104080002000002010B50124044002D0441020007C
:1040900010BD042810D90F2302681340042B07D148
:1040A000FFF720FA21000A2207F042FF0400EEE7A2
:1040B000032B01D10430F5E70D20FDF7FBF8E6E70F
:1040C0000868F8B5C3071AD5FFF7DCFF0300203BEB
:1040D0005E2B25D80520434301221D180020114ED8
:1040E0009D4219D005211024F75C3C4200D0801875
:1040F0000139520064100029F7D10133F0E7042898
:104100000ED90F2203681A40042A09D11B099BB259
:10411000002B05D00379DAE7012340001843F8BDEE
:104120000120FCE735D3000070B508680D00FFF7EB
:10413000A9FF04006868FFF7A5FF621E0100042ABA
:1041400014D8451E042D11D805236B439B1801225A
:1041500015009D402B00064805682B430360054B66
:104160001B68002B02D0200002F003FB002070BD72
:10417000F80F0020E41A002070B508680D00FFF762
:1041800081FF04006868FFF77DFF621E0100042ABA
:1041900013D8451E042D10D805236B439B1801220C
:1041A0009A400748036893430360064B1B68002B43
:1041B00003D00022200002F0DCFA002070BDC046CF
:1041C000F80F0020E41A0020F0B5050089B0086857
:1041D0000C00FFF757FF0690022D36DD6068FFF7F1
:1041E00051FF0190A068FFF74DFF04000127231D38
:1041F000661E0793731C0293079B9E4235D00523CE
:1042000073430593019B019D05330493049BAB42CB
:104210001ED0042E16D86B1E042B13D80122059B2A
:104220002349013B5B199A409446224A0B68106867
:10423000069A3A4003920DD062461A430A60012260
:1042400000280DD17F000135E0E701240194CDE77E
:10425000029ECFE7624693430B600028F2D0039A98
:104260000299280002F085FAECE7019B1E1D042E3E
:104270001AD8012C18D1002505273B0021006B43DB
:104280009B1999400B000A4A013511689943094B63
:1042900011601B68002B05D0019B0022581D2900CE
:1042A00002F067FA052DE8D1002009B0F0BDC04644
:1042B000F80F0020E41A0020086810B5C30703D5E2
:1042C000FFF7E0FE054B1860054B1B68002B03D081
:1042D000024B186802F04EFA002010BDF80F0020C3
:1042E000E41A00207FB5A04C2368002B0AD19F4A16
:1042F0001268002A06D19E4B1B68002B01D0FFF7E5
:1043000067FD7FBD9B4D2A68002A26D1984A126816
:10431000002A1BD0FFF75CFD0028F2D0FFF744FD18
:10432000924B24681A681C60002A16D0002C14D105
:1043300001AD0C229049280007F08CF9285D00217E
:104340000134FEF731FE0C2CF8D1DAE7874A126807
:10435000002AE5D1002BE3D0E0E700210D2003F097
:10436000BBFB00210E2003F0B7FB00210F2003F060
:10437000B3FB2E68012E5DD0022E00D1A2E0002EEC
:1043800051D101363100794C04202368994303F060
:10439000A3FB04212368052019404B42594103F037
:1043A0009BFB10212368062019404B42594103F022
:1043B00093FB80212368090119404B4259410C208D
:1043C00003F08AFB80212368090219404B425941BE
:1043D0000B2003F081FB80212368490219404B42E6
:1043E00059410A2003F078FB802123688902194093
:1043F0004B425941092003F06FFB80212368C90219
:1044000019404B425941082003F066FB8023216884
:104410001B0319404B425941072003F05DFB31005B
:104420000D2003F059FB2B680321581C05F0D0F830
:10443000296066E702214D4C0720236819404B4252
:10444000594103F049FB0820216801404B42594182
:1044500003F042FB80212368C90019404B425941B7
:10446000052003F039FB80212368490119404B42A4
:104470005941062003F030FB80212368C90119400F
:104480004B425941042003F027FB80212368890314
:1044900019404B4259410A2003F01EFB802321683A
:1044A0001B0419404B425941092003F015FB310010
:1044B0000C2003F011FB31000B2003F00DFB310049
:1044C0000E20AEE72021294C0720236819404B42DB
:1044D000594103F001FB40212368082019404B4259
:1044E000594103F0F9FA80212368092019404B4211
:1044F000594103F0F1FA80212368490019404B42E9
:1045000059410A2003F0E8FA802123688900194004
:104510004B4259410B2003F0DFFA802123688901C7
:1045200019404B4259410C2003F0D6FA80212368F0
:10453000490319404B425941062003F0CDFA80212E
:104540002368C90319404B425941042003F0C4FABF
:10455000802321685B0419404B425941052003F038
:10456000BBFA01210F205CE7F80F0020EC0F0020C0
:10457000FC0F0020E00F002029D30000012010B51F
:104580004042FFF7BDFC0020FFF7D4FB10BD000048
:1045900010B5034A0921034800F062FF10BDC04670
:1045A00010D6000058D600008023F0B502255B0528
:1045B0001A690A4C0A4BA1261D5103278025F600D3
:1045C000ED00BA43884202D300221A51F0BD5F5970
:1045D000002FFCD098518018F4E7C0460405000075
:1045E00000E0014010B5002806D1C020B0214002F3
:1045F0008902FFF7D9FF10BDB02080218002C902D7
:10460000F7E7000043425841064B40421840B023B0
:104610009B02C018036800201A0E532A01D11B0206
:10462000180A704700C0FEFF30B501248025054BF5
:10463000054AED009C505C59002CFCD00160002123
:10464000995030BD00E0014004050000434258414C
:10465000074B40421840B0239B02C018A62310B558
:104660000902DB05090A1943FFF7DEFF10BDC0464A
:1046700000C0FEFFF0B5012480260D4B0D4DF60065
:104680005C51002902DC00225A51F0BD57781478A1
:104690003F022743947824042743D4780432240625
:1046A0003C439F59002FFCD010C00139E9E7C046B8
:1046B00000E001400405000070B505004B680A00E9
:1046C0009C1C2100A400FFF7D5FF281970BD000035
:1046D000134B1B68002B0CD08022B023D2029B020C
:1046E00000280BD11A1D5B681B0E522B00D1100045
:1046F0007047B022C02392025B02F1E782420DD9DB
:1047000003681B0E522B09D1436802339B00C0186B
:10471000824203D903681B0E522BE9D00020E7E741
:1047200000110020F0B50020B7B00024FFF7D0FF43
:10473000270005002600002D2ED1284D2868FFF700
:1047400061FF32003B0001900094254904A807F066
:10475000E1FA04A801F07AF8224B64201C682B6867
:10476000A0215A425341204A5B421340B022920298
:104770009B18E41A6043490204F044FEA02252024E
:10478000030000921949220004A807F0C3FA04A804
:1047900001F05CF837B0F0BDFF226B6829689C46D9
:1047A0000233FF180B12013613409C4200DA1C0042
:1047B000FF200A14024003926246014001920091D8
:1047C000039A0B4904A807F0A5FA04A801F03EF8E3
:1047D0002800FFF77DFF0500ADE7C046001100206F
:1047E00062D700000411002000C0FEFF0CD70000BB
:1047F0004ED7000070B50020FFF704FF0400012031
:10480000FFF700FF844200DA04000A4B1D686A4289
:10481000554128001D60FFF7E5FEA0226B425202C1
:104820001340054A28009B18044A611C1360FFF7D7
:104830000DFF70BD00110020048001000411002054
:10484000F8B50020FFF7DEFE07000120FFF7DAFED3
:104850003E00204D0643204C0DD18021C020C902CE
:104860004002FFF7A1FE01213000FFF7EFFE1B4BD6
:104870002E6023601DE0874209DD0023B0212B60FC
:10488000164B8902236023680020012517E00123CD
:1048900080212B60124BC9022360F4E7120E522ACA
:1048A00008D0002800D023600E4800F0CFFFFFF7AB
:1048B000A1FFF8BD28005A68023292009B188B4273
:1048C00005D21A68561CE9D10028F2D0D1E7216040
:1048D000EFE7C04600110020041100200480010011
:1048E00004C0020027D7000070B50020FFF7F0FEDB
:1048F000FF260500002801D1280070BD03681C14A4
:104900003440FFF7E5FEDA2CF4D10500F2E70000B1
:104910008022F0B55200A1B00021674806F0B6FE33
:10492000802200215200654806F0B0FE644BFF274C
:104930001B681A00049353425A4110000592FFF776
:1049400051FE049C0020631E9C415E4B64421C404F
:104950005D4BE418FFF7C8FF0600002E2DD1049828
:10496000FFF750FE411C0598FFF770FE059A574D62
:10497000534B2C601A60FEF73FFD514B64201B68BF
:10498000A0215A4253414F4A5B421340B0222C6847
:1049900092029B18E41A6043490204F033FDA022FE
:1049A0005202030000924A49220007A807F0B2F918
:1049B00007A800F04BFF21B0F0BD326813141212AB
:1049C0003A403B4003921A000A3A092A49D83A4B26
:1049D000039A995C002931D110223E4806F056FE18
:1049E00035002B6803991A123A40914209D11A14E2
:1049F0003A400B2A27D0132A2DD00A2A01D1354B51
:104A00001D602800FFF764FE051EEAD1314B1968CE
:104A100000290FD02000FFF74FFE04002D4B5B193B
:104A20005968002903D02000FFF746FE0400043532
:104A30000C2DF3D1204B0121039A99543000FFF73C
:104A400047FE060089E73B40022BDADC214A9B0047
:104A5000D3185D60D5E7102200211E4806F016FE2F
:104A6000CFE71A00153A082AE8D8144A0399525C8D
:104A7000002AE3D13500152B00D015003000036863
:104A80001A143A40152A0FD01D2A00D10025FFF72D
:104A90001FFE0028F3D1002D04D020002900FFF7CD
:104AA0000BFE0400054BC6E7039A1B123B409A42DB
:104AB000EDD10500EBE7C0460010002008110020F2
:104AC0000011002000C0FEFF04C0020004110020FD
:104AD000F1D60000202F002010B5FFF719FF10BD00
:104AE000F0B585B0039203220333DC17294D14403F
:104AF000E4182B68284F5A42534180225B42D2026D
:104B0000A4103B409B18A21C0291244E91000091DE
:104B10000190316800980A18934215D2FFF7F8FE09
:104B20002B685A42534180225B421F40D202BF1879
:104B30003368009A9B189F4206D2194800F086FEFF
:104B40000025280005B0F0BD029B356819066B46AC
:104B50001A7BA423DB051343FF222F00090C194302
:104B6000019B12041B04134019432800FFF75CFD4E
:104B70000837281D21003760FFF756FD002C04D0B0
:104B80000A9A21003800FFF775FD009B083BFF18CB
:104B90003760D6E70011002000C0FEFF041100209E
:104BA000CBD6000070B59AB0FFF74AFEFF221E4C2C
:104BB000D2000021200006F069FDFF25FFF794FEDA
:104BC0000026002814D10200C300E3580130591E0A
:104BD0008B41D218FF28F7D1144901A807F09AF8A1
:104BE00001A800F033FE124800F030FE1AB070BD8C
:104BF00003681A142A400A2A0AD11A122A40FF2AE4
:104C000003D0D200A1180B71A050FFF761FDD8E7C7
:104C1000132AFAD11B122B40FF2BF6D0DB00E2182F
:104C20001671E650F1E7C0469825002097D700009E
:104C3000ABD700000021094B094A5960013151608E
:104C400059680029FCD000211961012393600222D8
:104C5000044B8131FF315A501A607047FC100040FC
:104C60000010004000E100E00222064B0121DA675B
:104C70000022054B5A61054A11615A69002AFCD08D
:104C80007047C04604E100E0FC1000400010004006
:104C900010B5044C2378002B01D0FFF7E5FF00206E
:104CA000207010BD09120020802301205B055B6E7F
:104CB0005B001843704700000120024B1B685B003B
:104CC000184370478C1200200120024B1B685B00C8
:104CD00018437047240000200120024B1B685B0032
:104CE000184370479012002070B504000D001600A4
:104CF000FEF74CF9802301215B055A6E26700026D1
:104D000053006170E1706272010A5A0A6071A17108
:104D1000A272010C5A0C000E5B0EA6702571E17197
:104D20002072E272237370BD10B5044C200007F0AE
:104D300037F801002000FEF7F5FD10BD95120020A8
:104D40000E4B10B51B680E4C5A1C0FD00D4C002B8F
:104D50000CD00D4C012B09D00C4C022B06D0094C69
:104D6000042B03D00A4C052B00D1074C200007F080
:104D700017F801002000FEF7D5FD10BD2800002027
:104D80003CD80000BCD0000047D80000C3D00000D1
:104D900041D8000070B5214C2278002A3DD1204B2B
:104DA00001215A608022D20511605A68002AFCD085
:104DB000002207201B4B1C4901255A50043958502A
:104DC00008315A5019481A4958501A491A485A5025
:104DD0001A495A50A622D2009D50082218495A500A
:104DE0000431585002201749585017491748585055
:104DF000174804395850182016495850C1218900C5
:104E00005A500539FF395858921802435A501249DE
:104E1000124A9950FFF70EFF257070BD091200204D
:104E2000FC000040001000400C0500007469627531
:104E30001C05000024050000200004022C050000D1
:104E400014050000340500003C050000FFFF0000D1
:104E500021100100540500000A1200200405000082
:104E600070B50E4B06001B78002B01D1FFF792FFA7
:104E700000200B4D2C7884420ED00A4B202219784A
:104E80000323091B1940084B4901C918300006F0DB
:104E9000E1FB0120013C2C7070BDC04609120020CE
:104EA00094120020081200200A120020002370B57E
:104EB00088B0984235DD0D6801262C0034409C42B4
:104EC0002FD12300042D2CD90F222B681A40230048
:104ED000092A26D16A683F2A23DD6846FFF7C0FF0A
:104EE000230000281DD06B4619783300A14203DB54
:104EF0006B461B5D5B003343A200AA18013493602C
:104F0000202CF2D1092169444A780B7812021A4305
:104F10008B781B041A43CB781B061343024A136099
:104F20000423180008B070BD9012002070B5454BE6
:104F30008AB01B78002B01D1FFF72CFF02AC2000B8
:104F4000FFF78EFF002802D100200AB070BD237841
:104F50000B2BF9D96378012BF6D1E378012BF3D130
:104F600000231120384E394D33602B70684423796B
:104F7000374A41781360027809021143827812049B
:104F80001143C27812060A4332490A60002B0ED13F
:104F9000152169444A780B7812021A438B781B0456
:104FA0001A43CB781B0613433360002318E0012B10
:104FB0001AD1152169444A780B7812021A438B786A
:104FC0001B041A43CB781A211B06134333600E23AC
:104FD000627C6944934200DD130000229A422CD186
:104FE00000220420EA54B0E7022B03D1627B103385
:104FF0001621EEE7042B0DD11521082269446846DD
:1050000006F028FB0098019902F0B2FD06F0D4F9F1
:105010003060CAE7052BC8D11521082269446846CB
:1050200006F018FB0098019902F0A2FD06F0C4F901
:105030003060627D0A231E21CBE7885CA8540132D0
:10504000CCE7C046091200208C12002095120020E7
:10505000280000209012002010B5134B04001B788C
:10506000002B01D1FFF796FEFFF7FEFD00200F4A4F
:105070000F49104B54505860013010605868002898
:10508000FCD0002018610130906018690028FCD025
:10509000094B0A481B785B011B185350FFF7E4FDCE
:1050A000FFF7C8FD10BDC0460912002000100040E7
:1050B00004050000FC100040081200200A12002025
:1050C00010B588B000281DDD0A68012113000B40CF
:1050D00018D1042A16D90F2014682040092811D1AC
:1050E00050683F280EDD98001018806800240842A0
:1050F00001D04010C4B26846C4540133202BF2D111
:10510000FFF7AAFF002008B010BD000010B500286E
:1051100013DD0C68E30710D56410532C0DD8084B31
:105120001B78002B01D1FFF735FEFFF79DFDA12372
:10513000044ADB00D450FFF77DFD002010BDC046BF
:10514000091200200010004010B500280EDD0C6888
:10515000E3070BD56410FF2C08D8054B1B78002BF8
:1051600001D1FFF717FE034A034BD450002010BDB6
:1051700009120020001000402405000013B500288B
:1051800014DD0C68E30711D5094B64100093094B3B
:105190000193072C0AD8084B1B78002B01D1FFF78D
:1051A000F9FD6B46054A1957054BD150002016BD35
:1051B000E2ECF0F4F8FC00040912002000100040BA
:1051C0000C05000070B588B0002820DD01240868B7
:1051D00004401CD104281AD90F2302681340042B61
:1051E00015D1FEF77FF9060006F0DAFD050012285A
:1051F00000D912252A0002210D326846FFF774FDFE
:105200006B465D73A54205DC6846FFF725FF00206D
:1052100008B070BD2300325D6B449A730134F1E72E
:10522000F0B50D008BB0012832DD086801220400C2
:1052300014402DD104282BD90F2301680B40042BD7
:1052400026D16B68134223D0FEF74CF96E68070035
:105250007310019306F0A4FD05000E2800D90E2559
:105260002A000121113202A8FFF73EFD6A46127999
:1052700002AB5A7302AA73129373019B76141B0E2E
:10528000D67313745574A54205DC02A8FFF7E4FE3B
:1052900000200BB0F0BD3A5D02A963189A74013486
:1052A000F1E730B589B0002814DD0C68E30711D5AB
:1052B000102268460021FFF717FD6B466A4665100D
:1052C0005D73684663122D0E64149373D473157462
:1052D000FFF7C2FE002009B030BD0000174B184A8E
:1052E0005968002903D00021596001319160196982
:1052F00000291FD0002018618023DB00D3581149FA
:10530000012B18D1A923DB00D3585B420B600E4957
:105310000B78032B01D801330B7003200B490B785A
:10532000013303400B700A495B015B180949535074
:105330000123936070470860FAE7C046FC10004004
:1053400000100040240000209412002008120020C9
:105350000A1200200405000010B5034A102103487A
:1053600000F07EF810BDC046BCD70000B3D70000E7
:10537000044A05491368C85401339B059B0D13600B
:105380007047C046C4160020C412002070B5114CEE
:10539000114A2368834202DC0023236016E0155C77
:1053A000411C2E00FA3E012E05D899420FDA555CB9
:1053B000013D1F2D01D90800ECE70100151A565CCC
:1053C0006E5401318B42FADC181A206070BD1570E2
:1053D000FAE7C046D01A0020D016002010B5FDF71D
:1053E000CBFD064B1A68824201D900221A601B6865
:1053F000C31A034898428041404210BDC0120020A9
:10540000204E000010B5094C094A236812689342E7
:1054100000D110BD074AD05CFDF7E6FF0028F8D0A8
:10542000236801339B059B0D2360ECE7C816002021
:10543000C4160020C412002010B50400064B074A11
:105440001B6812689B1ADB439B059B0DA34200DB84
:1054500010BDFFF7D7FFF1E7C4160020C8160020E3
:1054600070B5074E33680B2B08DC0C255D43054CEB
:105470000133285164196160A260336070BDC04679
:10548000CC160020302F002010B5FBF717FEFFF7D9
:105490007FF8FBF73BFEFDF73BFFFEF7F3FBFEF764
:1054A00031FCFFF759FF00F063FF01F065F901F0EF
:1054B000AFFB10BD962210B512010021034806F083
:1054C000E5F80022024B1A6010BDC046381C0020CF
:1054D000CC050020064B074A1B6812689B1ADB4369
:1054E0009B059B0D0122834200DC002210007047C7
:1054F000C4160020C8160020F8B505000C001600E0
:105500001F1E0ED10320FFF7E5FF002808D0FA2068
:10551000FFF72EFFE8B2FFF72BFFE0B2FFF728FFFF
:10552000F8BD501DFFF7D6FF0028F9D0FB20FFF78C
:105530001FFFE8B2FFF71CFFE0B2FFF719FFF0B260
:10554000FFF716FF3012C0B2FFF712FF3C00E31B5B
:105550009E42E5DD2078FFF70BFF0134F7E70000FE
:1055600070B50024F0250B4B1B68A34202DCFFF74B
:10557000A1FF70BD2B006343074A9B181A78002ACD
:1055800005D05978002311201A00FFF7B5FF013428
:10559000E9E7C046CC050020381C0020F8B507001C
:1055A0000024F0252B0063430C4A01349E18B742B7
:1055B00011D0317800290BD00133D15C00231120A8
:1055C0001A00FFF799FF2A000021300006F05EF86C
:1055D0000A2CE7D1F8BD024B1C60F9E7381C00200B
:1055E000CC050020F0B5150001222F00754C1740A6
:1055F000A54401900291002F11D005AB1A706A10DA
:105600005A70120E1A710522691299706D1402995E
:10561000DD70FFF771FFCF239B009D44F0BD042D8B
:105620001ED90F202A681040042826D1022304AA7C
:1056300028001371FDF756FF040006F0B1FB624B22
:10564000984200D91800B84204DC421C05AB02990C
:105650000198DEE701377B1EE35C05AAD355F2E72C
:10566000042D00D0A9E0032304AA043D13716B426A
:105670005D4105AB55710222E9E709287ED104227C
:1056800005AB1A706A685110009169465212097888
:105690009A70009A59701F2A01DD202200926A46F2
:1056A000127806ACDA70009BBB4202DC05ABE21A52
:1056B000CDE70126BB00EB189868064006D1042808
:1056C00037D90F210368194002290CD10123237017
:1056D0004310637042121B0E4014A270E0702371DD
:1056E00005340137DFE7042921D102232370FDF7B8
:1056F000F9FE039006F054FBA31C0C2809D8607037
:10570000864201D19C19ECE7039A925D9A550136C5
:10571000F6E70C226270039A925D9A550136092EC3
:10572000F9D12E23E372237363730E34D9E7012971
:1057300007D1032304382370434258416070023478
:10574000CFE7092909D10423237043685A106270F6
:105750005B12A370E6700434C3E703290BD1052361
:1057600023700068020992B2430F92000B40D31AD3
:1057700063701B12EDE726700134B2E7032800D0F6
:1057800049E7052105AB1970110989B2520F89004B
:1057900002408A1A111299705A701100642A00DDB1
:1057A00064210420D970C9B2041FA14201DC043273
:1057B0004DE72C5C1C540130F6E7002D00D02AE7A1
:1057C00051E7C046C4FCFFFF2303000070B5020090
:1057D0000024F0210D4E0800604380194578954261
:1057E00003D001340A2CF6D170BDF022002105F05F
:1057F0004DFF074A1368013BA34200D11460002308
:1058000029001A001120FFF777FEEDE7381C002071
:10581000CC05002010B5B2B002236A460400137014
:1058200006F0BEFAC72800D9C7200023984207DC3B
:10583000421C6B46FE211420FFF75EFE32B010BD05
:10584000694601335A1EA25CCA54EFE730B5B3B0C3
:1058500002236A460500137006F0A2FA0400C72866
:1058600000D9C72400239C420BDC20003230FFF714
:10587000E3FD621C6B46FF211420FFF73DFE33B0B1
:1058800030BD694601335A1EAA5CCA54EBE70000DA
:10589000F0B5BBB004900C00012803DC1B20FBF723
:1058A00009FD51E02A4B08680293C30709D4042874
:1058B00007D90F2302681340042B02D1FDF712FE13
:1058C0000290234B60680393C30709D4042807D9C7
:1058D0000F2302681340042B02D1FDF703FE03904F
:1058E00000271C4B1B680693069BBB420BDC039BEB
:1058F000194A0093C821029B08A806F0D9F908A804
:10590000FFF7A4FFCAE70C267E43144B0299F61852
:10591000306806F03BFA051E05D17368B668079338
:10592000079B9D4201DB0137DEE73068039905964E
:1059300006F02CFA0836002808D121000498059BAF
:10594000083102385B6898473BB0F0BD0135E7E7A6
:10595000C7D10000CC16002018D90000302F00203D
:10596000F7B5234B06001B68F02100930023009A33
:105970009A4211DC0024F0231A006243019201993B
:105980001C4A55182F78002F12D001340A2CF3D15D
:105990001948FFF75BFF29E00A005A4315488218AF
:1059A0005078B04202D11278002A1FD10133DEE7CD
:1059B000F0223900280005F069FE02230D4A019902
:1059C000EB6053540D4AF1008A58009B6E70AE7024
:1059D000AA602F616F61A34202DC054B01341C6099
:1059E000002331001A001020FFF786FDF7BDC046E6
:1059F000CC050020381C002061DD00009825002027
:105A000010B5FFF7ADFDFF24084AE3005B429B1889
:105A1000074AD35C043B012B03D8E043C0B2FFF735
:105A20009FFF013C002CEFD110BDC046FC070000D9
:105A300098250020F7B50F00FF247F2501901E4A0E
:105A4000E300D31A1D4A9A181278062A01D0032AB5
:105A500020D1FF22D2009B18186883682B401C2B92
:105A600018D1C3681A002A40042A13D102692A40B7
:105A7000192A0FD11B0A01339B000C30C018FDF707
:105A800031FD03780600002B10D006F089F90023C1
:105A9000B84209D0013C002CD1D1F7BD019AF15C8C
:105AA000D25C9142F6D101339F42F7DCE043C0B2B1
:105AB000FFF756FFEEE7C04698250020FC070000E0
:105AC00070B50500FF24084AE3005B429B18074AB3
:105AD000D35CAB4203D1E043C0B2FFF741FF013CCE
:105AE000002CF0D170BDC046FC07000098250020B6
:105AF000F7B5FDF741FA574B1A68824201D90022E7
:105B00001A601A685449821A8A420DD9FF225349F1
:105B10001860D3005248CB1A1B181B78073B022B86
:105B20000CD9013A002AF4D1F7BD0720FFF7C8FFCE
:105B30004C4B27E00820FFF7C3FF38E0FDF726FABB
:105B4000071E00D101270020FDF71AFB019000205D
:105B5000FDF72AFB019B0090434C444D002B12D0D3
:105B60002368002B6ED12B682760002B6ED0404B32
:105B700001261B78002BD8D10920FFF7A1FF394B54
:105B80001E703B4B1E70009B002B12D02B68002B0D
:105B90000FD123682F60002B1ED0324B01261B78BB
:105BA000002BC7D10920FFF78BFF2E4B1E70304B07
:105BB0001E702368002B0FD02A4E3278002A0BD19A
:105BC0009F4200D227602368FB1A312B04D907209B
:105BD000FFF776FF012333702B68002B0FD0244E84
:105BE0003278002A0BD1BB4200D92F602B68FF1AF4
:105BF000312F04D90820FFF763FF01233370236896
:105C0000002B0CD0019B002B09D1164E3378002BB2
:105C100002D10720FFF754FF0023236033702B6865
:105C2000002B00D180E7009B002B00D07CE7104CBC
:105C30002378002B02D10820FFF742FF00232B60BE
:105C4000237071E7009A002AA0D1B5E7009B002BD2
:105C50009FD1AEE7BC1200200F270000982500203E
:105C6000FC070000B0120020AC120020B41200208B
:105C7000B812002037B500240500FFF771FC01A819
:105C80000194FDF76BFA21002000FEF729F9FEF7D9
:105C900029FBFDF79DFAFDF717FBFDF731FBFEF73A
:105CA0006DFCFDF78FF9A54204D0FDF7C7FB024854
:105CB000FFF7CCFD37BDC04652DD0000002310B514
:105CC00001001A001120FFF717FC10BD07B56B4645
:105CD000197069465A7013128B701314120ECB7020
:105CE0000A716B46010005221320FFF705FC07BD72
:105CF00010B50A0001001220FFF774FC10BD70B54A
:105D0000050008000C003230FFF796FB2B00220044
:105D100000211B20FFF7F0FB70BD10B50C00030045
:105D2000110014202200FFF7E7FB10BD012370B51E
:105D3000FF24084A41185B42884201D3D84370BD12
:105D400006781D0A234073409B009B5801306B402E
:105D5000F2E7C04634D9000013B50400FE2813D87A
:105D60000A4BC200D05800280ED043680830990072
:105D7000FFF7DCFF01900920FFF75EFB01AB042277
:105D800021001720FFF7B8FB13BDC046982500205F
:105D9000F7B50190FEF7A8FD01250400FF276D422D
:105DA000002C01D12800FEBD266833143B40152B82
:105DB0000DD121000198083105F0E8FF002801D13C
:105DC00035123D402000FEF783FC0400E8E71D2B60
:105DD000F8D101256D42F5E7F0B580279FB0FFF7B8
:105DE00011FBB24CB24D2068FF00391A4019FDF783
:105DF000E1FA23680600C3182360002B0ED11FB000
:105E0000F0BD2068391A2818FDF7D4FA2368060077
:105E10001B182360FDF7B0F8A64B1860002EF0DCCD
:105E20002B78FA2B00D002E12368022B07DCFFF766
:105E3000D5FA0028E3D00120FFF7A8FADFE7687859
:105E4000AC78023818281FD803F048FA0D2024280F
:105E50002B341E3E707A7E94CDDE1E1E1E1E1E1E2C
:105E60001E1E1E1EEC00FF2C0ED02000FFF7AEFC05
:105E70000022914BE100CA505B181A712100009278
:105E800013001320FEF72CFE0320D5E72000FFF7B8
:105E900067FDF9E72000FFF799FCF5E7FFF7B0FD94
:105EA000F2E7FFF75DFB0020FFF7E4FE8348FFF712
:105EB000CDFCE9E7632CE7D8814BA200D258210042
:105EC0001520FFF78FFBDFE7FEF70EFDFF2704002D
:105ED000002CD9D025682B143B40152B04D0200072
:105EE000FEF7F6FB0400F3E72000083005F058FF4A
:105EF00006000530FFF7A0FAFB20FFF739FA2D1254
:105F00001D20FFF735FAE8B2FFF732FAF0B2FFF7DB
:105F10002FFA3012C0B2FFF72BFA25002B1B9E423E
:105F2000DDDD287AFFF724FA0135F7E700211D208F
:105F300000910B000A00FEF7D3FDFDF77FFAA3E7FF
:105F40002000FFF709FF9FE7FDF728F805AC5D4A41
:105F5000642100905C4B200005F0AAFE0223200083
:105F6000237005F01DFF2300020000211620FFF71B
:105F7000C3FA89E70026504AF3009B181C68002CDE
:105F800028D01B790393636808349F00B81D0293DF
:105F9000FFF752FAFB20FFF7EBF901207D1CFFF71A
:105FA000E7F9F0B2FFF7E4F9E8B22D12FFF7E0F9F4
:105FB000E8B2FFF7DDF90398FFF7DAF9E719A7422E
:105FC0000CD8FFF71FFA05230298584301F05AFB3B
:105FD000FFF718FA0136FF2ECDD155E72078FFF7ED
:105FE000C7F90134EBE70024FFF7BAFA22002100D9
:105FF00000942300DA20FEF773FDFF222100D20077
:106000002D4805F043FB98E7012C02D1FEF78AFBEF
:106010003AE7022C02D1FEF75FFD35E70120FFF7DA
:1060200029FE31E7002321001A001A209FE7FB2BED
:1060300000D000E72268042A00DCF8E62E79E87830
:10604000224B360206439E4200DDF4E6331D9A429F
:1060500000DCECE6EB5CFE2B00D0ECE66B78AC7879
:10606000771E1B2B76D019D8072B5CD0082B31D08C
:10607000012B19D1FF2C17D02000FFF7A7FB6D795A
:10608000134AB31E009221002A000A20FEF728FDC1
:10609000094BE400E0501B191D7105E01D2B6BD06E
:1060A0005DD31E2B00D17EE0701DC5E6D01A002006
:1060B000D0160020C01200209825002034DD0000FA
:1060C000902D00204BDD000046DD0000F6030000AF
:1060D000D6160020632CE7D86A79022A13D0032A47
:1060E0001BD0012AE0D1E979AB79090219432B7A57
:1060F000A4001B0419436B7A1B060B435B0013437C
:10610000324AA350D0E7002FCEDDB11E3048FDF754
:1061100009FC2E4BA400E050C6E7AB79A4005A1E40
:1061200093419B00ECE7632FBEDC05AD3A002949A3
:10613000280005F08FFA00232800EB55FFF728FE12
:106140000028B1DB214B8000C25821001520FFF749
:1061500049FAA9E739001F48FFF76CFCA4E7FF2CB8
:10616000A2D06A79022A9FD819490B2000912100F8
:10617000B31EFEF7B5FC97E7632F00DD632700230E
:1061800005A9BB420ADBFB430022DB173B40CB18CF
:106190001A70152000917B1C2100EAE7EA18527959
:1061A000CA540133EDE7012C00D07DE7002F00DC5D
:1061B0007AE76B79002B03D01C00322B00DD3224F0
:1061C00064235C43044B1C606EE7C046902D0020A6
:1061D000D6160020D51600200400002001207047AC
:1061E00010B5064C200000F043FE0549200000F0E9
:1061F00081FE0122034B1A6010BDC046081B00201F
:10620000801A0600D41A002010B501210D20FCF7D9
:10621000CBFE01210E20FCF7C7FE00210F20FCF76A
:10622000C3FE044C200000F065FD1021200000F0AA
:106230007DFD10BDE81A0020F8B501250C682C4240
:1062400003D10D20FBF736F8F8BD64102DD4FCF710
:10625000A9FEA04229DB00212000FCF7A5FEFA22BE
:106260002900D200200001F03FFA00281DD00025AF
:1062700000270726FA2201219200200001F034FABB
:10628000002812D0282802DD0123B3401F43013E1D
:10629000F0D20E4EAF550135052DE9D10122062170
:1062A0000920FDF7C1FA002801D10020CCE70B231B
:1062B000012443600023F25C9900520041182243FC
:1062C00001338A60052BF6D1BEE7C046D81A0020FC
:1062D00010B504680D20E30703D56410FF2C03D923
:1062E0001720FAF7E7FF10BDFFF78EFFE1B2024873
:1062F00000F03EFD0020F6E7E81A002010B5FFF799
:1063000083FF0021034800F033FD430001201843C0
:1063100010BDC046E81A0020A02101220B4BC90085
:106320005A500B480B4958500B491A604A68002ACA
:10633000FCD000224A60A121C900585801215960AF
:10634000A021C9005A50054BC0187047007000408A
:106350006A10000004050000FC700040FBFDFFFF18
:1063600010B5FFF7D9FF43000120184310BD00000E
:1063700010B5034A0A210348FFF772F810BDC04662
:1063800078DD0000C8DD0000F8B5012306681E4274
:1063900005D045681D4202D084681C4203D10D20FF
:1063A000FAF788FFF8BD76101520802EF8D86D100A
:1063B0001620FF2DF4D86410FF2C01D91720EFE729
:1063C0000B4B1B68002B01D1FFF70AFF094FF1B2FD
:1063D000380000F026FEE9B2380000F015FDE1B209
:1063E000380000F011FD380000F086FE0020D9E7EB
:1063F000D41A0020081B0020F7B501221400904297
:1064000022DD0D682A421FD01D4B15411B684C68C8
:10641000002B01D1FFF7E4FEE9B201272500194E58
:106420003D40300000F0FDFD002D0FD03C4130001C
:10643000E1B200F0E9FC300000F05EFE0024A04272
:1064400002D02320FAF736FF2000FEBD042CF2D93B
:106450000F2322681340092BEDD163685B10019371
:10646000019BAB42E7DDAB00E3189968394204D0E9
:106470004910C9B2300000F0C7FC0135F0E7C04652
:10648000D41A0020081B0020154B70B51B680500AE
:106490000E00002B01D1FFF7A3FE124CEDB2290034
:1064A000200000F0BEFDF1B2200000F0ADFC0021A4
:1064B000200000F0C1FD002801D0404270BD72B63E
:1064C00001222900200000F0A7FD62B6200000F0A4
:1064D0008CFC0028F2D0200000F08CFCEEE7C046D7
:1064E000D41A0020081B002010B5012403682342A1
:1064F00002D04168214203D10D20FAF7DBFE10BD26
:106500005810802801D91520F7E74910FF2901D933
:106510001620F2E7FFF7B8FF40002043EFE710B581
:106520000400012814D105211820FFF7ADFF7F28B2
:106530002BDC03007F3301DA7F204042C8235B421B
:1065400058437F2102F05EFF052C00D1404210BD70
:10655000032811D101001820FFF796FF7F2814DCD3
:1065600003007F3301DA7F204042C8235B42584357
:106570007F2102F047FFEAE70020052CF5D1072133
:106580001830FFF781FF7F2802DD0138FF38D0E7A0
:1065900003007F3301DA7F204042C8235B42584327
:1065A0007F2102F02FFFD1E710B50120FFF7B7FFE1
:1065B00043000120184310BD10B50320FFF7AFFFC3
:1065C00043000120184310BD10B50520FFF7A7FFB9
:1065D00043000120184310BD10B508211820FFF713
:1065E00053FF0300C00FC0180123401015304000B6
:1065F000184310BDF8B501231C0098422BDD0F682D
:106600003B4228D04E6835001D4024D1042E22D9AB
:106610000F2231680A40092A1DD173685C10202CB2
:1066200000DD2024144B1B68002B01D1FFF7D8FD9F
:1066300072B67F10F9B2114F2200380000F0ECFC66
:1066400062B6A54214DA380000F0CFFB002804D16E
:1066500001246D002C432000F8BD380000F0CAFB77
:106660000122AB004000F31810439860AD18E8E732
:1066700064000125EEE7C046D41A0020081B002064
:1066800070B52B4B86B01B68002B02D10120FFF7A1
:1066900046FF01AD14220021280004F0F7FF254E2B
:1066A0001821300000F0BDFC0321300000F0ACFBED
:1066B0000021300000F0C0FC041E13D172B6052288
:1066C0001821300000F0A8FC62B6300000F08DFB0D
:1066D000002802D0300000F08DFBA3000134E85008
:1066E000052CF2D1019B7F2B01DD013BFF3BAA680A
:1066F0007F2A01DD013AFF3A29697F2901DD01394D
:10670000FF39C820434342434843DB11D21152436F
:10671000C0115B4340439B18181804F083FE01F03E
:1067200057FB04F049FE43000120184306B070BD3A
:10673000E01A0020081B002000207047012070474D
:1067400000207047002070470120704700207047EC
:1067500000207047002070470020704700207047DD
:1067600000207047002070470020704700207047CD
:10677000704770477047000010B5034A0E21034868
:10678000FEF76EFE10BDC0462CDE00009CDE000051
:106790000378013B1F2B00D970470130F8E710B593
:1067A000FFF7F6FF0378002B0BD00130222B11D11D
:1067B0000378002B03D0421C222B03D11000FFF7DB
:1067C000E7FF10BD5C2B03D14378002B00D0821C67
:1067D0001000EDE73A2BF2D02C2BF0D07B2B0BD115
:1067E000FFF7D6FF0378002BE9D07D2B01D10130D4
:1067F000E5E7FFF7D4FFF5E720225B2B14D1FFF785
:10680000C7FF0378002BDAD05D2BF0D0FFF7C7FF6E
:10681000F7E7202BD3DD2C2BD3D0190091435D2932
:10682000CFD0222BCDD001300378002BF1D1C6E799
:10683000002210B5904216D0FFF7AAFF0378042279
:10684000222B10D0023A7B2B0DD0013A5B2B0AD0C1
:10685000190030390232092905D92D2B05D141788B
:10686000303909290AD8100010BD0522742BFAD03E
:106870000132662BF7D001326E2BF4D0581E8341C3
:106880005A42F0E770B5FFF783FF037801222D2B02
:1068900001D18018023A00230A2502E06B4301303F
:1068A000CB1801783039CCB2092CF7D95A431000F3
:1068B00070BDF8B50C001500FFF76AFF0378222BB6
:1068C00002D000232370F8BD0D236A1E2100082585
:1068D0000C260A279C4601300378222B02D1002384
:1068E0000B70F0E7002BFAD0441C5C2B0BD14378E3
:1068F000841C622B0ED0662B0ED06E2B0ED0722B0A
:106900000ED0742B0ED0002AE9DD0B70013A013154
:106910002000E1E72B00F6E73300F4E73B00F2E765
:106920006346F0E70923EEE710B50400FFF737FFF1
:10693000A04202D90378202B00D910BD0138F7E717
:1069400010B5002815D00378002B13D0FFF720FFD7
:106950002021037802008B4300205D2B09D010001A
:10696000FFF71DFF03782C3B5A425341C018FFF735
:106970000FFF10BD1800FCE70300002070B50C00ED
:1069800081420EDD1A785B2A0BD1581CFFF700FFFD
:106990000125AC4205D0FFF7D3FF002801D0013517
:1069A000F7E770BD70B50C001500002901D0002379
:1069B0000B70002820D00378002B1ED0FFF7E8FED4
:1069C000037806002C2B03D10130FFF7E1FE06000F
:1069D000337800207D2B0FD0844204D02A00210080
:1069E0003000FFF766FF3000FFF7D9FE03783A2B3F
:1069F00002D10130FFF7CCFE70BD1800FCE7F0B506
:106A00000D0004009DB02E78002E35D02E212800D8
:106A100005F0AEF9071E14D0431B0193303E092E3A
:106A200014D82800FFF72EFF01002000FFF7A4FF75
:106A30000400002C20D0002F1ED0019B0133ED1844
:106A4000E1E7280005F0ACF90190E7E723787B2B1C
:106A500011D1601C642203A9FFF7A4FF041E0BD010
:106A6000019A290003A805F0A2F90028E1D020002E
:106A7000FFF795FEEEE7002420001DB0F0BD70B5D5
:106A8000050000200C0081421DDD2800FFF7D0FE2C
:106A90000300681C012B14D00020022B13D100220C
:106AA000681C1100FFF77EFF012C0CD0FFF748FF98
:106AB00000221100FFF776FF013CF5E7FFF740FFEA
:106AC000013C012CFAD170BDF8B5050000200C0086
:106AD00016001F0081420DDD2800FFF7A9FE03000C
:106AE0000020022B06D1681C3A003100FFF75AFF44
:106AF000012C00D1F8BDFFF723FF3A003100FFF76A
:106B000051FF013CF4E710B50024A04218D0FFF774
:106B10003FFE03787B2B0AD1013000221100FFF7E2
:106B200041FF00280CD0FFF73AFE0134F5E75B2B5C
:106B300006D10130FFF704FF002801D00134F9E746
:106B4000200010BDF8B5002816DD0D68EB0713D541
:106B50006D10013D0124FDF7C7FE0026FF276442AA
:106B600000280CD1002E21D0300005F019F90100C9
:106B70003000FCF7D7FEF8BD01256D42EAE7036857
:106B80001A143A40152A0BD11B123B409C4200DAE2
:106B90001C009D4201D106000836FDF799FDDFE794
:106BA0001D2AFAD1012400266442F6E701200134AF
:106BB00064002043DFE7000010B508680C00FCF714
:106BC00091FCFFF7E5F8002803DB6268024B8000C8
:106BD000C250002010BDC046902D002010B508689E
:106BE000FCF780FCFFF7D4F80123002802DB024BFE
:106BF0008000C358180010BD902D002010B5086803
:106C0000FCF770FCFFF7C4F8C043C00F800010BD54
:106C100010B5034A04210348FEF722FC10BDC0460C
:106C20002CDF000025DF000010B5FCF77DFBFCF732
:106C30002BFCFEF729FC0448FEF708FEFDF7B2FF27
:106C4000FEF7DEFE10BDC0467BDF000010B5FCF78E
:106C50006BF810BD70B5002504AC24780573A9420B
:106C600005D10A4B0A4A23210A4804F085FC016039
:106C70000949920052589B0002715B58A40083712D
:106C80006358856043710223C37170BD93DF0000B8
:106C9000F2DF0000A1DF000050E00000037B002BCA
:106CA00004D143738373036101330373704700009E
:106CB0001FB50191A02100240068C900D2B2445040
:106CC000012A10D0A24209D0032A0AD0074A8350D1
:106CD000074B019AC250012343501FBD02221343A8
:106CE000F4E70422FBE70622F9E7C046540500005A
:106CF0002405000010B50400FFF7D0FFA12223688F
:106D0000A179D20099506179064A200099502179E1
:106D100004329950044B19685A689B68FFF7C8FF02
:106D200010BDC0460C050000FC1A00204BB2002B21
:106D30000FDB80233F290FD81F290FD80F290FD829
:106D400007290FD803290FD81B060168074A8B5063
:106D5000704780239B04F8E7DB04F6E71B05F4E7A4
:106D60005B05F2E79B05F0E7DB05EEE72405000095
:106D70000368074A99501A00FC32D1680029FCD0F8
:106D8000A321C90058580023C0B2D3607047C04641
:106D90001C05000007B58022074BD2051A600022AF
:106DA0009A6002321A7111230E320093034905339F
:106DB0000348FFF74FFF07BDFC1A002000300040DA
:106DC000E81A0020F8B505000E0017000024BC42A8
:106DD00008D02B68315D1B6828009847002801D037
:106DE0000134F4E72000F8BD704710B51C3000F006
:106DF000BDF910BD10B51C3000F0AAF910BD10B5DA
:106E00001C3000F0B9F910BD70B5437E0D00002BA9
:106E100001D1002070BD6430040000F0B6F90028F4
:106E2000F7D12000290000F084F90120F2E70000EA
:106E3000F7B50193FA23002504009B0083600B4BF8
:106E40004560083303601C300F00160000F066F93F
:106E50002000643000F062F96B461B79276166758B
:106E60006576A5762000A375FEBDC04630E0000023
:106E70000123827DC3751B4B9200F0B5D4582022AC
:106E8000210011404D1EA941457DC026AD005D5930
:106E9000A0272A40531E9A4153421F2214402A40E1
:106EA0002500B6004942C135FF0531403340FF356A
:106EB0000D4EC919AD006E501100C131FF31DB1903
:106EC0008900CE50CC210569084B4904E9500521C1
:106ED0000569243BE95001690833CC500169044B32
:106EE000CA50F0BD50E000000C0600002405000070
:106EF0000C050000A022002310B50469D200A350A5
:106F00000A4CA1420FD90A4C8C425B4109495B42B1
:106F10000B40CD21C9045B18046907496350052162
:106F20000369995010BDCC235B04F5E7A0860100EE
:106F300090D00300000098FD24050000F7B5040080
:106F400000200D000193824265D01600402A00D92E
:106F5000402627001C37380000F0F6F8B1232269DC
:106F6000DB00D55080220123216992008B50A27E44
:106F7000002A03D122691362226913600025731E5F
:106F8000AB4207D1019B002B04D080220221236950
:106F900092009950012223691A622369FC33DA684E
:106FA000002A02D19A6A002AF9D09A6A002A0BD1E3
:106FB000DA60A3232269DB00D1583800C9B2013559
:106FC00000F0B7F8B542DAD3019B2269002B0FD14C
:106FD0001300FC339B6A002B0AD10133A376D361E3
:106FE0002369FC33DA6C002AFCD00022DA640AE060
:106FF00000230121A37651611A002369FC339968AB
:107000000029FCD09A602369FC339A6A002A01D0D7
:1070100000229A62E8B2FEBD10B50123FFF78EFF91
:1070200010BD0300AC3310B504001970643000F0DB
:107030008BF80123637610BD0023020070B5AC32DB
:1070400043760D001178B12204000069D20081500E
:107050008022216992008B502269013313622269D8
:10706000936026006436300000F080F8002812D0CB
:10707000300000F06DF81E4B2269D0502369FC33BC
:107080001A6A002A02D19A6A002AF9D09A6A002A5A
:1070900001D11A62E5E723690122002D0DD1190003
:1070A000FC31896A002908D1DA612369FC33DA6C82
:1070B000002AFCD00022DA6407E05A612369FC331D
:1070C0009A68002AFCD000229A6000202369FC33D1
:1070D0009A6A82420BD098622169064A8B588B507B
:1070E0001800022B03D0181F431E9841033070BDB7
:1070F0001C050000C404000010B50121FFF79CFF2F
:1071000010BD000010B51323122202490248FFF7F8
:107110008FFE10BD00400040081B002010B540222B
:107120000021040004F0B2FA002320002364636409
:1071300010BD10B53F24026C531C2340446C9C428C
:1071400001D08154036410BD00230364436470477D
:10715000436C026C934206D03F21C25C01330B406A
:1071600043641000704701204042FBE7036C406C11
:10717000181A00D540307047436C026C934201D01E
:10718000C05C704701204042FBE73F22036C406C2B
:1071900001331340181A43425841C0B270470000EF
:1071A00003210A4802680A430260094802680A4348
:1071B00002600849084A094B9B1A03DD043BC85882
:1071C000D050FBDC00F012F8F8F79EFF24050040D9
:1071D000540500409CE500000000002064020020EF
:1071E000FEE7FEE7FEE7FEE7FEE7FEE72D4B10B504
:1071F0001A68D2B2012A0FD12B4A126812070BD19A
:107200002A4AE0241168F0220800104021422DD1C2
:107210002749096811422CD01A68D2B2012A12D12A
:107220002149096809070ED1F02020490968014069
:10723000402908D11E490968014204D18020C1219A
:10724000C005C90042501B68DBB2012B0DD1164BA3
:107250001B681B0709D1154B1A68F0231A40A02A96
:107260000FD1134A12681A420ED010BD3028CFD069
:10727000D2E7104A104911608021104A09021160BA
:10728000CAE7D02AF1D1ECE70D4B1A68012A04D0E5
:107290000C4A1A601A68012AFCD1C0220A4B1A60F3
:1072A000E3E7C046E00F00F0E40F00F0E80F00F065
:1072B000EC0F00F004050040DFFF07C0186C004031
:1072C00000EC06407593000014EC06400120704766
:1072D00010B503681322DB69984710BD70470000A2
:1072E000054B0269D1500369FC331A6A002AFCD0AD
:1072F000002201201A6270471C050000030010B52F
:107300005C331A781F231A401E3B19009140114A22
:10731000D167C222042104699200A150026953601E
:107320000269D360A02300220169DB00CA50012357
:107330000169094A5B428B500169084A8B50016917
:107340000C3A8B50016908328B501430FFF7FCFE69
:1073500010BDC04604E100E00C050000140500006B
:1073600010B51430FFF702FF10BD10B51430FFF751
:1073700003FF10BD10B51430FFF7EAFE10BD00008A
:10738000030070B55E331A780469724BE250030053
:107390005D331A780469704BE250030061331C7846
:1073A00002696E4B012C00D09EE005005F352E78FF
:1073B000A225ED005651020060321578A12206691F
:1073C000D200B5500269D4509623DB00994200D810
:1073D0008CE096231B01994200D88AE096235B013A
:1073E000994200D888E096239B01994200D885E015
:1073F000E1239B01994200D882E09623DB01994268
:1074000000D880E0E123DB01994200D87DE096239B
:107410001B02994200D87AE0E1231B02994200D86E
:1074200077E096235B02994200D874E0E1235B0287
:10743000994200D871E0E1239B02994200D86EE0A6
:10744000474B994200D86CE0E123DB02994200D817
:107450006AE0E122002312038A425B41414A5B4217
:107460001340802252059B1801693F4A8B50A0238C
:1074700004220169DB00CA5000210369FC33D96092
:107480000369FC331962012301690B6001698B6098
:10749000C1210469890062501F215C3002780A40D2
:1074A00093406231314AFF31535000214156002947
:1074B0003CDA0F230B40083B2D4C9B089B001B190B
:1074C00003242140A140FC348C40DD69A5432C00FD
:1074D000C0258D4029002143D9611F23017819401F
:1074E0001E3B8B40136070BD00246CE79E23DB02C3
:1074F000BAE79D231B03B7E71E4BB5E71E4BB3E767
:10750000EC239B03B0E71D4BAEE71D4BACE71D4BD7
:10751000AAE71D4BA8E71D4BA6E71D4BA4E71D4B93
:10752000A2E78023DB049FE71B4B9DE78C080F4BF2
:10753000A400E41803230B40FF21C025DB00994081
:10754000AD0066598E433100C0269E4033000B4388
:107550006351C2E70C050000140500006C05000033
:1075600090D0030000D0BEFE2405000000E100E042
:1075700000ED00E000B013000050270000A04E0016
:1075800000F0750000509D0000F0EB0000903A0103
:1075900000E0D70100B0AF0300705F07F7B50093BC
:1075A00008AB1B7800250193FA2304009B0083603D
:1075B0000E4B45600833036014300F001600FFF7D0
:1075C000ADFD23005C3327611E70009B084A9B00C1
:1075D000995823005D331970019B20009B009A5835
:1075E00023005E33DD701A70FEBDC046CCE00000A3
:1075F00050E00000036910B51A00FC32D2680400A4
:10760000002A0AD0A322D20099581430C9B2FFF739
:1076100090FD00222369FC33DA6010BD10B50248EA
:10762000FFF7E8FF10BDC046C01B00201D2307B5B3
:1076300002220093024901330248FFF7AFFF07BD62
:1076400000200040C01B002010B5002801D004F02D
:10765000D9FA10BD0849094A094B10B51B6888586A
:10766000FA22190A1B0618439200002302F002F8BE
:107670004904C00B084310BD001001400405000080
:10768000241C002070B5041E09D0FFF7E3FF05009D
:1076900000F014F8FFF7DEFF401BA042F8D370BDE6
:1076A0000022044B9A60044A13680133DBB2136072
:1076B0007047C046FC100140241C002070477047F2
:1076C00010B500F061F8FFF7FAFF0120FFF7DAFFCD
:1076D000FFF7AAFAFFF7BAFA024B002BFAD000E044
:1076E00000BFF7E700000000F8B516004C1EA141EE
:1076F0001F220125104B8000104FC3584C421340ED
:1077000038680F499D4001F0F3FD0A21704301F0F4
:10771000EFFD2C400300220029000A4800F016F873
:10772000FA21094C89004443386801F0E1FD010069
:10773000200001F0DDFDF8BD50E000002C0000202D
:1077400040420F00100500501027000030B50468BB
:107750000C40944206D1013B002BF8D112E0013BD2
:10776000002B0FD004680C409442F8D10024056827
:107770000D40954204D101349C42F8D1002002E032
:10778000201C00E0181C30BDC420114B80001A588A
:1077900010491140C02212020A431A50C02180220F
:1077A000490092025A501A608023A3220021DB056F
:1077B000D20099500122F9309A60074BFF301950DE
:1077C000C120023180001950403019501A607047B2
:1077D00000E100E0FF00FFFF00100140014B1860D6
:1077E0007047C04678000020F7B500231E285AD8FD
:1077F000384B8000C258042A5BD007D8022A54D0E4
:1078000055D80423012A09D000234CE0062A54D07D
:1078100051D31A2A53D002231B2AF5D12E4A1168BC
:1078200008294ED909294FD00A240226A020012573
:107830002A4AC00015502A482A4D07681C20BF005C
:1078400007402948019700685759009027481B02B4
:1078500007401F43C02300989B020340FF2057515D
:107860005759000207401F43019B1F43009B5801CB
:107870006023184007433E43565101251C4B1560B9
:1078800058680028FCD000205860A1230125DB00A7
:10789000D3585560A025ED0050511BB2A14202D033
:1078A00015D2611ACB401800FEBD0823B6E710239D
:1078B000B4E72023B2E74023B0E78023AEE70123FB
:1078C000ACE708240026B1E70C000126AEE7091B4F
:1078D0008B40E8E750E0000074000020007000409A
:1078E000300000200405000034000020FF00FFFFEE
:1078F000FC700040F0B51E285BD8364B8000C258A3
:10790000354B1E68002E30D1C227344BBF00D859EA
:10791000334C03250440C02000022043D851C0242A
:1079200080206400800018512E4F18602E4B803C40
:10793000D859FF3CA043D8510437D859A843204315
:10794000D8510837D8590C35A843844607206546D6
:107950002843D851A820C0001E50C1208026800096
:1079600076021E501C601C4B1C60142500202B004E
:107970001E4C2E0046433659771C1BD14343E25020
:10798000A0230325C132FF329200DB05D550184BEE
:107990001A68082A14D114234343E3189A6812483A
:1079A0005132FF32920059601150DA68C1239B00B6
:1079B000C250F0BD9642E1D001300328D9D1F8E79A
:1079C000082A02D9083AD140E5E708239A1A9140DB
:1079D000E1E7C04650E00000281C002000E100E084
:1079E000FF00FFFF04050000009000403800002069
:1079F000780000202149F0B54A6C2148002A14D0B3
:107A0000A025A12600230124ED05F600C258571C2D
:107A100006D0C7187F68002F02D027009740AF51CB
:107A200014333C2BF2D100234B64A0230121DB054E
:107A300000260F009C4614234B43C3181A1F1268DC
:107A4000104C0E4D920014195219526C002A10D08D
:107A50001A00143A1268551C09D0103B1B68FF2B02
:107A600005D03B00934065461A00074BEA50FC34B2
:107A7000666401310429DED1F0BDC046FC900040AF
:107A800038000020009000400C05000000B51E28C2
:107A900018D8104A80008358C0209A068000D21758
:107AA0000240A020C00512181F200340032909D856
:107AB0000800C133FF339B0001F010FC02090507E9
:107AC0000021995000BD0C21FBE70421F9E70321B7
:107AD000F7E7C04650E000001E2812D80B4B80008C
:107AE000C258C02093068000DB170340A020C005C9
:107AF0001B181F20104001228240002902D1044996
:107B00005A507047A121C900FAE7C04650E0000072
:107B10000C050000030000201E2B12D8C021094ACA
:107B20009B009A5889009306DB170B40A021C905DA
:107B30005B18A221C90058581F231A40D0401E3B91
:107B40001840704750E00000F7B506000D000C002B
:107B50008B180193019B671B9C4207D033682178E7
:107B60001B683000984701340028F3D13800FEBD6F
:107B7000F0B5C64600B5CB0F9846404A4B005B0DAA
:107B80009A1882B00D000400132A2FDC002A49DB6A
:107B90003B4F17413E000E40064323D07F0839007B
:107BA00029400C430AD03749BD438C4663445C42AC
:107BB0005C418023DB021341E4071D434146CE00B4
:107BC00031492B008E192200346875682000290085
:107BD00001F0F6FE009001910098019922002B001F
:107BE00003F086F802B004BC9046F0BD332A08DDED
:107BF0008023DB009A42F5D102000B0001F0E0FE89
:107C0000F0E7224A9446012263445242DA4002429B
:107C1000E8D052080242D1D094438022D2051A41C2
:107C20001443CBE74B005B080343DBD00B031B0B78
:107C30001C436342234380244D0C24031B0B23402D
:107C40006D042B4319004346DA000F4B9B181C6848
:107C50005D6802000B002000290001F0B1FE0090D9
:107C600001910098019922002B0003F041F842464F
:107C70004B005B08D60733431900B3E701FCFFFF55
:107C8000FFFF0F00EEFBFFFF00E10000EDFBFFFF39
:107C9000F8B5274A4B005B0D9A180C000700132A11
:107CA00010DC002A36DB234B13410B423AD08024F0
:107CB00024031441002064189C4306002500300072
:107CC0002900F8BD332A0EDD80230600DB000D00FD
:107CD0009A42F4D102000B003800210001F070FE3E
:107CE00006000D00EBE7144D0600AC460125634489
:107CF0006D42DD40AC4663460D000342DFD03323C6
:107D00009A1A323B93401818874200D94C1C63469C
:107D10009843D2E7C90FCC070020531CCDD1074BA5
:107D20001C43CAE706000D000028C0D1C7E7C046C3
:107D300001FCFFFFFFFF0F00EDFBFFFF0000F03F26
:107D400030B5214A4B0087B05B0893421EDD1F4AC5
:107D5000934205DD02000B0002F0CAFF07B030BD00
:107D600002AA00F095F803231840049A059B012805
:107D700013D002281DD0002814D00298039900F0D7
:107D80006FFB80231B069C466144E7E7002300222B
:107D90000093002301F0DEF8E0E70298039900F079
:107DA0005FFBDBE7012402980399009401F0D2F80D
:107DB000D4E7012402980399009401F0CBF88023C2
:107DC0001B069C466144C9E7FB21E93FFFFFEF7FAB
:107DD000F0B54746CE4680B58DB004000D0000F0EA
:107DE00067FA294B06001B780F005BB298460133F7
:107DF00010D022002B002000290003F0C1FA814698
:107E0000002807D1002200232000290001F00AFCED
:107E1000002806D1300039000DB00CBC90469946C0
:107E2000F0BD01230293194B0694079503934B462B
:107E30000A93434604940595002B15D00023002295
:107E40001900100002F0D8F8434608900991022B5F
:107E50000ED103F0AFFB212303600A9B0193002B9B
:107E60000CD1089E099FD5E70023002408930994AC
:107E700002A801F0C1F90028EFD1EAE703F09AFB6C
:107E80000A9B01930360ECE77C00002010E10000F6
:107E9000F0B54E464546DE465746E0B5E14B4C0050
:107EA0008FB09046894664089C4200DC87E0DE4B38
:107EB0009C4222DCDD4A002900DC92E0DC4B02F02F
:107EC00017FFDB4B06000F009C4200D17EE1D94A30
:107ED000D94B02F00DFF02000B00414630000A6052
:107EE0004B60390002F004FFD34BD24A02F000FF8E
:107EF000434601259860D9606BE0D04B9C4200DC82
:107F00008FE0CF4B9C4200DD55E1CE4A23159246CF
:107F10009A4451460905631A19001D00040003F034
:107F20004BFA03F07FFA02000B00200029000892B0
:107F3000099302F0DDFE0022C34B02F067FC0F0044
:107F4000060003F039FA03F06DFA04000D00020098
:107F50000B00300039000A940B9502F0C9FE002294
:107F6000B94B02F053FC002200230C900D9101F05C
:107F700053FB002800D192E10023002220002900B9
:107F800001F04AFB434243410133B04A414601926A
:107F9000022208A80092524600F07CFB4B460500E6
:107FA000002B16DA802243461206944642465B684E
:107FB000454263445360D3686344D36009E00B00D7
:107FC000020041460A604B600022002300258A60BF
:107FD000CB6028000FB03CBC90469946A246AB4609
:107FE000F0BD934B01F0ECFC914B06000F009C425E
:107FF00000D13DE18F4A904B01F0E2FC02000B0002
:10800000414630000A604B60390002F071FE894A37
:10801000894B01F0D5FC012543466D429860D9603B
:10802000D7E701F049F88A4A8A4B06000F0002F0B0
:10803000EDFB0022884B01F0C3FC03F0BDF9050005
:1080400003F0F0F9794A7A4B0490059102F0DEFBD7
:1080500002000B003000390002F04AFE754A0600AB
:108060000F0004980599744B02F0D0FB0290039125
:108070001F2D00DCC7E0029A039B3000390002F09C
:1080800037FE83468A4653465B0024155B0DE31A90
:10809000102B6CDD04980599D322674B520502F032
:1080A000B5FB02000B00300039000292039302F08E
:1080B0001FFE0A000100130006910792020039001A
:1080C000300002F015FE029A039B02F011FE06003A
:1080D0000F0004980599614A614B02F097FB32004A
:1080E0003B0002F005FE069E079F0B0002003900D0
:1080F00030000292039302F0FBFD4B005B0D8346C0
:108100008A46E41A312C32DD04980599B822544B82
:10811000920502F07BFB03000C0002000293039423
:108120000B000698079902F0E3FD02000B00060021
:108130000F000698079902F0DBFD029A039B02F0FC
:10814000D7FD484A0290039104980599464B02F0E6
:108150005DFB029A039B02F0CBFD02000B00300096
:1081600039000292039302F0C3FD83468A465A46C1
:108170005346414630000A604B60390002F0B8FDBA
:10818000029A039B02F0B4FD44460B000200A26079
:10819000E3604B46002B00DB1BE75B46236080233C
:1081A0001B065344636080231B069C466144A06009
:1081B000E1606D420DE70B00020002F099FD4346BD
:1081C00000259860D9601860596002E7D3221A4BE5
:1081D000520502F08DFD214A214B0D00040002F0F2
:1081E00087FD02000B00414620000A604B60290019
:1081F00002F07EFD1A4B194A02F07AFD4346012532
:108200009860D960E5E602000B003000390002F00A
:108210006FFD6B1E154A9B009B5883468A46A342FE
:10822000A5D130E7FB21E93F7BD902400000405453
:10823000FB21F93F3163621A61B4D03DFB21394122
:10824000FFFFEF7FEAFBFFFF0000704198E10000B5
:1082500083C8C96D305FE43F0000E03F7370032EB8
:108260008A19A33BC14920259A837B3918E1000074
:10827000D3220C4B520501F0A3FB0B4A0B4B04001D
:108280000D0001F09DFB02000B00414620000A603A
:108290004B60290002F02CFD034A044BB9E603238E
:1082A00073E6C04661B4D03D7370032E8A19A33BB8
:1082B000F8B54746CE46674B80B50A000F00190057
:1082C00005003940994200D19BE004000100002FD5
:1082D00069DD3F1500D1B4E05F4B12039C4680235B
:1082E000120B5B0313435B00CA0F67449B184A00E1
:1082F000F80703D5D20F5B009B188A0079108C46D3
:10830000002180201624894680030D189D4202DC3E
:1083100029185B1B8144D50F5B00013C5B1952009F
:108320004008002CF1D10020804680202025002725
:10833000000609E08B425CD0D40F5B00013DE318DE
:1083400052004008002D16D0C4198B42F2DD2718C8
:108350000E00002C49DB5B1AA242894149425B1A9C
:10836000121BD40F5B00013D80443100E318520022
:108370004008002DE8D113434ED143465B083749EE
:108380004A468846494652104244C90702D58021D0
:1083900009060B4361460F05BD18180029000CBCE7
:1083A00090469946F8BD7B005B0803433900002BDB
:1083B000F5D0002F3CD1E30A153A6405002BFAD022
:1083C0008020400303423FD1002700E00F005B0004
:1083D000791C0342FAD0250020208D40401A290044
:1083E000D71B2200C2401A4376E7FE43F60F8E19D0
:1083F000B1E79442A0D82718002CF6DB1E0000231A
:10840000AEE702003B002800390002F0FFF92A0025
:108410003B0001F0D5FAC2E74346013303D043469F
:1084200001335B08ABE7012398460023C144A6E76C
:108430003B00020002F05CFC02000B0001F0DCFDDE
:10844000ADE713000022BBE70127210020207F4277
:10845000C6E7C0460000F07F01FCFFFF0000E03FE0
:10846000F0B54746CE4680B587B000920193754B74
:108470004F00814688467F089F4263DC02F09CFFE4
:10848000002800D1D4E04A4643464846414602F01F
:10849000BDF904000D006C4A6C4B02F0B7F96C4A50
:1084A0006C4B01F08DFA22002B0002F0AFF96A4A02
:1084B0006A4B02F01DFC22002B0002F0A7F9684A6B
:1084C000684B01F07DFA22002B0002F09FF9664A0A
:1084D000664B02F00DFC22002B0002F097F9644A73
:1084E000644B01F06DFA22002B0002F08FF902902C
:1084F00003910022604B2000290002F087F9029AC4
:10850000039B06000F002000290002F07FF9009A6B
:10851000019B04000D004846414602F077F9020035
:108520000B002000290002F0E3FB02000B003000EA
:10853000390002F0DDFB02000B0000204F4902F081
:10854000D7FB70E002000B0002F060F904000D00A0
:108550003D4A3E4B02F05AF93D4A3E4B01F030FA9B
:1085600022002B0002F052F93B4A3C4B02F0C0FBC8
:1085700022002B0002F04AF9394A3A4B01F020FA66
:1085800022002B0002F042F9374A384B02F0B0FBD0
:1085900022002B0002F03AF9354A364B01F010FA6E
:1085A0002B00220002F032F9354B029003919F42DA
:1085B0009FDD344B00229F423DDC334900207B1875
:1085C0002E4916001F0002F093FB04900591002233
:1085D000294B2000290002F019F932003B0002F07B
:1085E00087FB029A039B06000F002000290002F07F
:1085F0000DF9009A019B04000D004846414602F027
:1086000005F902000B002000290002F071FB0200B6
:108610000B003000390002F06BFB02000B000498E5
:10862000059902F065FB07B00CBC90469946F0BD79
:1086300000201249F7E7154B002604920593144FCA
:10864000C5E7C046FFFF3F3ED43888BEE9FAA8BD63
:10865000C4B1B4BD9EEE213EAD529C804F7E923E91
:108660009015CB19A001FA3E7751C1166CC1563F47
:108670004C5555555555A53F0000E03F0000F03FD3
:108680003233D33F0000E93F0000E0FF0000E73F46
:108690000000D23FF0B5DE464E4645465746E0B5AF
:1086A000DC4CA5440D9114001900A49A0993DA4BEF
:1086B0009200D6584D1E03901821E01E0696029592
:1086C00000F0A0FEC3430100DB1719404B1C9A00C9
:1086D0009B1ADB001B190B9105934C1B771918D4BF
:1086E000A59BA5009C463F1922AE6544013707E0D3
:1086F000286802F097FE013403C60435BC4208D056
:10870000002CF5DA00200021013403C60435BC42F8
:10871000F6D1069B002B01DA00F0FDFB069B0399C6
:108720000133DB009A46099BDA009446009200224E
:10873000914672AA0492B94A6144934688469AAB1C
:1087400063449B44029B002B00DABCE15D4600269B
:108750000027039C4D442A686B6803CC02F056F84E
:1087600002000B003000390001F02AF9083D060034
:108770000F004445EFD1049B4B441E605F6008230B
:108780009C46E144D145DDD10EA8042184464942EE
:1087900061448C46069A93009C44614684460A9143
:1087A0000399083B63448C460C93009B00926344FE
:1087B0009B46009A0498D10003008C4663440891BC
:1087C0001E685F68002A33DD954980468C46624406
:1087D000D300984470AB9A460EAB99460022914B59
:1087E0003000390002F012F802F0E6FD02F01AFE45
:1087F00000228D4B04000D0002F008F802000B006F
:108800003000390002F074FA02F0D6FD4B4601C385
:108810009946434620001A685B68290001F0D0F8A9
:1088200008235B429C46E04406000F00D045D5D1AA
:10883000059B30001A003900984600F0DFFCFF234A
:1088400000229B0504000D0001F0E0FF00F038FC61
:108850000022764B01F0DAFF02000B002000290015
:1088600002F046FA0D00040002F0A6FD814602F077
:10887000D9FD02000B002000290002F039FA0600A1
:1088800040460F00002800DCEEE0009B18215A1E35
:1088900092000EAB9B58091A1D000D41A9448D4052
:1088A0005D1B0EAB9D5017231B1A1D41002D2DDDA6
:1088B00001239C46009BE144002B00DC1CE20E9C43
:1088C0000123002C00D0B5E0009A012A09D09900BC
:1088D0000EAA54580133002C00D0ACE0009A9A4202
:1088E000F5D1059B002B0EDD012B00D1A8E1022B59
:1088F00009D1009B0EA95A1E92000EAB9B580793FC
:108900009B029B0A8B50022D00D1C1E00023002264
:108910003000390000F080FE009B002800D194E276
:10892000069A591E8A4210DC414A0A9894460EAAB9
:108930006344944600229B0063441C68043B22432A
:108940008342FAD1002A00D0C0E0069B0EAA013B68
:108950009B00D358002B00D0B3E001220C9B043BBA
:10896000596801320029FAD0009B9C4662441100EC
:1089700007921A0001338B4246DC0B98634680460F
:10898000A59C4344A046099C9B00A1464A449844A8
:10899000D30022AA9146049A99449446089BA59A2A
:1089A00063448446614494469A468B006344009332
:1089B0004346586802F036FD4B4618605960029BEA
:1089C000002B24DB4D46039C0026002701E028688D
:1089D00069680CCC01F01AFF02000B00300039006E
:1089E00000F0EEFF083D06000F005C45EFD1534656
:1089F0009E60DF6004239C460433E0449C46009B59
:108A0000E144E2449845D3D1079B0093D1E6002688
:108A10000027ECE794FDFFFFE0E2000018FEFFFFF7
:108A2000FFFFFF1F0000703E00007041000020406B
:108A3000FFFFFF3F002180225204141B0EAA545056
:108A4000009999420EDD0EA884469B000EAA89006B
:108A5000D25861446344CF4800E01A68821A04C3C4
:108A60008B42FAD101243CE7059B002B06D1009BE9
:108A70000EAA013B9B00D558ED1517E70022C64B07
:108A8000300000F0EDFD002800D024E100253DE796
:108A900032003B000020C14902F02AF906000F0015
:108AA000002C00D132E7059A0020BC4900F0A6FB5B
:108AB00002000B003000390002F01AF906000F0026
:108AC00024E7012250E70026002754E64B46059A8A
:108AD000079388468B000EA9CB58183A0895059243
:108AE000002B0DD18C464146AD4B43449B00634463
:108AF000043B58680139183A0028F9D08846059295
:108B0000059A0020A54900F079FB434604000D00BA
:108B1000002B00DA05E29E000EAB9C464346DB00CC
:108B200066449C46059370AB9946049F6744009742
:108B3000306802F077FC22002B0001F067FE002273
:108B400038607960974B2000290001F05FFE083FF4
:108B500004000D00043EB945EAD14AAB03939B469D
:108B600000239A46069B42469946434601320292AA
:108B700004934B46002B00DAAAE080208A4B009D2C
:108B80009846C005894900260027002408E00823EC
:108B90009C460835E044544511DC43461868596842
:108BA0002A686B6801F032FE02000B0030003900C9
:108BB00000F006FF013406000F00A145E7DA5B462E
:108BC000C0C39B4601239C46009BE244083B0093A4
:108BD000029B9A45CDD1049B9846A49B022B00DDB5
:108BE0008EE0002B37DC1FD1059B00271D00039B67
:108BF00000249C461E006544083E2A686B683800C5
:108C0000210000F0DDFE083D07000C00AE42F4D16B
:108C1000089B002B03D080231B069C4664443A002B
:108C200023000D990A604B600720079B18409B2387
:108C30009B009D443CBC90469946A246AB46F0BD85
:108C4000009B0EA95A1E92000EAB9B5807935B0225
:108C50005B0A8B5057E64346002B00DA70E1002098
:108C60000021DB004AAAD61848AF32687368083E74
:108C700000F0A6FEB742F8D1089B002B00D025E1FA
:108C80000B0002004A984B990D9C2260636002F031
:108C90002FF8434607000C00002B13DD01254CAED6
:108CA000B14638002E0021004C4601360CCC00F0B5
:108CB00087FEA146B045F7DA089B07000C00002BA1
:108CC00000D015E13A0023000D998A60CB60ABE734
:108CD0000026002773E701239C46009BE144022500
:108CE000002B00DDEBE532003B0000202B4901F0BA
:108CF000FFFF06000F0009E60024F2E54AAB0393EC
:108D0000A49B032B00D08FE74346002B00DC14E12B
:108D1000039ADB009B46130091465B441E685F6824
:108D2000234B43440293DB00994448AB9A464B469D
:108D30005C681B681800210032003B000090019124
:108D400000F03EFE04000D0002000B0000980199A7
:108D500001F0CEFF3B00320000F032FE4B4698603F
:108D6000D9601C605D6008235B429C46E14426009C
:108D70002F00CA45DBD14346012B00DCE3E0039A18
:108D800013005B441E685F68029BDB0099464A44FF
:108D9000904610E0FFFFFF000000E03F0000F03FC2
:108DA000FFFFFF3F0000703EA0E20000FB21F93F03
:108DB000FFFFFF1F984643465C681B6818002100B0
:108DC00032003B000090019100F0FAFD04000D001C
:108DD00002000B000098019901F08AFF32003B006D
:108DE00000F0EEFD4346039A9860D9601C605D6018
:108DF000083B26002F009A42DCD14D4694460026BF
:108E000000244746083565442A686B683000210015
:108E100000F0D6FD083D06000C00AF42F4D1039BE4
:108E20004A9F5D689968D868089B002B65D08022AE
:108E3000120694460D9B6544604464441F605D6067
:108E40009960D8601E615C61EEE69A464B460793D6
:108E5000059B30005A423900089500F0CFF90022F6
:108E60003A4B06000F0000F0FBFB002824D0384BE3
:108E700000223000390001F0C9FC02F09DFA524690
:108E80000400950002F0CEFA0022304B01F0BEFC47
:108E900002000B003000390001F02AFF02F08CFACA
:108EA0000EAA50510122059B524418339046059357
:108EB00093000EAAD45023E65346300039009C009C
:108EC00002F07AFA0EAB1851D04619E680230D9ABB
:108ED0001B06CB18106053600B0002004A984B9998
:108EE00001F006FF434607000C00002B00DDD5E62D
:108EF00080231B069C466444E4E62B003A000D9D4B
:108F00002A606B600A000300AA60EB603200230055
:108F10002A616B6188E6099BDB00009372AB0493C6
:108F200032E4A49B022B00DDE8E6002B00DD92E694
:108F300000D079E6002700246AE6002600246EE7C8
:108F40000020002198E60026340068E70000704108
:108F50000000703EF0B5CE46474680B587B000921F
:108F60000193474A4B00814688465B08934207DCE1
:108F70004146484602F020FA4146031E484666D064
:108F80004A4643464846414601F040FC04000D0075
:108F900002000B004846414601F038FC394A3A4B82
:108FA00006000F002000290001F030FC374A384B42
:108FB00001F09EFE22002B0001F028FC354A364BC2
:108FC00000F0FEFC22002B0001F020FC334A344B61
:108FD00001F08EFE22002B0001F018FC314B324ACA
:108FE00000F0EEFC0E9B02900391002B34D0009811
:108FF000019900222D4B01F009FC029A039B049079
:1090000005913000390001F001FC02000B000498CA
:10901000059901F06DFE22002B0001F0F7FB009A8C
:10902000019B01F065FE224A04000D00214B300037
:10903000390001F0EBFB02000B002000290000F0DA
:10904000BFFC02000B004846414601F051FE07B04C
:109050000CBC90469946F0BD02000B002000290090
:1090600001F0D4FB124A134B01F042FE32003B00E8
:1090700001F0CCFB4A46434600F0A2FCE7E7C046BD
:10908000FFFF3F3E7CD5CF5A3AD9E53DEB9C2B8A7A
:10909000E6E55A3E7DFEB157E31DC73ED561C119D5
:1090A000A0012A3F1111813FA6F810110000E03FF6
:1090B000495555555555C53F49004B08190070474E
:1090C000474AF0B54F4691464B005B0D99444646E2
:1090D000D6464A46C0B505000C000E00884607007B
:1090E000132A27DC002A4BDB3E4B13419A460B0028
:1090F00052461340034318D03B4A3C4B2800210002
:1091000000F05EFC0022002300F0A0FA002847D007
:10911000002C04DA80234A465B03134198444646F8
:10912000534600279E43380031001CBC90469946A8
:10913000A246F0BD332A08DD8023DB009945F4D137
:1091400002000B0000F03CFCEFE7294A94460122A4
:1091500063445242DA4092460242E6D0224A234B0E
:109160002800210000F02CFC0022002300F06EFA01
:10917000002815D0002C1EDB534646469F430FE0C7
:10918000194A1A4B2800210000F01AFC0022002383
:1091900000F05CFA002803D0002C04DB0027002636
:1091A00038003100C1E76400640825430027002D22
:1091B000F6D0104EF4E74B46142B0BD03422D21AC3
:1091C000012393405D19BD4208D201239C462F0024
:1091D000E044D1E7133B9C46E044CDE72F00CBE7CA
:1091E00001FCFFFFFFFF0F009C7500883CE4377E09
:1091F000EDFBFFFF0000F0BF002070474B0070B593
:109200005B0D14000A00002B1AD14B005B080343CE
:1092100015D0234B002201F0F9FA224B9C422DDBA2
:109220000A004B005B0D363B1F4DE318AB422ADCB6
:10923000002B0DDD1D4C1B0522401A43110070BD93
:109240001B4DAB42F0D102000B0000F0B9FBF6E77A
:109250001D00353519DA174B02009C4209DD0B0061
:109260001548164900F032F8134A144B01F0CEFAB3
:10927000E5E70B001248134900F028F8104A114B9B
:1092800001F0C4FADBE70200E9E7084C363322407C
:109290001B051343190000220B4B01F0B7FACEE770
:1092A00000005043B03CFFFFFE070000FFFF0F80AF
:1092B000FF07000050C300009C7500883CE4377E27
:1092C00059F3F8C21F6EA5010000903C30B54A006A
:1092D000DB0FDB0752081A43110030BD02B47146A0
:1092E00049084900095C49008E4402BC7047C046E9
:1092F000002243088B4274D303098B425FD3030AD5
:109300008B4244D3030B8B4228D3030C8B420DD3E7
:10931000FF22090212BA030C8B4202D31212090275
:1093200065D0030B8B4219D300E0090AC30B8B42B3
:1093300001D3CB03C01A5241830B8B4201D38B0361
:10934000C01A5241430B8B4201D34B03C01A524106
:10935000030B8B4201D30B03C01A5241C30A8B4249
:1093600001D3CB02C01A5241830A8B4201D38B0234
:10937000C01A5241430A8B4201D34B02C01A5241D8
:10938000030A8B4201D30B02C01A5241CDD2C3094A
:109390008B4201D3CB01C01A524183098B4201D3C6
:1093A0008B01C01A524143098B4201D34B01C01AB1
:1093B000524103098B4201D30B01C01A5241C30829
:1093C0008B4201D3CB00C01A524183088B4201D398
:1093D0008B00C01A524143088B4201D34B00C01A84
:1093E0005241411A00D20146524110467047FFE7F0
:1093F00001B5002000F0F0F802BDC0460029F7D00A
:1094000076E7704703460B437FD4002243088B4224
:1094100074D303098B425FD3030A8B4244D3030BFB
:109420008B4228D3030C8B420DD3FF22090212BAC0
:10943000030C8B4202D31212090265D0030B8B423C
:1094400019D300E0090AC30B8B4201D3CB03C01A26
:109450005241830B8B4201D38B03C01A5241430B01
:109460008B4201D34B03C01A5241030B8B4201D3F1
:109470000B03C01A5241C30A8B4201D3CB02C01A5C
:109480005241830A8B4201D38B02C01A5241430AD4
:109490008B4201D34B02C01A5241030A8B4201D3C3
:1094A0000B02C01A5241CDD2C3098B4201D3CB016A
:1094B000C01A524183098B4201D38B01C01A524119
:1094C00043098B4201D34B01C01A524103098B421D
:1094D00001D30B01C01A5241C3088B4201D3CB0008
:1094E000C01A524183088B4201D38B00C01A5241EB
:1094F00043088B4201D34B00C01A5241411A00D29B
:1095000001465241104670475DE0CA0F00D0494203
:10951000031000D34042534000229C4603098B4273
:109520002DD3030A8B4212D3FC22890112BA030AFB
:109530008B420CD3890192118B4208D3890192117D
:109540008B4204D389013AD0921100E08909C30902
:109550008B4201D3CB01C01A524183098B4201D304
:109560008B01C01A524143098B4201D34B01C01AEF
:10957000524103098B4201D30B01C01A5241C30867
:109580008B4201D3CB00C01A524183088B4201D3D6
:109590008B00C01A5241D9D243088B4201D34B00F1
:1095A000C01A5241411A00D20146634652415B1033
:1095B000104601D34042002B00D549427047634614
:1095C0005B1000D3404201B5002000F005F802BD59
:1095D0000029F8D016E770477047C046D0400B1CF2
:1095E0001141203A03D49C4613411843634652422A
:1095F000934018437047C0468446101C62468C4610
:10960000191C634600E0C0461FB501F097F800281A
:1096100001D40021C8421FBD10B500F0EFFF404249
:10962000013010BD10B501F089F8002801DB0020E1
:1096300010BD012010BDC04610B501F07FF8002814
:1096400001DD002010BD012010BDC04610B501F0A5
:1096500011F8002801DC002010BD012010BDC0461B
:1096600010B501F007F8002801DA002010BD012034
:1096700010BDC046F0B5CE46474615042D0C2E0051
:1096800080B50704140C3F0C9946030C7E435D43E0
:10969000674363437F19340CE4199C46A54203D900
:1096A00080235B029846C4444B4643435143250CF8
:1096B00036046544360C2404A4195B19591820009B
:1096C0000CBC90469946F0BDF0B54E46574645460F
:1096D000DE46E0B543025B0A450083B00F1C9946A5
:1096E0002D0EC60F002D57D0FF2D24D08020DB007B
:1096F000C0041843002381469A469B467F3D7C0266
:109700007A00FB0F640A120E984623D0FF2A4BD032
:10971000E30080240020E4047F3A1C43AD186B1C56
:1097200047460193534677403A000F2B48D87D496E
:109730009B00CB589F46002B00D085E008339A460B
:10974000063B9B467C027A00FB0FFF25640A120E43
:109750009846DBD1002C00D090E0524601231A43FA
:1097600092460120DBE74C4658461700022824D0D9
:10977000032800D1CFE00022002301284DD1580258
:10978000D205400AFF071043384303B03CBC904663
:109790009946A246AB46F0BD002B5BD104239A4606
:1097A000033B00259B46AAE7FF35002C60D15246BB
:1097B00002231A4392460220B1E7FF220023DEE78C
:1097C0004B461B0C9C464B462604360C180461463F
:1097D0003300220C6446000C43434E435043544331
:1097E00080191A0C1218964203D9802149028C461E
:1097F00064441B041B0C1004C01883015E1EB3419B
:10980000800E1843130C1B199B0103431C002301FA
:1098100079D5012362081C401443019A7F32002A43
:109820004DDD630704D00F232340042B00D0043404
:10983000230103D53C4B019A1C408032FE2ABCDC3C
:10984000A3015B0AD2B29AE70C239A46093BFF2593
:109850009B4654E7180001F071FE4A46431F7625E7
:109860009A4000236D4291462D1A9A469B4646E740
:10987000524603231A439246032050E7200001F08A
:109880005DFE431F2D1A9C40763D002047E7802354
:109890000027DB03FF2272E7424666E74C463200B0
:1098A000584662E780234A46DB031A4222D01C4214
:1098B00020D123435B025B0A4746FF225FE7012377
:1098C0009A1A1B2A21DC23000199D3409E318C4037
:1098D0001A0023005C1EA34113435A0704D00F2231
:1098E0001A40042A00D004335A0111D49B015B0AA8
:1098F000002244E780234A46DB0313435B025B0AF2
:109900003700FF223BE7019587E70022002336E777
:109910000122002333E78023DB0323435B025B0A3E
:10992000FF222CE7F0E20000FFFFFFF770B50028F0
:109930003DD0C317C5185D40C40F280001F0FEFDDF
:109940009E22121A962A07DCD2B2082833DD083884
:1099500085406802400A23E0992A0BDD052329008F
:109960001B1AD94003001B339D402B005D1EAB41E9
:1099700019430D00052801DD431F9D402B000F49B1
:109980000B406E0709D00F263540042D05D0043357
:109990005D0102D59F220B40121A9B01580AD2B2D8
:1099A0004002D205400AE4071043204370BD002462
:1099B00000220020F4E76802400AF1E7FFFFFFFB06
:1099C000F0B54F464646D6460C000903C0B5490AD5
:1099D000470F5E0039431F03DB0F9C4665007B0A7F
:1099E000570F1F436D0DE40F760DA146C000B8461A
:1099F000D200AB1B64457BD0002B5FDD002E00D076
:109A0000A4E03E00164300D112E15E1E002E00D0FD
:109A10009EE1871A4346B84280410125C91A404257
:109A2000091A0B0200D431E149024E0A002E00D17E
:109A30006EE1300001F082FD0300083B1F2B00DDCA
:109A400061E120223900D21A9E40D1409F400E434E
:109A50009D4200DD51E15D1B6B1C1F2B00DD7CE195
:109A60002021C91A3D0030008F408840DD40791E1A
:109A70008F41310007222843D940002507433A404F
:109A8000002A09D00F233B40042B05D03B1DBB42CD
:109A9000BF417F42C9191F000B0200D426E26A1C95
:109AA000C64B55056D0D9A4200D106E1C44AFF0828
:109AB0000A40530752023B43120B8EE0002B00D0AA
:109AC000B8E06B1C5B055B0D012B00DC30E1871AF5
:109AD0004346B842B641CB1A76429E1B330200D5AC
:109AE0004CE13B003343A1D100220024002570E06B
:109AF000002B00DCE5E0002E00D183E0AF4EB54244
:109B000060D0802636043743B846382B00DC3EE16F
:109B1000434613431F007A1E97413F1887428041F6
:109B2000404209180B0200D4B0E0A44B01359D421D
:109B300000D1C3E0A24A7B080A4001210F401F4325
:109B40005108D30707221F433A4099E79B4EB5427D
:109B500038D0802636043743B846382B00DDDCE0A9
:109B60001F2B00DC30E11E004746203EF740BC467C
:109B7000202B04D04026F31A46469E40324317005D
:109B800063467A1E97411F43CCE0002B00D104E2CC
:109B90004346134300D159E14B07C00818438023C3
:109BA000C9081B03194208D04546ED081D4204D1DF
:109BB0004346D008590708432900420FC9007F4D8A
:109BC0001143C0004B07CA087C49C00803438D42BB
:109BD00068D012036D05120B6D0D002112031800E1
:109BE000130B0A0D12051A43764B2D0513402B4318
:109BF0005B00E4075B08234319001CBC90469946B0
:109C0000A246F0BD3E00164312D05E1E002E00D0CC
:109C100000E18718874280414144404209180125EC
:109C20000B0233D5022585E7644633004146100018
:109C30001D00C7E7002D00D0DAE00C000443F3D08C
:109C40005C1C00D19FE15D4CA64200D12FE1DB43BB
:109C5000382B00DD66E11F2B00DD83E120240500A9
:109C6000E41A0F00DD40D940A0404346A7405B1AEC
:109C7000441EA04198462F433843171ABA429241D6
:109C800043465242991A64463500CAE607223A40D2
:109C9000002A00D0F6E64B07CA084849FF083B43B4
:109CA0008D4296D11900114300D19EE18021090314
:109CB0000A431203120B414D8FE7150000220023C7
:109CC0008BE7002B00D0C7E06B1C5F057F0D012FD9
:109CD00000DCF1E0394DAB4200D1B9E085180A0053
:109CE000854289414244494251180722CF076D08F5
:109CF0002F4349083A401D00C2E607223049ED1AB9
:109D000031403A40BCE63E002838864000279FE6B6
:109D1000380001F013FC20308EE6434613431F0049
:109D20007A1E9741C71BB84280414042091A78E623
:109D30000E003B0006431343002D61D1002E00D0DE
:109D4000F4E0002B00D11BE164463900100039E734
:109D50001A4FBB427AD03300FFE630001F3DE84087
:109D6000202B03D04021CB1A9E4037437B1E9F41BE
:109D7000072207433A400021002589E7171A434686
:109D8000BA42B641591A76428E1B64464EE61F2BE4
:109D900000DDADE020264746F61AB740B946170069
:109DA000B246DF404E463E4337005646B240561E4E
:109DB000B24117434246DA408918AEE6FF07000079
:109DC000FFFF7FFFFFFF0F8020264746F61AB740B0
:109DD000B9461700B246DF404E463E43370056466E
:109DE000B240561EB24117434246DA40891A99E7FB
:109DF0007F4CA6425BD0802424045B42214327E7AA
:109E0000002E0CD1002B00D1CBE0644639001000AD
:109E1000774DD7E6764FBB4218D0330075E6002B5E
:109E200014D04B07C00818438023C9081B031942EC
:109E300007D0FC081C4204D17907D0080843E1464A
:109E400021004C46420FC9001143C000684DB9E6DD
:109E50001D0000220023C0E6002D5BD10D0005434C
:109E600000D1E2E65D1C00D1B0E0614DAE421FD0F2
:109E7000DB43382B71DC1F2B00DD96E020250F0023
:109E8000ED1AAF40B9460700AA46DF404D463D43B4
:109E90002F005546A840D940451EA8418844074395
:109EA000BF18974292415142414435003AE6644618
:109EB00035004146100085E60B000343002D00D01D
:109EC00063E6002BF5D04346134300D17AE68718AA
:109ED0008742804107224144404209183A400B0220
:109EE00000D4D5E6434B01351940C9E5380069E691
:109EF0001E004746203EF740BC46202B04D040269B
:109F0000F31A46469E403243170063467A1E974135
:109F10001F4302E6364DAE42CAD080252D045B4277
:109F20002943A6E70843411E8841A6E6002B00D13D
:109F300048E6871A4346B842B641CB1A76429E1B82
:109F400033024BD5171A4346BA429241591A52422C
:109F5000891A072264463A4092E501430F00791EB0
:109F60008F419DE71C000F00203CE740202B03D0D1
:109F70004024E31A99400843411E884138437CE657
:109F80000022002425E6171A4346BA429241591A84
:109F90005242891A6446350043E541461000144D8B
:109FA00010E680220024120380E61D000F00203DF1
:109FB000EF40BC46202B03D04025EB1A99400843C4
:109FC00007006346781E87411F4369E78718974259
:109FD0009B4141445B42C9183500A3E53B00334334
:109FE000CED0072231003A4052E600231A00F4E5B1
:109FF000FF070000FFFF7FFFF0B55746DE464E46E5
:10A000004546E0B5834607000E03480085B09246FA
:10A010001C00360B400DCD0F002800D19DE0954B64
:10A02000984239D08023F6001B041E43924A7B0FCE
:10A03000334399469446030063440093002300266B
:10A04000FF00029323031B0B98466300E40F524664
:10A050005B0D019400D1B3E086498B4200D19EE0B4
:10A060004246D100802212040A435146490F11434F
:10A070008B46814952468C4600996344CB1A002195
:10A08000D20000932B0063409A460F2E00D905E1C1
:10A090007A4BB6009B599F465B463343994600D0A6
:10A0A000B8E002230826002700900293CAE7CB46B7
:10A0B0003A0002990195019B9A46022927D003296B
:10A0C00000D180E2012944D06D49009B8C46634455
:10A0D0001C00002C38DD530700D013E2D2085B4689
:10A0E000DB0109D55946674B19408B468021C900D1
:10A0F0008C46009B63441C00634B9C4207DC5B4620
:10A1000064055F075B0217431B0B620D02E000232F
:10A110000027584A00211B031C0B0B0D1B05234372
:10A1200014055A4A380013401C4353466400DB07A9
:10A1300064081C43210005B03CBC90469946A246E9
:10A14000AB46F0BD0122524201231B1B382B00DC21
:10A15000ADE1002200230027DCE75B46334399464C
:10A160005ED0002E00D18AE1300001F0E7F9030053
:10A170000B3B1C2B00DD7BE11D22D31A5A4601004C
:10A18000DA4008398E4013005F46334399468F40CA
:10A190003F4B00261B1A00930023029352E74146CF
:10A1A00053460B433B499B468C46009B63440093BC
:10A1B0005B46002B3BD1022300221E43022161E7B4
:10A1C000434613439B4637D04346002B00D162E100
:10A1D000404601F0B3F903000B3B1C2B00DD53E1BB
:10A1E00002004146083A914088461D21CB1A51464B
:10A1F000D9400B0041460B439B46534693401A00FF
:10A20000009B25499C46604403008C4663440093B0
:10A21000002137E70323B14600900C26029311E793
:10A220000023009301330426002702930AE7032347
:10A23000C3461E43032125E701331E4300220121AB
:10A2400020E700239A46802300271B03094A61E781
:10A25000802349461B03194200D1E2E059461942C6
:10A2600000D0DEE00B431B0317001B0BA246014A84
:10A2700050E7C046FF07000001FCFFFF30E300008D
:10A28000FF030000FFFFFFFEFE070000FFFF0F803F
:10A290000DFCFFFF01F8FFFFF3030000D94500D9D3
:10A2A000CBE000D1C6E03C0048460027009B013BC4
:10A2B00000935B46160E1B021E431302984633049E
:10A2C0001B0C9946310C0191FFF798F84A4642431E
:10A2D0000B04210C050019438A4207D98919013D55
:10A2E0008E4203D88A4201D9851E8919881A01999C
:10A2F000FFF784F809048C464A4621046446424329
:10A30000090C030021438A4204D98919013B8E427A
:10A3100000D8F1E02D041D43AB464346891A42465E
:10A32000280C12041D0C5B46140C22001B041B0C91
:10A330005A4303946B434443029568431B19150C1D
:10A34000EB189C4203D980246402A44660441C0C90
:10A3500015041B042D0C20185D19814277D373D08E
:10A360000C1AA24A7D1BAF42BF419446009B7F421C
:10A370006344E01B1C00864200D1DBE00199FFF73B
:10A380003DF84A4642430B04290C070019438A4210
:10A3900007D98919013F8E4203D88A4201D9871E05
:10A3A0008919881A0199FFF729F809044A4689464C
:10A3B00029044D464243090C030029438A4207D928
:10A3C0008919013B8E4203D88A4201D9831E89191B
:10A3D0003F04891A3A00039F1A43380013041B0CE8
:10A3E000584381460298150C6F4343434543484602
:10A3F000000C8446DB1963449F4203D9802040024D
:10A400008446654448461F0C00041B04000C7D195B
:10A410001818A94200D284E000D17FE001231A433A
:10A4200057E680234A461B0313431B031B0BAA4614
:10A430006F4A6FE6BA4200D935E74B46DC07580849
:10A440007B081C43FF0734E70024AF4289D247440E
:10A450004745A4415B466442A4196418013BA642E7
:10A460001ED2A0426DD800D1B6E0241A9B4678E7F0
:10A4700003005A46283B9A400027914688E65846F2
:10A4800001F05CF8203072E603005246283B9A4007
:10A4900093460022B4E6504601F050F820309AE688
:10A4A000A642E2D1B845DCD9341A9B4659E71F2BA6
:10A4B00065DC504C0099A4465C46614408008C4021
:10A4C00011008240D940501E82410C4314435A4629
:10A4D000DA401300620709D00F222240042A05D077
:10A4E0002200141D9442894149425B181A0262D528
:10A4F0000122002300270DE68A4200D80AE7831EC6
:10A50000891907E70F231340042B00D1E6E5171D37
:10A510009742924153429B44FA08E0E5002800D15B
:10A52000D7E57118531EB14227D3A94215D358D08D
:10A530001A0073E7002B00DC04E6012300229B4491
:10A54000CDE502234744474589415B429C46494249
:10A5500089190C19E344241A03E743465F00474571
:10A560009B41B8465B429E19023A8919A94200D024
:10A5700054E7404500D051E7ABE51A00F6E71F214C
:10A580005F4649420C1BE740202B07D01A49009B2D
:10A590008C46634418005B4683401A43501E824138
:10A5A0003A4307270023174009D00F210023114009
:10A5B0001400042995D122005F075B021B0BD2080F
:10A5C00017430022A6E5802359461B030B431B03B8
:10A5D00017001B0B064A9DE5BD42B2D89B460024DE
:10A5E000BFE68045B9D31A00C3E7C046FF030000A9
:10A5F000FF0700001E0400003E040000F0B54F46B7
:10A600004646D6468446C0B58046194E18030F0309
:10A610004D00000B5C0082463F0B6D0DC90F91464B
:10A62000640DDB0F0120B5420AD0B44203D0A5422D
:10A6300001D157450CD01CBC90469946A246F0BDAE
:10A6400066463E43F7D1AC42F5D154461443F2D1AD
:10A650000120C845EFD1994207D0002DEBD16346C8
:10A660001F433800471EB841E5E70020E3E7C04636
:10A67000FF070000F0B54F464646D6464D00C0B530
:10A680000E03C90F8A462C491F035C008046360B17
:10A690006D0D91463F0B640DDB0F8D421ED08C4239
:10A6A00016D0002D1ED130438446002C01D13A43F0
:10A6B00023D06246002A1AD09A4529D0514602205A
:10A6C0000139084001381CBC90469946A246F0BDAD
:10A6D00039001143E5D002204042F4E73043FAD17B
:10A6E000AC420FD0002C0FD13A43E7D00CE001224E
:10A6F000013B934318000130E5E763460020002B3F
:10A70000E1D0DBE73A43E6D19A45D7D1A542D5DC83
:10A71000A54205DBBE42D1D808D00020BE42D2D22D
:10A7200050460123013898430130CCE7C845C5D8CD
:10A730000020C845F4D3C6E7FF070000F0B54F4638
:10A740004646D6464D00C0B50E03C90F8A462E496F
:10A750001F035C008046360B6D0D91463F0B640D68
:10A76000DB0F8D4218D08C4211D0002D18D1304310
:10A770008446002C1ED13A431CD163460020002B96
:10A7800030D0514602200139084001382AE0390012
:10A790001143EAD0022025E03043FBD1AC4226D061
:10A7A000002C26D13A4324D15146022001390840D9
:10A7B000013817E06246002A0FD09A45E1D1A54240
:10A7C00005DBBE42DDD819D00020BE420AD2504679
:10A7D000012301389843013004E00122013B9343F7
:10A7E000180001301CBC90469946A246F0BD3A4381
:10A7F000D0D19A45C5D1A542C3DCE0E7C845C0D851
:10A800000020C845E3D3EDE7FF070000F0B5574649
:10A81000DE464E464546E0B5834606000F03480037
:10A8200087B092461D003F0B400DCC0F002800D191
:10A830006FE0DE4B984238D08023FF001B041F439B
:10A84000730F3B430193DA4B0027994600239B4645
:10A85000F60081442B0369001B0B52469846490DB4
:10A86000ED0F002900D185E0D04B994200D173E073
:10A870004346DA0080231B0413435246CC48520F50
:10A8800084461343524600206144D200894421008B
:10A89000694000918C46012149448A460F2F00D916
:10A8A00090E0C449BF00CF59BF465B463B4301938C
:10A8B00000D06AE102230827002681469B46C9E7AB
:10A8C00032005846019B61460091022800D175E094
:10A8D000032800D1FEE1012800D02CE1002300274D
:10A8E000002600253F032A0D3F0BB34812053A43CB
:10A8F00002401B051343009A5B00D1075B080B4322
:10A900003000190007B03CBC90469946A246AB46C1
:10A91000F0BD5B463B43019300D12FE1002F00D1F6
:10A92000A5E1380000F00AFE03000B3B1C2B00DD04
:10A9300096E11D22D31A5A460100DA405E460839D4
:10A940008F4013008E403B4301939C4B00271B1A02
:10A95000994600239B467DE7414653460B43934966
:10A960008C46E144002B00D01AE10222022017435A
:10A9700000228CE7134300D10DE14346002B00D1A8
:10A9800081E1404600F0DAFD02000B3A1C2A00DDAE
:10A9900072E10100434608398B4098461D239A1AFC
:10A9A0005346D3401A004346134352468A40494611
:10A9B000081A824989468144002068E77B4B0027BA
:10A9C00000268EE7140C1204120C1100370C36040A
:10A9D000350C794328008C462E0060436044834642
:10A9E00056432100300C804658467943404402913A
:10A9F000844506D98846802149028C46E044414678
:10AA000002913604010C360C00048B4681191E0C91
:10AA10001B041B0C0391190079438C4628007543D5
:10AA20006544A8465843050C45447743A94203D9D9
:10AA3000802149028C466744290C8C463900000469
:10AA4000000C2D042D186144AB4405915946049126
:10AA500001990F043F0C080C3900514342439046C2
:10AA600002008C46090C8B4662437C4344445C44A0
:10AA7000A04503D98021490288464244210C8846DA
:10AA800061460904090C8C4639005943434370431D
:10AA90007E430F0CF6182404BE19644442448C46CD
:10AAA000B34203D980235B0298464044029B61462F
:10AAB0009846049B370443449B46AB45AD416B42EB
:10AAC0000D0405992D0C8C467F196744FD18A84686
:10AAD0005D462D19A542A44193466442A446C34451
:10AAE000DC448F42BF4198459B4193459241A44528
:10AAF000A4415B427F421F43360C52426442BF195D
:10AB00002243BF18624638184302D20D03991343FB
:10AB10006A020A43501E82416146ED0D2A434E02ED
:10AB20003243D90100D4B3E0012650083240024339
:10AB3000DE0732435B08224C5444002C62DD51078F
:10AB400009D00F201040042805D0101D90429241DA
:10AB500052429B180200D90104D580241948E40010
:10AB6000034054441848844200DD27E75E075B0237
:10AB7000D2081F0B630516435B0DB2E6002399460E
:10AB80000133042700269B4664E603230197814690
:10AB90000C279B465EE6012201201743002276E641
:10ABA000032303201F43434671E6C046FF0700000E
:10ABB00001FCFFFF70E30000FFFF0F800DFCFFFFB3
:10ABC000FF030000FFFFFFFEFE07000000238027B9
:10ABD00000933F030026434B83E6019B3200A446CB
:10ABE000584670E6AC466EE6802701993F0339422D
:10ABF0002DD03B422BD11F433F033F0B0095160046
:10AC0000384B6EE601252D1B382D00DD66E61F2D25
:10AC100040DC35481C005044160082408440EE4021
:10AC2000501E824134431443EB40620709D00F2287
:10AC30002240042A05D02200141D94428041404243
:10AC40001B181A023ED501230027002649E680275B
:10AC5000019B3F031F433F033F0B0094214B40E602
:10AC600003005A46283B9A40002601926DE658465A
:10AC700000F064FC203057E603005246283B9A401F
:10AC80001300002293E6504600F058FC20307BE68B
:10AC9000CA4650E71F201E004042041BE640202DFC
:10ACA00003D0124C5444A3401A43501E82413243F5
:10ACB00007260027164009D00F200023104014005B
:10ACC0000428B9D122005E075B021F0BD20816438D
:10ACD000002306E680273F031F433F033F0B160078
:10ACE000004BFEE5FF0700001E0400003E040000CC
:10ACF000F8B557464E464546DE460C000903E0B51A
:10AD0000490A460F5F0031431E03DB0F760A9B465C
:10AD1000530F3343C84E6500C000E40FD2006D0DE1
:10AD2000A24681467F0D9C469046B74200D1B9E0CD
:10AD30005B46012673409B46EE1BA34500D183E092
:10AD4000002E63DD002F00D0B1E06346134300D135
:10AD500023E1731E002B00D0BAE1861A6346B0428D
:10AD600080410125C91A4042091A0B0200D447E16B
:10AD700049024B0A98464346002B00D189E14046E0
:10AD800000F0DCFB0300083B1F2B00DD7CE12022F0
:10AD90003000D21A4146D040994002009E400A43FA
:10ADA0009D4200DD6AE15D1B6B1C1F2B00DD94E101
:10ADB000202110003500C91A8E40DA408840DD405D
:10ADC000711E8E41110007222843002506433240A0
:10ADD000002A09D00F233340042B05D0331DB34282
:10ADE000B641764289191E000B0200D43DE26A1C6E
:10ADF000914B55056D0D9A4200D119E18F4AF60825
:10AE00000A40570752023743120B9BE0002E00D036
:10AE1000C5E06E1C7605760D012E00DC48E1674624
:10AE2000861ACB1BB042BF417F42B8461F00434643
:10AE3000FF1A3B00B8461B0200D55FE137439AD1A9
:10AE400000220024002579E0002E00DCFAE0002F2B
:10AE500000D18DE0784B9D4267D0802367461B046C
:10AE60001F43BC46382E00DC52E1634613435A1E92
:10AE700093411E1886428041404209180B0200D4BB
:10AE8000BEE06D4B01359D4200D1D2E06B4A7308A4
:10AE90000A4001210E401E435108D30707221E43DA
:10AEA000324095E71E00164300D045E740E7624B6D
:10AEB0009D423AD0802367461B041F43BC46382E70
:10AEC00000DDEBE01F2E00DC3AE133006746203B5B
:10AED000DF403B00202E05D04027BF1B6646BE400A
:10AEE000324390464646721E96413343DAE0002BC9
:10AEF00000D114E26346134300D168E180234E077A
:10AF0000C008C9081B030643194208D06046C008A0
:10AF1000184204D163460100D2085E071643F300CD
:10AF20009946C900720F444D11434B46DE08424B0F
:10AF30004F073743CA089D4200D16EE012036D05EA
:10AF4000120B6D0D00211203130B0A0D12051A438B
:10AF50003B4B2D0513402B435B00E4075B08234369
:10AF6000380019003CBC90469946A246AB46F8BD55
:10AF70006346134311D0731E002B00D007E18618DF
:10AF80008642804161444042091801250B0237D5B1
:10AF900002257BE73E00614691463500C5E75C46E9
:10AFA000002D00D0E1E00B000343F3D0731C00D16F
:10AFB000ACE1214B9F4200D13AE1F343382B00DD55
:10AFC0006FE11F2B00DD8CE120250E00ED1AAE4055
:10AFD000B0460600AA46DE40454635432E0055469B
:10AFE000D940A8406346451EA8415B1A9C463043A1
:10AFF000161AB242924163465242991A3D00B4E693
:10B0000007223240002A00D0E4E60B4BF6084F0737
:10B010003743CA089D4200D090E73B00134300D15C
:10B02000A6E180231B031A431203120B024D89E78A
:10B0300015000022002785E7FF070000FFFF7FFFC4
:10B04000FFFF0F80002E00D0C7E06B1C5E05760D61
:10B05000012E00DCF0E0C84DAB4200D1B9E085180C
:10B060000A00854289416244494251180722CE07AD
:10B070006D082E43490832401D00A9E6BF49ED1A6C
:10B08000114007223240A3E63200283882400026D1
:10B0900086E6300000F052FA203073E66346134330
:10B0A0005A1E9341C61AB04280414042091A5CE6DA
:10B0B0000E00674606431743002D5ED1002E00D0D8
:10B0C000F3E0002F00D11EE15C46614691462CE77B
:10B0D000A94FBE427BD01E00F1E610001F3DE840A4
:10B0E000202B03D04021CB1A9A401643731E9E4159
:10B0F0000722064332400021002583E7161A6346E3
:10B10000B2428041591A40420B1A98465C4632E6D8
:10B110001F2E00DDABE02027BB1B9A466346574637
:10B12000BB40994613004F46F3401F433B00574630
:10B13000BA40571EBA4113436246F240891898E656
:10B140002027BB1B9A4663465746BB4099461300CF
:10B150004F46F3401F433B005746BA40571EBA4183
:10B1600013436246F240891A9CE7834B9F425FD0AB
:10B1700080252D047342294320E7002E0CD1002F97
:10B1800000D1D0E05C46614691467B4DCDE67A4FDA
:10B19000BE421CD01E0065E6002F18D0C0084E0726
:10B1A00006438020C9080003014208D06346DC083A
:10B1B000044204D12100DA46D2085E071643F300A8
:10B1C000994601245346C900720F11431C406A4D31
:10B1D000ABE61D0000220027B4E6002D59D10B007C
:10B1E000034300D1D6E6731C00D1B2E0624B9F420C
:10B1F0001ED0F343382B6FDC1F2B00DD97E020259A
:10B200000E00ED1AAE40B0460600AA46DE404546A6
:10B2100035432E005546A840D940451EA8418C44D0
:10B220000643B61896429241514261443D0025E6DC
:10B230003D006146914678E60B000343002D00D0A7
:10B2400055E6002BF5D06346134300D16DE6861812
:10B250008642804161444042091800220B0200D41A
:10B26000D0E6464B01351940B2E5B1465DE6330004
:10B270006746203BDF403B00202E05D04027BF1B08
:10B280006646BE40324390464646721E9641334360
:10B29000EFE5394B9F42CBD080252D0473422943E3
:10B2A000A8E70843411E8841A2E6002F00D13CE6F2
:10B2B0006346861ACF1AB0429B415B42FB1A9846FE
:10B2C0001B024ED5161A6346B2429241591A524297
:10B2D000891A5C4600227BE501430E00711E8E41F7
:10B2E0009FE71D000E00203DEE40B046202B04D00D
:10B2F0004025EB1A99400843814648464346411E83
:10B300008841184374E60022002417E6161A6346A3
:10B31000B2429241591A5242891A3D0025E56146CE
:10B320009146154D01E680220024120379E61D00A6
:10B330000E00203DEE40B046202B04D04025EB1AF5
:10B340009940084381464E464346711E8E411E4336
:10B3500067E7861896429B4161445B42C9183D00ED
:10B360008CE547463743CED007224146324049E676
:10B3700000273A00E6E5C046FF070000FFFF7FFF19
:10B3800070B50C4E0D031C0349005B002D0B490DDD
:10B39000240B5B0DB14208D0064900208B4203D13B
:10B3A00014432000441EA04170BD05430120002D20
:10B3B000FAD1F1E7FF07000030B5144D0A034B0046
:10B3C000120B5B0DC90F0024AB4211DD104CA342E0
:10B3D00010DC8024640322430E4CE41A1F2C0CDD85
:10B3E0000D48C31ADA4013005C42002900D11C004A
:10B3F000200030BD094BCC18FAE7094DE040AC46BF
:10B4000063449A4013000343EEE7C046FE03000086
:10B410001D0400003304000013040000FFFFFF7F41
:10B42000EDFBFFFF70B500282DD0C317C5185D4098
:10B43000C40F280000F082F8154B1B1A5B055B0D4A
:10B440000A2815DD0B38854000222D032D0B002125
:10B4500010002D030A0D2D0B12052A430D4D1B055F
:10B460002A4013435B00E4075B082343190070BDC7
:10B4700002002900153291400A000B21081AC5402C
:10B480002D032D0BE3E70024002300250022DEE737
:10B490001E040000FFFF0F804100090E4B1C70B519
:10B4A000DBB24602750AC40F012B14DDE0239B00BA
:10B4B0006D07360BCB1800210A0D280012051C4D14
:10B4C00032435B052A405B0813435B00E4075B08DB
:10B4D0002343190070BD002914D1002D1ED028006F
:10B4E00000F02CF80A281CDC0B232A001B1ADA4077
:10B4F000030015339D400F4B12031B1A5B05160BFF
:10B500005B0DD8E7002D06D0320B802636036D0781
:10B510001643094BCFE7084B0026CCE70023002653
:10B52000C9E703002A000B3B9A400025E3E7C04629
:10B53000FFFF0F8089030000FF0700001C2101238B
:10B540001B04984201D3000C10391B0A984201D306
:10B55000000A08391B09984201D30009043902A2E4
:10B56000105C40187047C04604030202010101014B
:10B57000000000000000000030B51C00094B050071
:10B580001B6885B0D868084B002A01D1074B1A0008
:10B590000292019300912B002200054900F026F849
:10B5A00000F0A6FD80000020B0E30000C7D100003D
:10B5B000BDE30000014B18687047C04680000020C2
:10B5C000084B10B50400002B02D0002100E000BFA2
:10B5D000054B1868836A002B00D09847200001F0C3
:10B5E0005DFBC04600000000ECE300000EB403B5B4
:10B5F000010003AB044804CB0068019300F076F827
:10B6000002B008BC03B018478000002070B50026C7
:10B610000C4D0D4C641BA410A64209D1002601F06C
:10B620003FFB0A4D0A4C641BA410A64205D170BD15
:10B63000B300EB5898470136EEE7B300EB58984754
:10B640000136F2E750020020500200205002002094
:10B6500060020020002310B59A4200D110BDCC5CDE
:10B66000C4540133F8E710B5884202D98B189842C8
:10B6700003D3002307E08B5C8354013AFBD210BD57
:10B68000CC5CC45401339A42FAD1F8E70300121893
:10B69000934200D1704719700133F9E7936810B5F0
:10B6A000013B9360002B04DA9469A34207DB0A296B
:10B6B00005D01368581C10601970080010BD00F008
:10B6C0004BFC0100F9E7F8B506000F001400D5188F
:10B6D000AC4201D1002007E021783A003000FFF7AA
:10B6E000DDFF0134431CF3D1F8BD0000F0B59FB07D
:10B6F00002900F0016000593002805D0836904937B
:10B70000002B01D100F0F4FD7B4B9F425BD1029BEB
:10B710005F68BB891B0762D53B69002B5FD00023A4
:10B7200006AC6361203363761033A37635002B7843
:10B73000002B01D0252B5CD1AB1B04930CD0320025
:10B7400039000298FFF7BFFF431C00D1C4E06269D3
:10B75000049B9446634463612B78002B00D1BBE0CB
:10B76000012200235242626002A9543252186E1C18
:10B770002360E360A3601370A365317805225F48FE
:10B7800000F0D4FE751C002835D12268D30604D5FC
:10B79000532302A95B1820211970130704D55323E2
:10B7A00002A95B182B21197033782A2B2CD0350075
:10B7B00000210A20E3682A786E1C303A092A64D9ED
:10B7C00000292ED026E04E4B9F4202D1029B9F685B
:10B7D0009FE74C4B9F429CD1029BDF6899E7390061
:10B7E000029800F00FFC002899D0012040421FB0C1
:10B7F000F0BD01359BE7414B2268C01A012383400D
:10B80000134323602E00B8E7059B191D1B680591A3
:10B81000002B01DB099304E05B42E3600223134346
:10B8200023602B782E2B0AD16B782A2B35D1059BE0
:10B8300002351A1D1B680592002B2BDB0793324E35
:10B8400029780322300000F071FE002806D0402342
:10B85000801B834022680135134323602978062228
:10B860002A486E1C217600F061FE00283AD0284B51
:10B87000002B25D10722059B0733934308330593FB
:10B880006369039A9B18636150E7434301219B1846
:10B89000350090E701235B42D0E700230A201A001D
:10B8A0000135636029786E1C3039092903D9002BD2
:10B8B000C5D00792C3E74243012352183500F1E790
:10B8C00005AB00933A00134B2100029800E000BF43
:10B8D0000390039B0133D3D1BB895B0600D584E77A
:10B8E0000B9884E705AB00933A000A4B21000298BD
:10B8F00000F080F8ECE7C04644E40000F0E300000C
:10B9000064E4000024E40000F6E30000FAE3000031
:10B9100000000000C7B60000F7B5150001938A6863
:10B920000B6900900C00934200DA130022002B6098
:10B9300043321278002A01D001332B6023689B0622
:10B9400002D52B6802332B60062723681F4027D0BF
:10B95000230043331B785A1E93412268920630D449
:10B960002200019943320098089EB047431C25D01D
:10B97000062320682A68E16803400025042B03D1D0
:10B980008D1AEB43DB171D40A3682269934201DD4A
:10B990009B1AED180027BD4220D1002010E001378E
:10B9A000E3682A689B1ABB42D2DD220001231932C8
:10B9B00001990098089EB047431CF0D101204042F5
:10B9C000FEBD3020E1184331087021005A1C45317A
:10B9D0000978A218433202331170C1E72200012313
:10B9E0001A3201990098089EB047431CE6D00137EF
:10B9F000D1E70000F0B589B004920A004332059304
:10BA0000039002920A7E0C000E9B6E2A00D186E003
:10BA10001FD8632A33D008D8002A00D18CE0582AD6
:10BA20004DD0250042352A7030E0642A01D0692AC1
:10BA3000F7D1196825680A1D280629D508681A60F3
:10BA4000002803DA2D23029A404213706B4E0A2716
:10BA50004FE0732A74D008D86F2A1FD0702AE0D123
:10BA6000202209680A43226003E0752A16D0782A4A
:10BA7000D7D12200782145321170614E22E0250095
:10BA80001A684235111D196013682B70012365E097
:10BA900008681A606906D3D500B2D1E7196825682D
:10BAA000081D186008682E0605D5544E08276F2A11
:10BAB0001BD00A2719E06D06F7D580B2F5E74531AE
:10BAC0004E4E0A7018682268011D0068196015063C
:10BAD00021D5D30702D520231A432260102700283E
:10BAE00003D1202322689A4322602300002243339B
:10BAF0001A706368A360002B58DB0422216891430D
:10BB00002160002854D1029D002B5AD025003378A3
:10BB100042352B7055E05506DBD580B2D9E71A685F
:10BB20000D68101D4969186013682E0601D519604B
:10BB300002E06D06FBD519800023029D23614FE0D2
:10BB40001A68111D1960156800216268280000F04C
:10BB5000EDFC002801D0401B606063682361002376
:10BB6000029A13703CE023692A0004990398059D0A
:10BB7000A847431C3ED023689B0715D4079BE06869
:10BB8000984239DA180037E022000123193204996B
:10BB90000398059EB047431C2CD00135E368079AF3
:10BBA0009B1AAB42F0DCE9E70025F7E70028ADD0AF
:10BBB000029D3900FDF722FC735C013D2B700028CB
:10BBC000F7D1082F09D12368DB0706D563682269FE
:10BBD000934202DC3023013D2B70029B5B1B2361EF
:10BBE000059B07AA00932100049B0398FFF794FE8E
:10BBF000431CB8D10120404209B0F0BD01E400006F
:10BC000012E400000D4B70B51C680500A36B002BFF
:10BC10000FD1182000F06EFC094BA0630360094BA4
:10BC200001224360084B83600B2383810023026160
:10BC300043610022A36B1D615A6170BD800000202A
:10BC40000E33CDAB34126DE6ECDE0500124B10B5B1
:10BC50001C68A36B002B0FD1182000F04BFC0F4B7E
:10BC6000A06303600E4B012243600E4B83600B23E5
:10BC70008381002302614361A46B0B4A20696169DF
:10BC80000A4BFDF7F7FC012200238018594120617F
:10BC900061614800400810BD800000200E33CDAB2C
:10BCA00034126DE6ECDE05002D7F954C2DF45158D5
:10BCB0000CB430B5164B9DB00C1E1D6808DA8B23F2
:10BCC00001202B6040421DB030BC08BC02B01847B8
:10BCD000822302A99B008B810023029008619C4271
:10BCE00000D0631E8B604B6101235B42CB81209AA5
:10BCF00021AB2800019300F055FD431C01DA8B2392
:10BD00002B60002CDFD00023029A1370DBE7C046C3
:10BD1000800000200EB400B50B499CB01DAB029012
:10BD20000690079104910948094904CB05910068E0
:10BD300002A9019300F036FD0023029A13701CB093
:10BD400008BC03B01847C046FFFFFF7F80000020FB
:10BD50000802FFFF020010B51378541C002B05D118
:10BD6000CC5CD4540133002CFAD110BD2200F3E78F
:10BD7000C9B20378002B04D08B4200D17047013048
:10BD8000F7E74B42594149420840F7E702780B7800
:10BD9000002A03D0013001319A42F7D0D01A7047FF
:10BDA0000023C25C0133002AFBD1581E70470023D8
:10BDB00030B59A420AD0013AC45CCD5CAC4204D1A1
:10BDC000934202D00133002CF6D1631B180030BD22
:10BDD00030B50500002A00D130BD0C78013A6B1C4B
:10BDE0002C700131002C05D19A189A42F4D01C70A5
:10BDF0000133FAE71D00EDE710B50378002B0FD1F2
:10BE00000B785A4253415B42184010BD0023CA5C74
:10BE1000002AFAD0C45C944201D10133F7E7013023
:10BE20000378002BF2D11800EFE70000F0B51F00F7
:10BE30000E0087B00590019102920C98347800F0C2
:10BE4000EAFA082200194378751C134036D12D2CCC
:10BE500036D1B51C74780126002F62D0102F09D17D
:10BE6000302C07D120222B789343582B54D1102704
:10BE70006C7802352D4B3900F31818000393FDF749
:10BE8000BDFA049101210023494202008C461800AA
:10BE90002100303909291AD80C00A74223DD591C8A
:10BEA00009D06346824206D302D10499A14202DB43
:10BEB0000123784320182C780135E9E72E00BCE7F0
:10BEC0002B2C01D01E00C7E7B51C7478FAE72100BF
:10BED0004139192901D8373CDFE721006139192997
:10BEE00001D8573CD9E75A1C08D1059A233313606F
:10BEF000029B0398002B09D107B0F0BD002E00D0A3
:10BF00004042029A002AF7D0002B01D06B1E019309
:10BF1000029B019A1A60EFE73024002FAAD108276C
:10BF2000A8E7302C9ED00A27A4E7C046FFFFFF7F7A
:10BF300037B51300064A05001068046A002C00D1CA
:10BF4000044C0A0000942900FFF770FF3EBDC04674
:10BF500080000020E4000020F8B505000E00140069
:10BF6000002804D08369002B01D100F0C1F9224BD5
:10BF70009C422DD16C68A369A360A3891B0731D5AE
:10BF80002369002B2ED023682269F7B2981A6369BF
:10BF9000F6B2834205DC2100280000F03BF90028BE
:10BFA00026D1A3680130013BA36023685A1C22609C
:10BFB0001F706369834204D0A389DB071AD50A2E58
:10BFC00018D12100280000F025F9002812D00FE038
:10BFD0000A4B9C4201D1AC68CDE7094B9C42CAD1C7
:10BFE000EC68C8E72100280000F00CF80028CAD04F
:10BFF000012676423000F8BD44E4000064E400000D
:10C0000024E40000364B70B51D6806000C00002DBE
:10C0100005D0AB69002B02D1280000F069F9314B43
:10C020009C420FD16C680C23E25E93B219072DD4A9
:10C03000D90611D409230120336037331343A38178
:10C04000404270BD284B9C4201D1AC68EBE7274BC6
:10C050009C42E8D1EC68E6E75B0713D5616B0029E9
:10C0600008D023004433994202D0300000F06AFA2D
:10C07000002363632422A3899343A3810023636085
:10C08000236923600823A2891343A3812369002B1A
:10C090000BD1A0218022A389890092000B409342FA
:10C0A00003D02100300000F0E1F90123A289134000
:10C0B00011D00023A36063695B42A3610020236960
:10C0C0008342BED10C23E25E1306BAD5402313434C
:10C0D000A3810138B5E7920700D46369A360EDE757
:10C0E0008000002044E4000064E4000024E4000038
:10C0F00010B5062000F090FC012000F0CFFD0000FC
:10C10000F7B58A8905000C00130760D44B68002B33
:10C1100004DC0B6C002B01DC0020FEBDE76A002F65
:10C12000FAD000232E682B6080235B01216A1A401D
:10C1300034D0606DA3895B0706D56368C01A636B52
:10C14000002B01D0236CC01A0200216A00232800B2
:10C15000E76AB847A189431C06D12B681D2B30D84C
:10C160002B4ADA40D3072CD5002363602369236070
:10C17000CB0405D5431C02D12B68002B00D1606590
:10C18000616B2E600029C7D023004433994202D04E
:10C19000280000F0D7F900206063BEE701232800E3
:10C1A000B847431CC6D12B68002BC3D01D2B01D030
:10C1B000162B01D12E60AFE74023A2891343A38140
:10C1C000ABE740230B430120A3814042A5E70F6961
:10C1D000002FA1D00B680F60DB1B01930023920797
:10C1E00000D14B69A360019B002B00DC94E7019B0D
:10C1F0003A00216A2800A66AB047002803DC4023E1
:10C20000A2891343DFE7019B3F181B1A0193EAE75A
:10C21000010040200B6970B505000C00002B01D116
:10C22000002070BD002804D08369002B01D100F0EC
:10C230005FF80B4B9C4209D16C680C22A35E002B6B
:10C24000EED021002800FFF75BFFEAE7054B9C4298
:10C2500001D1AC68F1E7044B9C42EED1EC68ECE70D
:10C2600044E4000064E4000024E40000002310B56E
:10C27000040003604360836081814366C28103617F
:10C2800043618361190008225C30FFF7FFF9054B19
:10C2900024626362044BA362044BE362044B236396
:10C2A00010BDC04659CA000081CA0000B9CA0000CA
:10C2B000E5CA000010B5024900F08CF810BDC04678
:10C2C00015C2000070B568254A1E55430E002900AE
:10C2D000743100F081F9041E08D000212A000160A9
:10C2E00046600C30A0606832FFF7D0F9200070BDC6
:10C2F000836913B50400002B28D18364C3640365EC
:10C30000134B144A1B6882620193984201D10123A6
:10C310008361200000F020F86060200000F01CF82D
:10C32000A060200000F018F80022E060042160689E
:10C33000FFF79CFF01220921A068FFF797FF022267
:10C340001221E068FFF792FF0123A36113BDC046ED
:10C35000ECE30000B5C20000F8B51C4B07001E68F6
:10C36000B369002B02D13000FFF7C2FF4836B46832
:10C370007368013B04D53368002B07D03668F6E7B5
:10C380000C22A55E002D0DD06834F2E704213800A0
:10C39000FFF798FF30600028F0D10C2304003B60C9
:10C3A0002000F8BD20000A4B656625606560A56029
:10C3B000E36025616561A561082229005C30FFF713
:10C3C00065F96563A563A564E564E9E7ECE300004E
:10C3D0000100FFFFF7B50400070000260191483473
:10C3E000002C01D13000FEBD6368A5680093009B5E
:10C3F000013B009301D52468F2E7AB89012B08D9F2
:10C400000E22AB5E013304D029003800019B98470F
:10C4100006436835EBE7EC300068704770B50E00F6
:10C420001D000E23C95E96B01400002907DA002310
:10C430002B60B3891B0611D48023DB000FE06A4612
:10C4400000F088FB0028F2DBF022019B120213406F
:10C45000054A9B185A4253412B60EDE740230020C8
:10C46000236016B070BDC04600E0FFFFF7B502269E
:10C470008B8905000C00334206D02300473323602C
:10C48000236101236361F7BD01AB6A46FFF7C6FF75
:10C4900000990700280000F09FF8002808D10C221E
:10C4A000A35E9A05EFD4032293431E43A681E4E7DB
:10C4B0000F4BAB628023A28920601343A381009BB2
:10C4C00020616361019B002B0DD00E23E15E2800EB
:10C4D00000F052FB002806D00322A38993431A00E0
:10C4E00001231343A381A0893843A081CBE7C04631
:10C4F000B5C2000010B5034B0100186800F06CF8DD
:10C5000010BDC0468000002082B0002900D101A9E2
:10C51000101E06D0002B06D013780B601078431E37
:10C52000984102B0704702204042FAE7C9B282182F
:10C53000904201D10020704703788B42FBD001303C
:10C54000F6E7000070B50500002910D00C1F236825
:10C55000002B00DAE418280000F034FB1D4A1368B1
:10C56000002B05D163601460280000F02CFB70BD27
:10C57000A34209D9216860188342F3D118685B6827
:10C5800041182160EEE713005A68002A01D0A24248
:10C59000F9D919685818A0420BD120680918581801
:10C5A00019608242E0D110685268411819605A60DF
:10C5B000DAE7A04202D90C232B60D5E72168601886
:10C5C000824203D1106852684118216062605C6049
:10C5D000CAE7C0462C1C0020032370B5CD1C9D4328
:10C5E000083506000C2D1ED20C25A9421DD830009E
:10C5F00000F0E8FA254A14682100002919D1244CDA
:10C600002368002B03D1300000F0CAF92060290014
:10C61000300000F0C5F9431C2BD10C2330003360EF
:10C6200000F0D1FA03E0002DDFDA0C2333600020A4
:10C6300070BD0B685B1B19D40B2B03D90B60CC1896
:10C64000256003E04B688C420DD11360300000F090
:10C65000BAFA200007220B30231D9043C31AE7D0FB
:10C660005A42E250E4E763600C00EFE70C004968CF
:10C67000C3E70323C41C9C43A042E1D0211A30002D
:10C6800000F08EF9431CDBD1C7E7C0462C1C00200C
:10C69000301C0020F8B507000D001600002905D158
:10C6A0001100FFF799FF04002000F8BD002A03D114
:10C6B000FFF748FF3400F7E700F086FA2C00B0429D
:10C6C000F2D231003800FFF787FF041EECD02900BA
:10C6D0003200FEF7BFFF29003800FFF733FFE3E722
:10C6E000F0B58E6885B007000C00039201939E425E
:10C6F0003CD890238A89DB001A4234D0032509698B
:10C7000023685B1A0293636902985D43EB0F5D191E
:10C71000019B6D1001331B18AB4200D91D0053055E
:10C7200032D529003800FFF757FF061E09D10C2328
:10C730003B6040230120A28940421343A38105B0FE
:10C74000F0BD029A2169FEF785FFA389144A1A40B9
:10C7500080231343A381029B2661F618266065613E
:10C76000019EED1AA560019B9E4200D9019E3200F8
:10C7700003992068FEF777FFA36800209B1BA36046
:10C7800023689E192660DAE72A003800FFF782FF47
:10C79000061EE0D121693800FFF7D4FEC7E7C04686
:10C7A0007FFBFFFFF0B59FB0029005938B890F00D0
:10C7B00016001B0611D50B69002B0ED14021FFF787
:10C7C0000BFF38603861002805D10C23029A01382C
:10C7D00013601FB0F0BD40237B61002306AC636192
:10C7E000203363761033A37635002B78002B01D0ED
:10C7F000252B46D1AB1B04930CD032003900029894
:10C80000FFF76EFF431C00D1AEE06269049B9446C3
:10C81000634463612B78002B00D1A5E00122002343
:10C820005242626002A9543252186E1C2360E360C7
:10C83000A3601370A365317805225448FFF776FE94
:10C84000751C00281FD12268D30604D5532302A9E2
:10C850005B1820211970130704D5532302A95B1814
:10C860002B21197033782A2B16D0350000210A208D
:10C87000E3682A786E1C303A092A4ED9002918D06C
:10C8800010E00135B1E7414B2268C01A0123834013
:10C89000134323602E00CEE7059B191D1B680591ED
:10C8A000002B01DB099304E05B42E36002231343A6
:10C8B00023602B782E2B0AD16B782A2B35D1059B40
:10C8C00002351A1D1B680592002B2BDB0793304E97
:10C8D000297803223000FFF729FE002806D04023E4
:10C8E000801B834022680135134323602978062288
:10C8F00028486E1C2176FFF719FE00283CD0264BF5
:10C90000002B25D10722059B07339343083305935A
:10C910006369039A9B18636166E7434301219B188F
:10C920003500A6E701235B42D0E700230A201A0066
:10C930000135636029786E1C3039092903D9002B31
:10C94000C5D00792C3E74243012352183500F1E7EF
:10C9500005AB00933A00114B2100029800E000BFA4
:10C960000390039B0133D3D1BB890B985B0600D4A2
:10C970002FE7012040422CE705AB00933A00074B1C
:10C9800021000298FFF736F8EAE7C046F0E300001E
:10C99000F6E30000FAE3000000000000E1C600003A
:10C9A000002370B5064C05000800236000F060F914
:10C9B000431C03D12368002B00D02B6070BDC04600
:10C9C000C02F002070B504000D001F2904D91623C4
:10C9D00003600120404270BD436C002B04D08A00EC
:10C9E0009B181A68002A08D1200000F031F82A00AC
:10C9F0000100200000F01AF8EDE70020012AEAD03B
:10CA0000511C03D1162301302360E4E700242800E1
:10CA10001C6090472000DEE710B5034B010018684A
:10CA2000FFF7D0FF10BDC04680000020002370B586
:10CA3000064C050008001100236000F001F9431CBA
:10CA400003D12368002B00D02B6070BDC02F0020C5
:10CA500010B500F0E5F810BD70B50C000E25495F6B
:10CA600000F0BAF8002803DB636D1B18636570BD26
:10CA7000A389024A1340A381F9E7C046FFEFFFFFF5
:10CA8000F8B51F008B8905000C001600DB0505D5E5
:10CA90000E23C95E0022022300F080F8A389054A14
:10CAA00028001340A38132000E23E15E3B0000F01A
:10CAB0002BF8F8BDFFEFFFFF70B50C000E25495FA6
:10CAC00000F06CF8A389421C03D1054A1340A381EE
:10CAD00070BD802252011343A3816065F8E7C04610
:10CAE000FFEFFFFF10B50E23C95E00F021F810BD67
:10CAF0000B1E04D0FF2A04D98A2303608B3B180045
:10CB000070470A700123FAE770B5050008001100AC
:10CB10000022064C22601A0000F0B8F8431C03D132
:10CB20002368002B00D02B6070BDC046C02F0020B2
:10CB3000002370B5064C05000800236000F060F883
:10CB4000431C03D12368002B00D02B6070BDC0466E
:10CB5000C02F0020002370B5064C0500080011000E
:10CB6000236000F055F8431C03D12368002B00D04C
:10CB70002B6070BDC02F0020002370B5064C05004F
:10CB80000800236000F054F8431C03D12368002BF5
:10CB900000D02B6070BDC046C02F002070B50500CE
:10CBA000080011000022064C22601A0000F050F824
:10CBB000431C03D12368002B00D02B6070BDC046FE
:10CBC000C02F0020704770470B1F1B68181F002BD9
:10CBD00001DA0B58C018704770B505000800110045
:10CBE0000022064C22601A0000F03AF8431C03D1E0
:10CBF0002368002B00D02B6070BDC046C02F0020E2
:10CC000058220120014B40421A607047C02F00207B
:10CC100058220120014B40421A607047C02F00206B
:10CC200058220120014B40421A607047C02F00205B
:10CC30005822024B00201A607047C046C02F0020C7
:10CC400058220120014B40421A607047C02F00203B
:10CC500058220120014B40421A607047C02F00202B
:10CC600058220120014B40421A607047C02F00201B
:10CC7000044A1368002B00D1034B181810601800E9
:10CC80007047C046341C0020C82F002058220120C5
:10CC9000014B40421A607047C02F0020FEE7C0469B
:10CCA000F8B5C046F8BC08BC9E467047F8B5C0460B
:10CCB000F8BC08BC9E4670476461746100000000C7
:10CCC0003CCD0000EF01000045CD0000E302000074
:10CCD0004DCD00000509000054CD0000150A0000EC
:10CCE00059CD00002D05000064CD00005303000065
:10CCF00069CD00006D0C000075CD00001F02000022
:10CD00007FCD00000D0800008DCD0000B9060000A9
:10CD10009ACD0000EF04000072616E646F6D0061D7
:10CD20006C6C006C6173740066616C736500747286
:10CD3000756500252E3135732E2E2E006D616B65C5
:10CD40004C697374006164644C6173740064656C55
:10CD5000657465006A6F696E00636F707946726F03
:10CD60006D546F0066696E64006A6F696E53747209
:10CD7000696E677300756E69636F646541740075F1
:10CD80006E69636F6465537472696E67006E657770
:10CD900042797465417272617900667265654D65AC
:10CDA0006D6F7279000000000DCE0000D5100000FC
:10CDB00012CE0000F31000004DCD0000F71000006F
:10CDC00018CE0000D910000022CE0000FB10000099
:10CDD0002BCE0000FF10000035CE00000311000034
:10CDE00040CE0000071100004CCE0000DD10000016
:10CDF00055CE0000EB1000005FCE0000E1100000F7
:10CE00006ACE0000EF10000066696C65006F706507
:10CE10006E00636C6F736500656E644F6646696C87
:10CE20006500726561644C696E650072656164429B
:10CE30007974657300617070656E644C696E65002D
:10CE4000617070656E6442797465730066696C65C3
:10CE500053697A650073746172744C697374006EFF
:10CE6000657874496E4C6973740073797374656D79
:10CE7000496E666F00000000341300004413000088
:10CE80005E130000DC130000141400004A140000BC
:10CE900082140000A8140000E4140000261500000D
:10CEA0007C150000C01500002C1600007416000050
:10CEB0009A160000D2160000181700003E17000056
:10CEC0006C1700009A170000DC17000060180000C3
:10CED000281900009E190000081A0000541A0000CA
:10CEE000741A0000961A0000481B00008E1B0000F8
:10CEF000061C0000341C0000641C00009A1C00008A
:10CF0000021D0000861D0000CC1D0000141E000044
:10CF10008A1E0000001F0000481F00008E1F000036
:10CF2000C41F00000A2000005020000098200000CC
:10CF3000F42000004821000086210000F0210000BC
:10CF4000262200006E220000B6220000FE22000011
:10CF50003823000080230000C82300003225000091
:10CF60006C170000D21600003024000034130000BB
:10CF70006624000092240000D0240000FC2400005D
:10CF80003413000034130000341300003413000085
:10CF9000AC250000EE2500003426000084260000A9
:10CFA000B0260000002700002627000054270000BC
:10CFB000341300003413000078270000A827000075
:10CFC000D82700000E28000038280000A428000000
:10CFD000CE280000F62800001E2900004E2900007F
:10CFE0007E290000A8290000D2290000022A0000A2
:10CFF0002C2A000034130000341300003413000006
:10D0000034130000341300005C2A0000882A00005A
:10D01000B42A0000E02A00000C2B0000422B000084
:10D02000782B0000AE2B0000E42B0000102C000039
:10D030003C2C0000722C000034130000341300005C
:10D0400034130000341300003413000034130000C4
:10D0500034130000341300003413000034130000B4
:10D0600034130000341300003413000034130000A4
:10D07000A82C0000DE2C00005B2564206974656D1F
:10D08000206C6973745D002825642062797465736F
:10D090002900286F626A65637420747970653A208C
:10D0A00025642900537461636B20756E6465726634
:10D0B0006C6F7700626F6F6C65616E006E756D628C
:10D0C000657200737472696E67006C6973740062D4
:10D0D00079746520617272617900000007000000B8
:10D0E000030000003DD10000012E000045D10000EA
:10D0F000B12E00004ED100005B2F000057D1000080
:10D10000052E000060D100005F2F000068D10000F4
:10D11000492F00001C000000010000000200000078
:10D1200004000000050000000600000010000000E0
:10D130001100000043616C6C696F70650068617379
:10D14000546F6E6500706C6179546F6E6500686134
:10D1500073536572766F00736574536572766F00F2
:10D16000646163496E6974006461635772697465D0
:10D1700000474320746F6F6B2025642075736563CF
:10D18000733B206672656520256420776F72647337
:10D19000003C496E74656765723E003C4C6973746F
:10D1A0003E003C4F626A6563743E003C42797465A0
:10D1B00041727261793E000D0A564D2050616E69D0
:10D1C000633A2025730D0A006D6973630000000047
:10D1D00005D20000313C00000ED20000C13B00002F
:10D1E00012D20000153B00001AD20000BB3A00002A
:10D1F00024D20000513A000030D200005339000020
:10D200006E756C6C00686578546F496E7400736954
:10D210006E006A736F6E476574006A736F6E436F5A
:10D22000756E74006A736F6E56616C75654174003B
:10D230006A736F6E4B6579417400000098D20000EC
:10D240009D3C0000A0D20000A13C0000AAD200003A
:10D25000BF3C0000B3D20000C93C0000BED20000B9
:10D26000D33C0000CAD20000DD3C0000DFD2000049
:10D27000E73C0000F4D20000F13C000000D30000C5
:10D28000FB3C000010D30000AB3C00001CD30000AE
:10D29000B53C00006E6574006861735769466900AB
:10D2A0007374617274576946690073746F7057695B
:10D2B00046690077696669537461747573006D79A6
:10D2C0004950416464726573730068747470536587
:10D2D0007276657247657452657175657374007214
:10D2E0006573706F6E64546F4874747052657175B5
:10D2F0006573740068747470436F6E6E6563740058
:10D30000687474704973436F6E6E6563746564000E
:10D3100068747470526571756573740068747470A4
:10D32000526573706F6E7365000D0E0F04050C0B64
:10D330000A06070809000000000008080800080A9B
:10D340004A4000000A5FEA5FEA0ED92ED36E193216
:10D350004489330C924C924D080800000004880860
:10D3600008040804848488000A448A4000048EC4A7
:10D3700080000000048800000EC0000000000800CB
:10D3800001224488100C9252524C048C84848E1CCE
:10D39000824C901E1EC244924C06CA525FE21FF09D
:10D3A0001EC13E02448ED12E1FE24488100ED12EA3
:10D3B000D12E0ED12EC4880008000800000480047D
:10D3C000880244880482000EC00EC008048244888B
:10D3D0000ED126C0040ED135B36C0C925ED2521C15
:10D3E000925C925C0ED010100E1C9252525C1ED0B9
:10D3F0001C901E1ED01C90100ED013712E12525E67
:10D40000D2521C8808081C1FE242524C1254981435
:10D4100092101010101E113B75B131113935B371D6
:10D420000C9252524C1C925C90100C92524C861CE6
:10D43000925C92510ED00C825C1FE4848484125260
:10D4400052524C1131312A44113135BB7112524CB8
:10D450009252112A4484841EC488101E0EC80808E3
:10D460000E10080482410EC242424E048A4000005F
:10D47000000000001F0804800000000ED2524F1070
:10D48000101C925C000ED0100E02424ED24E0C9236
:10D490005C900E06C81C88080ED24EC24C10101CA0
:10D4A00092520800080808024002424C10149814D6
:10D4B000920808080806001B75B131001C925252F0
:10D4C000000C92524C001C925C90000ED24EC20096
:10D4D0000ED010100006C8049808080EC8070012E5
:10D4E00052524F0011312A4400113135BB00124C09
:10D4F0008C9200112A4498001EC4881E06C48C8495
:10D5000086080808080818080C881800000C8360B2
:10D510000000000001000000020000000300000005
:10D5200004000000050000000600000007000000E5
:10D5300008000000090000000A0000000B000000C5
:10D540000C0000000D0000000E0000000F000000A5
:10D55000100000001200000014000000160000007F
:10D56000180000001A0000001C0000001E0000004F
:10D570002000000023000000260000002900000019
:10D580002C0000002F0000003200000036000000D8
:10D590003A0000003E00000042000000460000008B
:10D5A0004B00000050000000550000005A00000031
:10D5B00061000000680000006F00000076000000BD
:10D5C0007D000000840000008B000000920000003D
:10D5D00099000000A0000000A7000000AE000000BD
:10D5E000B5000000BC000000C3000000CA0000003D
:10D5F000D1000000D8000000DF000000E6000000BD
:10D60000ED000000F4000000FB000000FF0000003F
:10D6100060D600001D3D00006BD60000B94200003E
:10D6200075D60000E13E000082D6000029410000CE
:10D6300089D600007941000092D60000C94100005F
:10D640009ED60000C1400000AFD60000513F000050
:10D65000BCD6000051400000646973706C617900B1
:10D660006C696768744C6576656C006D62446973BB
:10D67000706C6179006D62446973706C61794F669A
:10D6800066006D62506C6F74006D62556E706C6FE9
:10D6900074006D62447261775368617065006D62F9
:10D6A0005368617065466F724C6574746572006E84
:10D6B000656F506978656C53656E64006E656F5078
:10D6C0006978656C53657450696E004E6F7420659F
:10D6D0006E6F75676820726F6F6D206576656E205E
:10D6E000616674657220636F6D70616374696F6EDB
:10D6F00000436F6D70616374656420466C6173688C
:10D7000020636F64652073746F72650A25642062FC
:10D71000797465732075736564202825642525292F
:10D72000206F6620256400426164207265636F7219
:10D730006420666F756E6420647572696E67206917
:10D740006E697469616C697A6174696F6E002564D1
:10D750002025642025642028256420776F72647357
:10D7600029002564207265636F7264732C20256420
:10D7700020776F7264732C206D6178494420256492
:10D780002C20636F6D70616374696F6E20637963C1
:10D790006C657320256400526573746F7265642034
:10D7A00025642073637269707473005374617274BA
:10D7B000656400726164696F000000004CD800006D
:10D7C000914C000059D800002D4F000069D800008E
:10D7D000AD4E000077D80000C150000082D8000094
:10D7E000B94C000092D80000414D0000A6D80000BE
:10D7F000294D0000B5D80000A3520000C1D8000098
:10D8000021520000CAD80000C5510000D5D8000040
:10D810000D510000E0D8000049510000E9D8000097
:10D820007D510000F2D80000C94C000001D9000071
:10D83000A94C00000AD90000D94C00006E6F6E653B
:10D84000006F746865720070616972006469736169
:10D85000626C65526164696F006D657373616765C1
:10D860005265636569766564007061636B657452C7
:10D87000656365697665007061636B657453656E99
:10D8800064007265636569766564496E7465676591
:10D89000720072656365697665644D65737361676F
:10D8A0006554797065007265636569766564537463
:10D8B00072696E670073656E64496E746567657240
:10D8C0000073656E64506169720073656E645374B1
:10D8D00072696E67007365744368616E6E656C0093
:10D8E00073657447726F757000736574506F7765F8
:10D8F00072007369676E616C537472656E677468E9
:10D90000006465766963654944006C6173744D65B4
:10D910007373616765494400556E6B6E6F776E2057
:10D920007072696D6974697665205B25733A257339
:10D930005D00000000000000963007772C610EEEBD
:10D94000BA51099919C46D078FF46A7035A563E956
:10D95000A395649E3288DB0EA4B8DC791EE9D5E07D
:10D9600088D9D2972B4CB609BD7CB17E072DB8E77C
:10D97000911DBF906410B71DF220B06A4871B9F3D1
:10D98000DE41BE847DD4DA1AEBE4DD6D51B5D4F40A
:10D99000C785D38356986C13C0A86B647AF962FD6F
:10D9A000ECC9658A4F5C0114D96C0663633D0FFABC
:10D9B000F50D088DC8206E3B5E10694CE44160D5C2
:10D9C000727167A2D1E4033C47D4044BFD850DD2AC
:10D9D0006BB50AA5FAA8B5356C98B242D6C9BBDBBF
:10D9E00040F9BCACE36CD832755CDF45CF0DD6DCBA
:10D9F000593DD1ABAC30D9263A00DE518051D7C861
:10DA00001661D0BFB5F4B42123C4B3569995BACFEB
:10DA10000FA5BDB89EB802280888055FB2D90CC60C
:10DA200024E90BB1877C6F2F114C6858AB1D61C185
:10DA30003D2D66B69041DC760671DB01BC20D298A4
:10DA40002A10D5EF8985B1711FB5B606A5E4BF9F31
:10DA500033D4B8E8A2C9077834F9000F8EA8099624
:10DA600018980EE1BB0D6A7F2D3D6D08976C64918F
:10DA7000015C63E6F4516B6B62616C1CD8306585A8
:10DA80004E0062F2ED95066C7BA5011BC1F4088285
:10DA900057C40FF5C6D9B06550E9B712EAB8BE8BC6
:10DAA0007C88B9FCDF1DDD62492DDA15F37CD38C4F
:10DAB000654CD4FB5861B24DCE51B53A7400BCA34D
:10DAC000E230BBD441A5DF4AD795D83D6DC4D1A47F
:10DAD000FBF4D6D36AE96943FCD96E34468867AD56
:10DAE000D0B860DA732D0444E51D03335F4C0AAAF5
:10DAF000C97C0DDD3C710550AA41022710100BBEF8
:10DB000086200CC925B56857B3856F2009D466B93E
:10DB10009FE461CE0EF9DE5E98C9D9292298D0B073
:10DB2000B4A8D7C7173DB359810DB42E3B5CBDB720
:10DB3000AD6CBAC02083B8EDB6B3BF9A0CE2B603A1
:10DB40009AD2B1743947D5EAAF77D29D1526DB0456
:10DB50008316DC73120B63E3843B64943E6A6D0DA1
:10DB6000A85A6A7A0BCF0EE49DFF099327AE000AEC
:10DB7000B19E077D44930FF0D2A3088768F2011E7F
:10DB8000FEC206695D5762F7CB67658071366C1916
:10DB9000E7066B6E761BD4FEE02BD3895A7ADA1037
:10DBA000CC4ADD676FDFB9F9F9EFBE8E43BEB71718
:10DBB000D58EB060E8A3D6D67E93D1A1C4C2D838A2
:10DBC00052F2DF4FF167BBD16757BCA6DD06B53F08
:10DBD0004B36B248DA2B0DD84C1B0AAFF64A033647
:10DBE000607A0441C3EF60DF55DF67A8EF8E6E31C6
:10DBF00079BE69468CB361CB1A8366BCA0D26F250F
:10DC000036E2685295770CCC03470BBBB91602225B
:10DC10002F260555BE3BBAC5280BBDB2925AB42B70
:10DC2000046AB35CA7FFD7C231CFD0B58B9ED92C85
:10DC30001DAEDE5BB0C2649B26F263EC9CA36A75EA
:10DC40000A936D02A906099C3F360EEB85670772A1
:10DC500013570005824ABF95147AB8E2AE2BB17B08
:10DC6000381BB60C9B8ED2920DBED5E5B7EFDC7C8F
:10DC700021DFDB0BD4D2D38642E2D4F1F8B3DD68E6
:10DC80006E83DA1FCD16BE815B26B9F6E177B06FE1
:10DC90007747B718E65A0888706A0FFFCA3B0666CE
:10DCA0005C0B0111FF9E658F69AE62F8D3FF6B615B
:10DCB00045CF6C1678E20AA0EED20DD75483044EFD
:10DCC000C2B30339612667A7F71660D04D4769498B
:10DCD000DB776E3E4A6AD1AEDC5AD6D9660BDF409E
:10DCE000F03BD83753AEBCA9C59EBBDE7FCFB24751
:10DCF000E9FFB5301CF2BDBD8AC2BACA3093B35336
:10DD0000A6A3B4240536D0BA9306D7CD2957DE543E
:10DD1000BF67D9232E7A66B3B84A61C4021B685D17
:10DD2000942B6F2A37BE0BB4A18E0CC31BDF055A90
:10DD30008DEF022D416C6C207461736B73207374D2
:10DD40006F707065640076313035002025732025B2
:10DD500073004D656D6F727920636C6561726564E7
:10DD6000004E6F2066726565207461736B20656E6E
:10DD70007472696573000000D0DD000081660000E8
:10DD8000DDDD0000D9650000E9DD0000A9650000C7
:10DD9000EFDD0000B9650000F5DD0000C965000099
:10DDA000FBDD0000DD61000005DE0000F565000020
:10DDB0000DDE0000F963000016DE0000396200008D
:10DDC0001EDE00006163000073656E736F72730086
:10DDD000616363656C65726174696F6E0074656D13
:10DDE00070657261747572650074696C7458007442
:10DDF000696C74590074696C745A00746F75636847
:10DE0000526561640069326352656164006932631E
:10DE100057726974650072656164444854006D69A5
:10DE200063726F70686F6E6500000000A0DE000016
:10DE300039670000AEDE00003D670000B7DE00007D
:10DE400049670000C1DE00004D670000CADE000027
:10DE500051670000CFDE000055670000D4DE0000EF
:10DE600059670000E0DE00005D670000E7DE0000AB
:10DE700061670000F0DE000065670000F5DE00006D
:10DE80006967000000DF00006D6700000ADF000026
:10DE90004167000014DF00004567000074667400ED
:10DEA000656E61626C65446973706C617900676569
:10DEB0007457696474680067657448656967687455
:10DEC00000736574506978656C006C696E650072EA
:10DED00065637400726F756E646564526563740087
:10DEE000636972636C6500747269616E676C65006A
:10DEF0007465787400746674546F75636865640043
:10DF0000746674546F7563685800746674546F75E2
:10DF100063685900746674546F75636850726573F2
:10DF20007375726500766172730000004CDF00004B
:10DF3000FD6B000056DF0000DD6B00005FDF0000BE
:10DF4000B96B00006BDF0000456B00007661724525
:10DF50007869737473007661724E616D65640073E5
:10DF600065745661724E616D6564007661724E61D2
:10DF70006D65466F72496E6465780057656C636FB6
:10DF80006D6520746F204D6963726F426C6F636BB7
:10DF9000732100705F73706920213D204E554C4CF9
:10DFA000002F686F6D652F6769742F2E706C617418
:10DFB000666F726D696F2F7061636B616765732F38
:10DFC0006672616D65776F726B2D61726475696ED3
:10DFD0006F6E6F726469636E7266352F6C69627200
:10DFE00061726965732F5350492F5350492E6370E6
:10DFF0007000535049436C6173733A3A535049432C
:10E000006C617373284E52465F5350495F54797068
:10E01000652A2C2075696E74385F742C2075696EC2
:10E0200074385F742C2075696E74385F7429000031
:10E030000000000000000000096E0000C56D000037
:10E04000EB6D0000F56D0000FF6D0000E96D000054
:10E0500000000000010000000200000016000000A7
:10E06000040000000500000006000000070000009A
:10E0700008000000090000000A0000000B0000007A
:10E080000C0000000D0000000E0000000F0000005A
:10E090001A0000001B000000140000001300000024
:10E0A0001100000017000000100000001C0000001C
:10E0B0001D0000001E0000001200000015000000FE
:10E0C000030000001800000019000000000000001C
:10E0D00000000000E1720000497B00006173000055
:10E0E000757300006B730000DD720000D1720000D8
:10E0F00081730000FD720000CD720000000000007E
:10E10000000000000000304300000000000030C3A9
:10E110007371727400000000FB21F93FFB2109407C
:10E120007CD91240FB2119407A6A1F407CD92240D9
:10E13000BBFD2540FB2129403A462C407A6A2F40FE
:10E140005C4731407CD932409C6B3440BBFD35404C
:10E15000DB8F3740FB2139401BB43A403A463C4004
:10E160005AD83D407A6A3F404C7E40405C4741402F
:10E170006C1042407CD942408CA243409C6B44408E
:10E18000AC344540BBFD4540CBC64640DB8F4740E5
:10E19000EB584840FB21494083F9A200444E6E00F1
:10E1A000FC291500D1572700DD34F50062DBC000E3
:10E1B0003C999500419043006351FE00BBDEAB00EB
:10E1C000B761C5003A6E2400D24D42004906E00016
:10E1D00009EA2E001C92D100EB1DFE0029B11C00A3
:10E1E000E83EA700F535820044BB2E009CE9840080
:10E1F000B4267000417E5F00D69139005383390008
:10E200009CF439008B5F840028F9BD00F81F3B00A7
:10E21000DEFF97000F980500112FEF000A5A8B00C0
:10E220006D1F6D00CF7E360009CB2700464FB7002B
:10E230009E663F002DEA5F00BA277500E5EBC70038
:10E240003D7BF100F739070092528A00FB6BEA0030
:10E250001FB15F00085D8D00300356007BFC460057
:10E26000F0AB6B0020BCCF0036F49A00E3A91D0090
:10E270005E619100081BE60085996500A0145F00AF
:10E280008D40680080D8FF0027734D0006063100DE
:10E29000CA561500C9A873007BE260006B8CC000F1
:10E2A00000000040FB21F93F000000002D44743EB7
:10E2B000000000809846F83C0000006051CC783B9C
:10E2C00000000080831BF0390000004020257A38D0
:10E2D000000000802282E336000000001DF3693553
:10E2E000020000000300000004000000060000001F
:10E2F000C09700006A9700006A9700009898000095
:10E3000066970000669700008E98000098980000BD
:10E31000669700008E9800006697000098980000AD
:10E320009C9800009C9800009C980000A498000015
:10E330009CA200000EA1000052A10000B6A00000A7
:10E3400052A1000042A2000052A10000B6A00000AD
:10E350000EA100000EA1000042A20000B6A0000025
:10E36000AEA00000AEA00000AEA0000050A20000D1
:10E37000C4A90000C6A80000C6A80000E4AB0000C5
:10E38000C0A80000C0A80000CCAB0000E4AB0000B7
:10E39000C0A80000CCAB0000C0A80000E4AB0000A7
:10E3A000DAAB0000DAAB0000DAAB0000E8AB00004B
:10E3B0002C2066756E6374696F6E3A20006173730A
:10E3C000657274696F6E2022257322206661696C04
:10E3D00065643A2066696C6520222573222C206CC6
:10E3E000696E65202564257325730A00840000206A
:10E3F000232D302B2000686C4C006566674546472E
:10E4000000303132333435363738394142434445B0
:10E41000460030313233343536373839616263641F
:10E420006566000000000000000000000000000021
:10E4300000000000000000000000000000000000DC
:10E4400000000000000000000000000000000000CC
:10E4500000000000000000000000000000000000BC
:10E4600000000000000000000000000000000000AC
:10E47000000000000000000000000000000000009C
:10E48000000000004300504F534958000020202056
:10E490002020202020202828282828202020202054
:10E4A0002020202020202020202020202088101024
:10E4B0001010101010101010101010101004040480
:10E4C000040404040404041010101010101041413E
:10E4D000414141410101010101010101010101012C
:10E4E0000101010101010101101010101010424240
:10E4F00042424242020202020202020202020202FC
:10E50000020202020202020210101010200000009B
:10E5100000000000000000000000000000000000FB
:10E5200000000000000000000000000000000000EB
:10E5300000000000000000000000000000000000DB
:10E5400000000000000000000000000000000000CB
:10E5500000000000000000000000000000000000BB
:10E5600000000000000000000000000000000000AB
:10E57000000000000000000000000000000000009B
:10E58000000000000000000000000000000000008B
:04E590000000000087
:08E59400741BFF7F0100000071
:10E59C00FFFFFFFFD007000001000000E803DC05CF
:10E5AC00DC05DC05DC050000FFFFFFFFFFFFFFFFC4
:10E5BC001800000019FCFFFFFFFFFFFF0024F40010
:10E5CC000200000003000000FFFFFFFF000000003E
:10E5DC00010000000000020001000000FFFFFFFF2F
:10E5EC000000000002000000000004000200000017
:10E5FC00FFFFFFFF00000000030000000000080008
:10E60C00030000000A0000000800000001000000E8
:10E61C00840000200000000044E4000064E40000DA
:10E62C0024E40000000000000000000000000000D6
:10E63C0000000000000000000000000000000000CE
:10E64C0000000000000000000000000000000000BE
:10E65C0000000000000000000000000000000000AE
:10E66C00000000000000000000000000000000009E
:10E67C00000000004300000000000000000000004B
:10E68C00000000000000000000000000000000007E
:10E69C00000000004300000000000000000000002B
:10E6AC00000000000000000000000000000000005E
:10E6BC00000000004300000000000000000000000B
:10E6CC00000000000000000000000000000000003E
:10E6DC0000000000430000000000000000000000EB
:10E6EC00000000000000000000000000000000001E
:10E6FC0000000000430000000000000000000000CB
:10E70C0000000000000000000000000000000000FD
:10E71C0000000000430000000000000000000000AA
:10E72C0000000000000000000000000000000000DD
:10E73C00000000004300000000000000000000008A
:10E74C0000000000000000000000000000000000BD
:10E75C0000000000F1CA000009C500000000000024
:10E76C008CE400003ACD0000C7D10000C7D10000F6
:10E77C00C7D10000C7D10000C7D10000C7D100002D
:10E78C00C7D10000C7D10000C7D10000FFFFFFFFB9
:10E79C00FFFFFFFFFFFFFFFFFFFF000001004153E2
:10E7AC004349490000000000000000000000000088
:10E7BC0000000000000000000000000000004153B9
:10E7CC004349490000000000000000000000000068
:10E7DC00000000000000000000000000000000002D
:10E7EC00E9000000956D0000057100002D76000019
:04E7FC00C100000058
:04000003000071A1E7
:00000001FF
